:100000000100000000000000000400000094511AEC
:100010001CF09FE51CF09FE51CF09FE51CF09FE5A0
:100020001CF09FE51CF09FE51CF09FE51CF09FE590
:100030000F440F12C42E0400602E0400702E040022
:10004000742E0400842E0400942E0400A42E0400B8
:10005000B02E0400000000EA5BEC00EA28008FE20A
:10006000000C90E800A08AE000B08BE001704AE24A
:100070000B005AE154EC000A0F00BAE814E04FE21A
:10008000010013E303F0471013FF2FE1EC3C0400E1
:100090003C3D04000030A0E30040A0E30050A0E39A
:1000A0000060A0E3102052E27800A128FCFFFF8A44
:1000B000822EB0E13000A128003081451EFF2FE1E3
:1000C00004309FE503308FE013FF2FE129B50300D3
:1000D000002070470200144810B50068682109F339
:1000E0006AF910BD10B5104C206800280CD101F041
:1000F000E1FB20600D4A2021A06009F35CF90C4A65
:100100006068202109F357F910BD10B5064C20682E
:10011000002808D00022132109F34DF9206809F3C3
:100120002EF90020206010BD00000004F9B6030085
:1001300035B7030010B542F00CEF05F33FF900208E
:1001400010BD10B5EF480C00FFF7C4FFEE49486B37
:1001500002229043486321000A2042F06CEF012004
:1001600010BD70B50D0003F029FF0400E548401CE8
:10017000FFF7B0FFE549E0074C6002D029000520F9
:1001800015E0A00702D52900062010E0600702D57F
:10019000290007200BE0200702D52900082006E0EF
:1001A000E00602D52900092001E02900002042F0E4
:1001B00042EF012070BDF1B50020D5490E68D54F42
:1001C000340005000AE0E10706D0A9007A58002AA9
:1001D00002D000993000904764086D1C002CF2D1C9
:1001E000012807D0C7481938FFF774FF009900208D
:1001F00042F020EFF8BDC54910B5886005F079FBE5
:1002000010BD202800D3FEE7C24A80001358002BFF
:1002100000D0FEE7115000207047BE4A0021800048
:1002200011500800704702688368C16810001847C1
:1002300070B5052804D2B84D84002B59002B01D08D
:10024000012070BD2C23B44E4343DC3E9B192B513F
:1002500035000401F03528516019C2608160002129
:100260004160AE4919615861002070BDFEB50E00B5
:100270001700052815D2A8490201143155186968DC
:10028000A54B840000290DD101220197009602920E
:1002900018594369026906F373FC002801D1012053
:1002A0006860FEBD18591D0006F3A6FC28593A00E7
:1002B000310006F353FC285906F340FCFEBD934978
:1002C00070B50878401C0006000E08700121490432
:1002D0004018FFF7FFFE8C4D6C6AE00705D003F372
:1002E0006CE909F3BBF8A81768628D4EA00709D521
:1002F0002020F0600221C9436962B1680143B16006
:1003000009F3A4F8600705D5A86A04218843A86208
:1003100009F3C5FB20070AD5A86A08218843A8620B
:100320008020F060C9436962B1680143B160012077
:1003300070BD70B501247A4D8440EC6000203CF023
:10034000BAFDA8682043A860012070BD0121744A4D
:10035000814010B5D1600D3800D5FEE7022800DBE2
:10036000FEE7704C00238000041923606D4C40347C
:1003700000190362906808439060012010BD70B5B9
:100380000125674E8540F56003F0F0FD040040054F
:1003900032D509F064FA402802D103201CF014FD84
:1003A00002F0FBFD002815D002F08DFC002809D0DA
:1003B00029201CF009FD012120008902084003F0DA
:1003C000E0FD19E002F004FD002815D032201CF0F9
:1003D000FBFC11E00AF044FB00280DD011F020F9DD
:1003E000002809D01AF091FD002805D01AF023FB4F
:1003F000002801D111F058F9600708D504F066FD16
:1004000020000421084003F0BCFD04F03D5AE150F7
:1004100001000000FC030000000400005AEF5E131E
:10042000A4FD200003F0BCFDB0682843B0600120AB
:1004300070BDF8B5414DEC68E00702D0A817E86040
:100440000440200606D58020C043E8608020844315
:1004500003F0B5FD200407D50126F603300003F0B4
:10046000AEFDF043E860B4436003400F06D00720C0
:10047000000421000140C943E96084430B262000A9
:1004800036053040070005D0380002F065FBF84320
:10049000E860B443E000400F09D00727BF062600FC
:1004A0003E40300002F0EAFAF043E860BC43E00668
:1004B0000FD51020C043E8601020844303F0AEFE47
:1004C000002806D010F01AFA002802D0102002F0FE
:1004D000D3F9002C06DA0120C00702F0EAFA184826
:1004E000E860044081200003044205D0200002F0AF
:1004F00081F9200005F0A2FE0E498868012212054C
:1005000010438860F8BD0B4B0122120510B5DA606C
:10051000FFF78FFF012010BD5A000100003400805A
:10052000140000040031008064C40004542C000452
:10053000170200000030008040E800808022008028
:10054000FFFFFF7F70B52024048146690419B67946
:10055000267040690025C0796070080A21716071B9
:10056000100AA271E071180AA370E070F948406A9D
:10057000C030807FE074280013F0DCFB2878207600
:1005800013F0CEFB6076200070BDFFB581B0002275
:1005900006000D000398417800780F0207432037CA
:1005A00038003A300104EC48090C1BF323F804002E
:1005B00037D038001A30A0802020666120812018B2
:1005C0001A2100901AF354EB3B04049A1B0C1A21D5
:1005D0002000FFF7B7FF002D12D028892E002881B8
:1005E0001C360B20072130567156401A3EF0B9F9DF
:1005F00000990873072030563EF0A6F90099487319
:100600003A202081039920183A001AF36CEA00215D
:1006100020003BF04AF9207B202805D120003BF048
:1006200021F9002005B0F0BD202020813FF043F9E2
:10063000002802D005201CF0D1FB3BF0D7F8C84BB6
:100640000500C64821001C68002200680523A04759
:1006500028003BF0CFF80120E4E7FFB501209040EF
:1006600004060E0083B003991120240E40010F18D8
:10067000F879150020422FD1FF229132462301A99B
:1006800002A811F02AFD002826D0F879172120436E
:10069000F871019C103420001AF3EAEA0698002849
:1006A00001D1052000E00D20607225722000627AE1
:1006B0000C990A301AF316EA310006220C31A01CFC
:1006C0001AF310EA607A01990A308872000AC87237
:1006D0000299039811F0CCFC07B0F0BDF3B5FF30E0
:1006E000401C0500006A81B0002803D009F37FFA9E
:1006F00000202862686A401C01D10120FEBD974F8E
:1007000000241FE097481AF3DEFF060002D0386885
:10071000002801D10020FEBD029800280ED13FF034
:10072000CAF8002802D005201CF058FB8C4B310081
:100730001E68002238680523B04702E030003BF015
:1007400091F8641C686AA042DCD800206862D4E793
:1007500084490020086048608860C86008612C39BE
:1007600048627047F8B504000E007F4D3BF03EF83C
:10077000070021002800FFF7B1FF7A4C0C3C012E46
:1007800006D1FF21213128001AF348EA0020A07287
:100790000020C043208138003BF02CF8FFF7D8FF41
:1007A000F8BD70482C38406A002801D0401C01D1A7
:1007B0000020704701207047F3B583B00021050089
:1007C000049EFF30B61D213000910191029049E056
:1007D0006A7801202C1D0021012A0FD0022A12D094
:1007E000032A13D13388614A93420FD1738893420D
:1007F0000CD1B388934209D1012107E03178C907B0
:10080000C917491C02E03178C907C90F002900D176
:100810000020002717E0608804996278E4BEB76E74
:1008200001000000F80700000004000009358D7F7A
:100830000818211D3AF00FFC01002078802803D110
:100840000120002907D005E0812803D1002901D02B
:10085000012000E0002008347F1C012804D1287802
:10086000B842E2DC0120009001982435401C019040
:100870000098002804D102980199807A8842B1DC5E
:100880000098D9E60800FF310022491C0A621100D5
:100890002EE770B501253CF09AF800280CD0364CB4
:1008A0002C3C606A401C07D034480121FFF720FF30
:1008B00005000020C0436062280070BD10B53CF008
:1008C00086F8002805D12C482C38416A491C00D1F3
:1008D000416210BDF8B505000C0000273AF090FF0A
:1008E0000090E168A06800232E005940584008435A
:1008F0004CD0A088A779234BC11940392A1A8C46BD
:100900000100D21840315B009A4205D99A1CA842D6
:1009100001D2AE1A00E0AE18664535DD8E4233DAFC
:10092000B0420FDD801B0604360CE168A06832007F
:1009300019F3ACEEE160B919A17101210843A5805A
:10094000A06029E0301A0204120C974200D2A27172
:100950000021012019F39AEEA268E36810431943BD
:10096000E160A06018E000003CC7000480190004AA
:10097000040000043403000410C60004E4C40004AE
:10098000FFFF0000FF07000011F0A5FC0020A5807C
:100990000121A071A160E06000983AF035FFF8BD38
:1009A000FFB59FB006000800376800211791219914
:1009B0007C69002910D060301E901AF3E0E922997A
:1009C00005004118C0782031400602D4B88823B011
:1009D000F0BD2888882801D80020F8E719AA1891C6
:1009E0000092219918981AAA17AB0DF3E3F8280082
:1009F0000DF307F9002853D0002104AAFF4801ABEA
:100A000007C318ABFE4A00921D7910AB1A7F38005D
:100A10002B001AA90CF321F905002DD1112040015A
:100A20002018C179090624D5002C0CD00D2189018C
:100A30006118896B002906D018AB1A7992006832C8
:100A40008B585B1C8B50C1794906490EC1711E98A9
:100A50001AF394E918AB1D7921992A01521B5218F7
:100A60000E320092010010AB1B7F2A002000FFF71E
:100A7000FEFD00203060AFE7356028891E994019DF
:100A80001AF38CE90088A88011204001201818ABC7
:100A90001B7901263200C1799A409143C1711DE052
:100AA00010AB197F009101952A8818991898843AFB
:100AB000091D1AAB10F357F806001CD0112018AB13
:100AC0001A79400120180123C17993409943C171DB
:100AD000288808382880B8880838B880002C08D0C2
:100AE0000D2080012018806B002802D0416E491C27
:100AF000416630006BE7002C14D00D2080012018D7
:100B0000816B00290ED018AB1A79920068328B588D
:100B10005B1C8B50816B0A69521C0A61806BC16837
:100B2000491CC1601E981AF32AE9010018AB187914
:100B3000219A03011B1A9A180E320092020010AB80
:100B40001B7F2000FFF793FDD3E700280CD00D2179
:100B500089014118886B002806D00269521C026185
:100B6000886BC16C491CC1647047F0B58446059D13
:100B700014682E68A64203D11F880888874203D9CB
:100B8000601C03D0A64201D20120F0BD60460028BF
:100B900003D018880880286810600020F0BDFFB5D9
:100BA00085B0002405001E000E9F21F04BF80028A0
:100BB00047D03000603004901AF3E0E88078403687
:100BC0000409307E46070698760F808B03900698BE
:100BD000006A029028003FF03DFD00282BD0687984
:100BE000022828D0082C26D3082E02D3012009B0D1
:100BF000F0BD30001BF3BCF9810002AA00921D2257
:100C0000491952018A1840003B2140190901411835
:100C1000079803ABFFF7A9FF040004981AF3AEE8A6
:100C2000784A0C3031001AF3CFFE77494DB60028D0
:100C300001000000F40B000000040000FD5AF8CB96
:100C40000968884207D20020DBE702AA00923A0036
:100C50002C32111DE6E72000D3E7F0B5012A069DEE
:100C6000059C13D0022A15D0042A2DD14A780E787B
:100C7000120292194E790F793602F619CF781204C2
:100C80003602120CF6198978360212E00A788E784C
:100C9000120202E04A780E7812029219CE798F7908
:100CA0003602F6194F79120436020979120CF61938
:100CB0003602711826688E4202D11F88974203D2ED
:100CC000771C03D08E4201D90120F0BD002801D04D
:100CD0001A8021602A80079801600020F0BDFFB5CE
:100CE00083B004001E000C9F0E9D3FF0BDFC002849
:100CF00020D0607902281DD0082E1BD3082F01D3E5
:100D00000120FDE438001BF33DF9030080001D25A0
:100D100000196D01119A109940196D4607C55800C8
:100D20003B210019090143180D9A05990498FFF712
:100D300094FFE5E40FA807C86C462B0007C4F3E74F
:100D4000F7B592B014000F00129800680D900020C3
:100D50000A900D9845690800603011901AF318E860
:100D6000060020300990280020F076FF21002C3169
:100D70001091091D403700280F9122D0109807AA22
:100D800008A903AB07C36B46E0790F9A0107387EC9
:100D9000090F4007400F07C30021B078099A0309E3
:100DA0002800FFF79CFF00280BD0002D08D00D2055
:100DB00080012818806B0028F8D0016D491C01655E
:100DC00093E030888828FBD922004C32883803040D
:100DD000111F081F0692021F0591049003920C39FF
:100DE00038381C3A029101900092387E1B0C47075C
:100DF0007F0F1A00099930003B000FF3D6FD070062
:100E000030000CF308FF002847D000200BAA07E0B1
:100E100060FA02C00CB701C09CCB000498F8000433
:100E20000AA9009101920A900D9B099A310038009D
:100E30000CF3D1FD002858D0614A0092614A624B00
:100E40000D9831001AF3ECFC002802D112990860C9
:100E50004BE012990600086001890818119919F3EE
:100E6000A8EF0E900A9800284AD00BAA0092099980
:100E70000E98230032000CF3DDFD070040D1002D59
:100E800008D00D2080012818806B002802D001684E
:100E9000491C01600E98807922E0002F28D0380785
:100EA000800F0FD0002D20D00D2080012918886BD5
:100EB00000281AD0C26C521CC264886B0169491C9C
:100EC000016112E0B80710D5002D08D00D20800177
:100ED0002818806B002802D00168491C0160B07995
:100EE000C107C90F280042F010E9002015B0F0BD7D
:100EF0003088143830800D980D9980881438888097
:100F0000079C6B461A8C10990F9823000CF3ADFDCB
:100F1000002F0AD1002D08D00D2080012818806BE9
:100F2000002802D0416E491C41660120DEE7F7B57A
:100F300082B014000025029807680398019760307A
:100F400019F326EF0600C0787F69400605D42037E4
:100F5000B87D400731D401252FE0002C01D10020BD
:100F600099E4A07AC00721D0E0790007000F01289A
:100F700005D10399220001A8FFF7E2FE05E00399DD
:100F80002200002301A8FFF715FD02990500019832
:100F90000860B079C00710D1002D0ED0A07980076D
:100FA0000BD5210038003BF050FD06E00D208001FC
:100FB0003818806B8168491C816028006BE4000050
:100FC00000B701C008B701C060FA02C070B50500E3
:100FD000008944193EF083FC00280AD0607B217B05
:100FE000000208430B2804D00A2802D005201BF079
:100FF00009FFFD4BFB481C68002229000068022302
:10100000A04770BDF948010008394860F84801213F
:101010004170002101707047F44900200839486090
:10102000F34948700870704710B5F14C607800289B
:1010300007D001202070A06D002802D0B0DE41133F
:1010400001000000F00F000000040000AE802BA79C
:101050000EF382F8606510BD70B53AF0E5FB05004F
:10106000E9481AF34EFB040028003AF0E1FB0225A0
:101070000DE020002573FFF7B3FF3AF0D5FB060023
:10108000E1481AF33EFB040030003AF0D1FB002C9B
:10109000EFD170BD70B53AF0C7FBDA4C050060784F
:1010A000002809D0D64904200856411C04D0811CD0
:1010B00002D0012107F38EFBD4480078012802D129
:1010C00014201BF08DFE0020207204200AF00AFC80
:1010D000CF48002200680C2108F395F9FFF7BCFF08
:1010E00028003AF0A5FB70BD10B5FFF7D3FFC54946
:1010F0000020087048704865C649086010BDC148A6
:10110000017A032901D0032101727047FF2800D022
:1011100008407047C04910B509683AF076E87D226A
:10112000D20019F316EF8905800A084301D041F077
:1011300032EF10BDF8B50024160005000F002200A4
:10114000002901D03889C2193BF04AFC002879D027
:10115000AC49087A032876D00228FCD0680726D547
:10116000002F24D0507B117B04020C430B2C08D0A1
:1011700010DC032C0BD0082C09D0092C07D00A2C2A
:1011800013D1A648A6490088097808430BD0FF254B
:10119000052615E0102CFAD0122CF8D04F2C04D1D3
:1011A000FF2507260CE004208543042608E0062ED0
:1011B00006D193480838406819F3F4EDC0056CD4A3
:1011C0008F480838406819F3EEED01002800FFF75A
:1011D0009DFF002861D08B484030818B002900D1D1
:1011E0008683904D002C1CD0288800280FD084497D
:1011F00004200856401C0AD108000838406840798D
:10120000FFF788FFFFF770FF002028805CE03AF0CE
:101210000BFB04007C4839001AF3CBFA20003AF0AB
:1012200007FB774F0426083F786886573BF0D8FBCA
:10123000002813D0734C606D00280FD0A06D0028DB
:101240000CD004E03AE02AE0774803F065FF0DF3A4
:1012500083FF616D401AA16D8842F5D36948022170
:101260000172701C05D0B01C03D00021300007F3C0
:10127000B1FA78684079FF2829D0FFF74BFF28881A
:10128000002824D03BF0ACFB002804D0FFF72CFF53
:10129000002028801BE0288819E00020F8BD68079E
:1012A00015D5002F13D03AF0BFFA04005648390084
:1012B0001AF37FFA20003AF0BBFA08E0680706D577
:1012C000002F04D0FFF7C8FE3800FFF789FE012089
:1012D000F8BD4C48602110B519F3BEEC10BDF8B54F
:1012E00000200C00474F1500B882B8651DE06078FB
:1012F000217800020843FF38163819D0A1280AD1F6
:101300002000062D07DB4179027908027D23104376
:10131000DB005843B865E178A27808021043291A27
:10132000091F0D042D14241D0419042DDFDCF8BD44
:10133000E178A27809021143CE082000F200914220
:10134000E9D1121D11040914A942E4DC0821082E78
:1013500000D23100CA00011D2A48143019F3E0EB15
:1013600006E0F000C019002114300A0006C0761C07
:10137000082EF6DBCFE7FFB58BB00A2000261D0054
:101380000A9605900B983700406907903FF060F887
:1013900006900B980B990089441820314118E07889
:1013A000C00701D1A01D01E020001230A2789446B0
:1013B0001207930F012B04D16046000908286CD056
:1013C0003AE0920F02D14026092034E00388174A00
:1013D000934209D14388934206D18388934203D133
:1013E00001263700300026E00078C00720D008260C
:1013F000032702201FE0000004000004340300045F
:10140000A0000004CC2C0004F83700046805000498
:101410000000000414070004C0B601C0543C0004DE
:101420008C0600049006000488130000FFFF0000F3
:101430000226370003202880A0780007800F0228AA
:1014400073D10D9A002010700B98891D858055BCB2
:1014500001000000EC1300000004000011450E1410
:101460000A9140690290002823D0614808900A98A8
:10147000022208A939F00DFE00281AD102983BF08B
:10148000EDFA002803D002988068400704D402983F
:1014900007F000F9002803D00D98012101708EE0BB
:1014A0005448406819F388ECC005F8D40620288019
:1014B00088E007984079022841D10C98002827D06D
:1014C0000C9840300500007D8006400F012809D9A6
:1014D000032805D80C98183019F36EEC000701D5D5
:1014E000012200E00022A17800200B079B0F022BB5
:1014F00003D10909090700D50120024308D0287E3D
:101500003D4A41072000490F0C301AF37BFA059041
:1015100004A903AA009101920698112149014018DB
:101520000378059A079821003AF031FB03980028C8
:1015300002D00D9901200870049800283FD02D4852
:10154000406819F33AEC304239D0A0780007800F98
:10155000022837D1294EB08A002833D0C120C000DC
:101560000025099026E0B84202D0254988421ED1C4
:10157000E08A2349884207D021000A9816310222C6
:1015800039F087FD002812D1A069401C1AD00A98B2
:10159000022209A939F07DFD002808D10A9821000E
:1015A0001A301831042239F074FD00280AD06D1C5D
:1015B000082D04DAE8008419A08A0028D3D100207D
:1015C0000FB0F0BD0120FBE70A480078C00700D04B
:1015D0000120704700B53BF018FA002805D0FFF74E
:1015E000F3FF002801D0012000BD002000BD000055
:1015F000888E0000980000049CCB0004CC2C0004D2
:10160000FFFF0000F3B591B00C001198002837D00F
:10161000207D0E2834D214264643BB4D4021A859C4
:10162000401CA85101A819F322EB200001A91DF0CC
:1016300005F9677D607E0090206801218068800048
:1016400000281FDB0098401C02062069120E0028AB
:1016500000D0002111981DF0A2FF206901A90028E7
:1016600024D10E2F05D21420784340194268521C11
:101670004260009800280BD170198168491C816074
:1016800013B0F0BD2069002800D000210022E1E75E
:1016900000200206120E142353438A5C5B199C68D7
:1016A000401CA2180E289A60F3D3E9E7E07D0028D9
:1016B00004D070190269521C026103E07019C268FB
:1016C000521CC26000200206120E142353438A5C8F
:1016D0005B199C68401CA2180E289A60F3D3CFE7D0
:1016E00010B5FF2419348849220019F38EEA864880
:1016F000210019F3BCEA10BD70B50D00002805D01B
:101700000D2189014018846B002C06D1002D03D0D7
:101710004C21280019F3D4EA70BD7C4AD1687C487A
:1017200043685918794B4160403B2162596B866888
:10173000711881606162196BC3685918C160A16238
:101740001168026951180161002DA163E4D0A06CF9
:10175000290019F342EB6069291D19F33EEB2900BA
:10176000A069083119F338EB2900E0690C3119F34D
:1017700034EB2900206A103119F32EEB2900606A3E
:10178000143119F32AEB2900A06A183119F324EB5C
:101790002900E06A1C3119F320EB2900206B20316D
:1017A00019F31AEB2900606B243119F316EB2900A9
:1017B000A06B283119F310EB2900E06B2C3119F3E1
:1017C0000CEB2900A06E343119F306EB2900E06E12
:1017D000383119F302EB2900206F3C3119F3FCEA90
:1017E0002900606F403119F3F8EA1DF000FC290070
:1017F000443119F3F2EA1DF0F7FB2900483119F3DF
:10180000ECEA70BDF0B400283BD00D2292018218A2
:10181000926B002A35D03E4C23685B1C23609B06EC
:101820002FD14C7ED36A1B19D3620B69002B23D1B5
:101830000D682B6FDE78F60707D09E783607B60F57
:10184000022E02D19E7CF60702D19B79DB0702D0E3
:10185000936C5B1C9364D36B5B1CD363D3B1C83AAA
:1018600001000000E817000000040000429FDD783E
:10187000AB689B000DD4002C0BD093695B1C012C32
:10188000936106D9D3695B1CD36102E053695B1C89
:101890005361F0BCC0E6F0BC7047002808D00D22B0
:1018A00092018018806B002802D0826951188161F2
:1018B0007047002810B51AD00D239B01C318986BF0
:1018C000002806D04469641C4461986BC36B5B1CA0
:1018D000C3630E290BD214204843104B1958491CDE
:1018E000002A195003D0C0180169491C016110BDBC
:1018F000002809D00D2189014018806B002803D0F1
:1019000080300188491C01807047FF21034819314C
:1019100010B519F3B6E9002010BD000024C600047C
:1019200040A80080A8000004C0207047010002A069
:1019300010B507F330FD10BD7364696F000000003F
:10194000F7B5150006000024002A1FD1002E14D080
:101950007079022811D002E0012004F063F8200021
:10196000641C022807D20022F848110019F374FE03
:101970000500F1D00AE0002D08D10022F448110042
:1019800003233EF07EF8050000D1FEBD6E61FFF737
:10199000CBFF0004000C28810827441912212000E5
:1019A0002F7319F398E9300023F0B9F9207314204C
:1019B0002071002060717079022803D1DF20A071AE
:1019C000002001E0380AA771E071B0792070F07949
:1019D00060700198143404602800FEBD10B5040046
:1019E0000321363019F376E920001C21393019F330
:1019F00072E92034A07E01210843A07610BD70B5A5
:101A00000400FFF7EBFF2000FF30FF220421993094
:101A100039F074EB2000FF2158304131050019F3F3
:101A200030E9FF34413401210020A161E0612075DB
:101A3000280016F3CDFD70BD0F21890170B5441843
:101A4000E168002926D10079002803D0032801D0BD
:101A500004281FD139F0FCFE0500BE480021FF22FA
:101A60009D324A438258002A0AD1FF239D335943AD
:101A700001220E1842503000FFF7C1FFE66002E07D
:101A8000491C0229EBDB280039F0E6FEE06800285B
:101A900000D1FEE770BD0F2189014018C1680029FF
:101AA00002D000220A60C260704710B5028912316C
:101AB00012189170090AD1700F213AF0BFFF10BDC2
:101AC0000A000F218901411810B5C9682A311DF09B
:101AD00081FF10BDF0B58FB00500149E159C170056
:101AE000092918D1382101A819F3CAE804206B4646
:101AF00098809948D88002A806223900801C19F3E2
:101B000024E804A832002100801C102304F07FF98F
:101B10006B46188105E023000022310001A816F36E
:101B200081F9280001A904F0F9FE0FB0F0BDFEB55F
:101B30000C3A0D0014060600240E1021102C00D8BB
:101B4000210030000A00FF30290019300831070059
:101B500018F3FAEFFF3601970094761C2B78706922
:101B6000AA1C0921FFF7B6FFFEBD70B50500487934
:101B70000B00C00620D5180060308178407809023B
:101B8000014318000922633016F33AFA040013D017
:101B9000607810220C38102800D80200280021009C
:101BA000FF300E31193039F07EFA002804D0627807
:101BB000A11D2800FFF7BBFF012070BD0F21890187
:101BC000401810B5C068583016F3A4FD10BD7CB5A0
:101BD0000C001500069900910F21079A8901401801
:101BE0000192C0682A003930210015F338FF7CBD0E
:101BF000FFB585B000220E001D0001894469081858
:101C00000390200004A9FFF79BFE070002D10120EA
:101C100009B0F0BD0F20800100962618F2680399E4
:101C20001300049830332A3216F3AEFA0498817CFC
:101C3000012910D0002200920192F26801001300E5
:101C400030332A3271312000FFF7C1FF049960312F
:101C5000C873000A0874079904982B00012216F330
:101C60007BF901003800FFF720FF0020C2DCFE7482
:101C700001000000E41B000000040000B6F0A8CC46
:101C8000D0E70F229201801810B5C068393016F3E2
:101C90004BF810BD30B504000D2080012018002A3B
:101CA0008FB009D0002C10D0806B00280DD0803070
:101CB000C5886D1CC58008E0002C06D0806B00280C
:101CC00003D0803045896D1C458101A816F3B4F816
:101CD000200001A904F02CFE0FB030BD70B5050046
:101CE0000F2080012C18E06828220100FF312D31DF
:101CF000DC3018F39EEF01212800FFF7C2FFE368F4
:101D00000100DC3301222800FFF7C4FF70BD70B56D
:101D100044692720400125186878002801D0002058
:101D200070BD2000FFF7DAFF0F2080012018C26885
:101D30000121C0325161C068C0308069002803D0E1
:101D4000827AFD231A4082726970E8E7F8B5446927
:101D50002720400127183878002809D00020F8BD36
:101D6000401A00046C190004144904000404000023
:101D700000212000FFF785FF0F2189016518EB681E
:101D80000100FF335B1D00222000FFF783FFE8689E
:101D90000126C030C660E868C0300169002904D15E
:101DA00006610121200020F0F8FA002120003E7099
:101DB00022F009FAD2E7F7B584B005000E004769B2
:101DC0000089002240190290380003A9FFF7C2FDE4
:101DD000040002D1012007B0F0BD0F2000228001D5
:101DE00038180092C26802991300039830332A32DF
:101DF00016F3D4F93100039801224031002316F381
:101E0000B5F80700706F00280BD0607B01210843F4
:101E100060730698002801D0FF4800E0FF48A061E9
:101E200009E00698002803D0280000F094FB02E0A7
:101E30002800FFF76CFF39002000FFF740FE00206C
:101E4000C9E7FEB500220E00018945690F18280078
:101E500001A9FFF77FFD040001D10120FEBD0F2085
:101E60000022800128180092C268019813003033C4
:101E70002A32390016F392F93100019801224031DB
:101E8000002316F373F8617B012211436173E44967
:101E9000A16101002000FFF712FE0020FEBDF7B592
:101EA0008AB005260A9847690F2080013D18EC6822
:101EB000002008900120583407900020069002E08E
:101EC000012003F0B9FD761E03D3E86840680128BD
:101ED000F6D10A98210016F3E7FA0028099019D0E4
:101EE000089800283FD1E8683E3015F379FD0028B6
:101EF00039D0E8683E3015F388FD0028E86804D042
:101F0000417A0A301DF096FD02E02A3015F31FFADF
:101F1000060002D100200DB0F0BDE8683E3016F397
:101F2000D9F902002100D4312000503002AB07C3A0
:101F30000D0022004032B439019200910B9A0C99A5
:101F40002300300016F348FA2000102229008430C4
:101F500039F0B3F8002804D027210020490179186E
:101F6000487001200690079800280CD0220021001C
:101F70000A98403220310023FFF744FE002802D0A7
:101F80000020069015E00698012812D1002F09D0F4
:101F90000D2080013818806B002803D06030418B01
:101FA000491C418309992000093115F318FF0020CD
:101FB000A0670698AFE7F8B5060045690F208001D5
:101FC0002818C76830005837390016F386FA04001D
:101FD00001D10020C3E620790122022800D000228E
:101FE00039003000FFF7E7FE002801D02000B6E6F8
:101FF000002D09D00D2080012818806B002803D007
:102000006030418B491C418321000931380015F3B0
:10201000E6FEDEE7F0B50E008DB0476916F344FA30
:10202000040046D032005032200001A916F339F8DE
:1020300001207067F01DF9300500806807F313FE7A
:102040000021A96031002079AC313500C03502286B
:102050000C9130D120006030817840780902014332
:102060002000633001AA15F3FCFF0C98102201A98F
:1020700039F023F8002805D1272001211657C8C3BD
:1020800001000000E01F000000040000E52A7BA022
:102090004001381801700FE00C98282201A918F3AC
:1020A000D2ED6B46188D28820020C0432721E860BE
:1020B00000204901791808705F4A21001268300039
:1020C0009047002829D100202FE720006030817838
:1020D00006000A0240782100024363310C980B91FC
:1020E00038F0F5FF002801D1012012E0B0787178B6
:1020F00002020A430B990C9818F33AEDA0796B464B
:102100008006800F6882188D28820020C043E86016
:1021100000202721490179180870200005E7F8B54B
:10212000070044690F2080012018C668380058361F
:102130003100FFF779FF050005D031003800FFF7C7
:102140008AFE002801D0002013E6002C09D00D20C3
:1021500080012018806B002803D06030418B491C1F
:10216000418329000931300015F343FE280000E6C1
:10217000F8B505000E000089170040198179002488
:10218000090716D54079C00709D02800FFF71DFFC1
:10219000EFE5642002F0E8FF641C2406240E3A00F8
:1021A00031002800FFF785FE0028F1D1072CF0D37D
:1021B000DFE52800FFF7B3FFDBE5FEB50C00060006
:1021C000086F1700401C06D1E06E401C03D12000B0
:1021D00016F312FAFEBD39F04FFB050002E00021B4
:1021E00039F038FB154819F3B4FA0028F7D1280064
:1021F00039F046FB0022300001A9FFF7B5FB0500CE
:10220000E8D00F20800136180094F268019813007E
:1022100030332A32390016F31DF8F0683E3016F3D9
:1022200063F80200F0682030417F09E0BB24000021
:10223000731C0000B11C0000B8FC000428D000048E
:10224000807E0907CB0F8006C10F019816F322F993
:10225000E06E401C0128E06602D1206F401C206720
:102260002100019801224031002315F389FE01006D
:102270002800FFF72EFCFEBDF3B581B006000F204D
:1022800080013518E8680400FF3059300700006805
:102290005834002820D0FC20005D00901DF064FD23
:1022A000029A21003000FFF788FF0098002814D020
:1022B000012811D1E868B14A2030017E0823491C69
:1022C00001760098210016F30BFAAD4AAD492000C3
:1022D00008237E6116F3F0F9FEBDA84A009821009C
:1022E000082316F3FDF9E8682030C17D491CC1754B
:1022F000FEBD70B50E0011000F2292018418E56832
:10230000FF22583515325051E0680622303018F35C
:1023100030ECE06806222A30310018F32AEC9A4AA1
:102320009A492800082316F3ABF970BDFFB581B0B8
:10233000050016000A9F3AF0AFFB00282CD02800B9
:10234000FFF750FC0F2080012C18E06802990A303A
:10235000320018F30EECE0683A0046720499280047
:10236000FFF7C7FFE16801204860E0682821DC3002
:1023700018F39AECE0682821FF30401D18F394EC24
:10238000E0682821FF30713018F38EEC27200021FF
:10239000400128180170417005B0F0BD0F2189017E
:1023A0004018C068FF304130C0690006000E704719
:1023B0000F218901401808B5C068408F009008BD02
:1023C000020010B53AF068FB00280BD00F20800106
:1023D0001018C16820314A7E520852004A76C068FF
:1023E000FFF710FB10BD0F2189014018C0680122C2
:1023F0002030417E114341767047F0B585B00E0024
:102400000B9915000A9F0C9A0400002902D10020A4
:1024100004A904900F2080012018019700930392D3
:102420000291C0682B000100FF3199313930320030
:1024300015F3E6F9B0E7F0B506000F208001341877
:10244000E0680F00417A15000A308FB01DF0FCFAE9
:10245000002810D001002B003A0001A815F322FC3F
:10246000300001A904F06EFA3000FFF7BBFBE06812
:102470000121C03001610FB0F0BD70B505000F2023
:1024800080012C18E0682030417EC9071886DF35AE
:1024900001000000DC23000000040000CDBBFE1D95
:1024A00012D0817EC9060FD5007F00220007C10F20
:1024B0002800FFF7CAFFE06801222030007F0007F4
:1024C000C10F2800FFF7C1FF70BD0FB50F218901B3
:1024D0004018C1686B46FF319A8881310A83C16810
:1024E0001A7AFF3181318A76C068197BFF308130DA
:1024F000C1760FBD30B50F24A4010019C468FF34A4
:102500008134257E0D70647E4C70C168FF3181314D
:10251000897E1170C068FF308130C07E187030BD78
:1025200030B50F24A4010019C4682034A57E0D70B5
:10253000E47E4C70C1682031097F1170C068203082
:10254000407F187030BD0F21890110B54418E06834
:1025500000280BD0FF304130006A002806D007F376
:1025600096FBE0680021FF304130016210BDEAE7D0
:102570000F2189014018C068FF307130704710B5D5
:102580000400FFF7D8FB2000FFF7F4FB002010BD8C
:1025900055853100409C000081853100809698006F
:1025A000A985310070B5002503891C186678436938
:1025B000002E17D0032E20D1002B09D00D24A4010A
:1025C0001C19A46B002C03D0803465886D1C6580B9
:1025D0005B79022B02D106F027F901E0FFF7D2FD6B
:1025E00001250AE05879032801D0012805D1207976
:1025F000012802D1080013F0BFFB280070BD10B500
:102600001DF04EFA002010BD10B502F0C2FF0028E8
:1026100005D0A748807DC00701D040F0B6ED10BDC1
:1026200010B5FFF7F1FF23F007FF40F0BCEC23F0FB
:1026300004FF10BD10B501F0A9FD002812D001F073
:10264000A4FD9C49012000058860401101F0FEFCBA
:1026500022F0B1FCFFF7D8FF40F0A4EC22F0C7FC59
:1026600001F092FD10BDFEB5002439F00FF906000F
:1026700000F096F990480168080602D5480600D592
:10268000012403F010FE050002D1012003F01FFE1B
:102690000120C007807802210840800717D4002C51
:1026A0001BD100228548009200680822012101AB5D
:1026B0003AF02DFA012200920022110010001300BE
:1026C0000DF05EFF012819D100F06AF905E07C48A1
:1026D0000068002812D1002C10D0002D0ED0754CAF
:1026E000A568E017E060E70C380001F0B8FCFFF7E0
:1026F000A1FF380001F0AAFCA56001E0FFF790FF00
:10270000300039F0C7F8FEBDADE710B539F0BEF8BE
:10271000040040F03EED22F03FFC200039F0BAF812
:1027200010BD70B5040039F0B1F8050062480168C9
:1027300021430160600601D4200618D5480616D54D
:10274000080612D501F09AFD5A48FF21491CC160C4
:1027500040685C49086861225205904308605A4904
:10276000486928229043486101E001F087FD280074
:1027700039F090F870BD10B50DF0ACFC002801D117
:10278000524810BD524810BD10B502F0B5FE514977
:102790004000085A504B4C495843096A0B071B0F1D
:1027A00018F30CEC080507060609090B0B06400890
:1027B00010BD800810BDC00810BD000910BD10B5C7
:1027C000FFF7E2FF4549884201D1454810BD454920
:1027D000884201D1444810BD444A4549904219D02D
:1027E000444A904201D1444810BD444A904202D12B
:1027F0004148D23810BD424A904201D1414810BDF3
:10280000414A904201D1414810BD414A904201D114
:10281000404810BD080010BD70B5040039F036F80E
:10282000050025480168A1430160600601D4200627
:102830001BD5480601D5080617D422480168612235
:1028400052051143016001684205114301601949B5
:10285000C00D886001F02AFD1B4841692822114300
:10286000416102F02FFF0CF043FD280039F012F80F
:1028700070BD114A010012680020914300D101206F
:102880007047C00005D50C4820304068002800D0B3
:10289000004770470300402010B5FFF76A6493F4C7
:1028A00001000000D8270000000400009E612D7187
:1028B000EAFF002804D0180302D5102000F036F8F3
:1028C00010BD0000A001008000300080C80000049E
:1028D000E0BD01C0CC06000400210080002800807B
:1028E0003F3D00007F841E0098360400A086010052
:1028F000001BB70054150000405DC600B013000077
:1029000000F82401540D000000366E01AA0A0000F0
:1029100080BA8C0100F04902AA0600000075190374
:10292000EB040000007C9200AA1A000010B52A49AE
:1029300004000020086029490860C020FFF776FFE6
:1029400001F0CDFCE00602D51DF09CFA10BD1DF093
:102950003AFA10BD0020E9E70221032010B51EF06D
:10296000B6FC00280FD1032108001EF0B0FC00289F
:1029700003D040F01CEC002805D1FDF76CFF0028C7
:1029800001D1012010BD002010BD10B501F0A0FC48
:1029900001280CD1FFF7E0FF002808D00DF00FFD53
:1029A0000F480088012802D001F0AAFC10BD01F0F8
:1029B0009EFC10BD084910B509680020002900D010
:1029C000402006490968002901D080210843FFF70B
:1029D000B2FEFFF7DAFF10BD6007000464070004D1
:1029E000DA070004052804D2664983001818085C39
:1029F0007047FF2070470A00032010B5FFF7F2FF71
:102A0000904201D1FFF7A6FF10BDFF280CD05D4A10
:102A100000218B005B18D35C834202D10806000EB4
:102A20007047491C0529F4D3FF207047FF280ED0BA
:102A3000544A00218B005B189B185B78834203D1BA
:102A400088004018105C7047491C0529F2D3FF200C
:102A50007047052805D24B49830018184018407864
:102A60007047FF207047FF280ED0464A00218B0098
:102A70005B18D35C834204D18800401880184078EA
:102A80007047491C0529F2D3FF207047FF280ED05C
:102A90003C4A00218B005B18D35C834204D1880040
:102AA0004018801880787047491C0529F2D3FF2010
:102AB0007047344A00218B005B18D35C834207D1F6
:102AC000880040188018C0784007C017401C704725
:102AD000491C0529EFD30020704710B50024FFF7EB
:102AE00094FFFF2806D02749830018184018007962
:102AF0008007C40F200010BD70B505000C00100049
:102B000001F096FB200001F0B4FA2800FFF78EFFD9
:102B1000022805D0032803D0042801D0052803D1BA
:102B2000200000F073F870BD2000FFF7B4FE70BD08
:102B300010B50400C00005D50122120311040C20B9
:102B4000FFF7DAFF200105D50122D20211040B2084
:102B5000FFF7D2FF600105D50122920211040A207D
:102B6000FFF7CAFF10BD0120C00310B501F060FBE4
:102B70000120C00701F07DFA0349086A80229043D2
:102B8000086210BDCC00000400280080F3B581B0BD
:102B90000F000198FFF739FF05000198FFF763FF69
:102BA00006000198FFF772FF0400032D07D1042EE1
:102BB00005D1102001F03CFBB00401F068FA002FB1
:102BC0001ED10198FFF775FF002819D0231F18F3B5
:102BD00000EA06171717170A04170198FFF77DFF79
:102BE00001000D200AE00198FFF777FF264AA900AF
:102BF00049198918C978CA080100100005F326FE92
:102C0000FF2201991000FFF7F6FEFEBD10B504008B
:102C1000C00203D501210220FFF7B8FFA00207D5AB
:102C200001210320FFF7B2FF01210420FFF7AEFFCF
:102C3000200203D501210520FFF7A8FF012000078E
:102C4000844205D04010844202D0401084421AD100
:102C5000FF208206A11808D0891804D0C20689185E
:102C600004D10C2002E00B2000E00A20FFF7DEFE7A
:102C7000022805D0032803D0042801D0052802D15A
:102C80000121FFF783FF10BDCC0000043EB5040016
:102C900002E0012002F07CFA03F046F90028F8D0A7
:102CA00002206B46187000205C70987020D1611F64
:102CB00001000000D42B0000000400006A0E58C57B
:102CC000D8700121684603F09EF93EBD01B5C948A0
:102CD000012240686946083003F06EF92020FFF7B2
:102CE000DFFF08BDC34808B50168012220316846EE
:102CF00003F062F96B46187808BD10B50400BD48B2
:102D000098B0016824220FA803F056F960070ED589
:102D100024220FA905A817F3B4EFB7491422684677
:102D200017F3AEEFB44810380FC808F04EF820077C
:102D300004D510AB9979587907F0CFFDE00609D595
:102D4000FFF7D0FF002805D0AC48406AC030C07FF4
:102D5000FFF7BCFFA848242210380FA917F390EF03
:102D600018B010BD10B54078FFF7C7FF03F0C0F9E9
:102D7000002010BD9F4800B5016889B02422684634
:102D800003F01AF96B4619780120002902D019794D
:102D9000002904D06B465978002900D1002009B0E1
:102DA00000BD944808B501680122491C684603F03B
:102DB00003F96B46187808BD8E4808B501680122F2
:102DC000C91C684603F0F8F86B46187808BD8948B6
:102DD00008B5016801220F31684603F0EDF86B4633
:102DE000187808BD834808B5016801221F3168467C
:102DF00003F0E2F86B46187808BD7E4808B5016814
:102E000001220B31684603F0D7F86B46187808BDED
:102E1000784808B5016801220C31684603F0CCF807
:102E20006B46187808BD1CB50122724C01A82168B8
:102E30000E3103F0C1F8216801221931684603F010
:102E4000BBF86B4619780020002903D01A798A4212
:102E500000D101201CBD674808B5016801220A3174
:102E6000684603F0A9F86B4619780120002900D0C4
:102E7000002008BD002008B500905E4801220168CE
:102E80006846083103F098F86B4619780120072945
:102E900000D3002008BD574808B5016801220D3154
:102EA000684603F089F86B46187808BD514808B5A4
:102EB000016801221831684603F07EF86B461878E5
:102EC00008BD4C4808B5016801221A31684603F074
:102ED00073F86B46187808BDF8B505000E00454C30
:102EE000012221686846891D03F066F86B46187850
:102EF000434B01225843286021686846C91D03F0EE
:102F00005BF86B4618783E4B58433060F8BD394843
:102F100008B5016804221031684603F04DF80098A6
:102F200008BD344808B5016804221431684603F02E
:102F300043F8009808BD2F4808B5016801221D31EB
:102F4000684603F039F86B46187808BD294808B57B
:102F5000016801221E31684603F02EF86B4618788E
:102F600008BD01B5234801224068694603F024F8F2
:102F700008BD012808B500D0002000901D4801229E
:102F800040686946093003F017F808BD01B51948D3
:102F9000012240686946401C03F00EF808BD01B5E7
:102FA0001448012240686946801C03F005F808BDFA
:102FB00001B51048042240686946001D02F0FCFF7C
:102FC0000220FFF76DFE08BD10B5040022F05EFE82
:102FD000002802D12000FFF7EBFF10BD054808B51F
:102FE000416801220831684602F0E6FF6B46187816
:102FF00008BD0000B83D04005C4C04003CC7000460
:10300000710200007CB504000D00160002203DF0A6
:10301000B5FA00280FD0FF21CB316B46198004216F
:1030200059801C715D7100219E71D9710823762130
:103030006A460FF03DF97CBD70B50025FFF771FFC2
:10304000012801D2012400E00024FFF760FF0128DD
:1030500001D2012000E00020002C0AD0002808D076
:10306000FFF7CBFE002804D1FFF7A6FE002800D111
:103070000125280070BDF94840687047603010B5E0
:1030800017F3D6EE80780107890F022908D10009CD
:10309000042805D00C2803D0F149086A401C0862B6
:1030A00010BDEF49886AC96A704710B507F096FDF0
:1030B000002809D038F0FEFBE84A117CA81FFA0C62
:1030C00001000000D02F00000004000039D48BA9BB
:1030D000002901D0491E117438F0FAFB10BDE448F4
:1030E00070B5683803F300FEE1483C3803F3FCFD9B
:1030F000DF481838007C062813D002203DF048FA3B
:1031000007E020001BF04CFCE279A17920001DF0C3
:10311000ACF90400F5D13DF03BFA002801D01BF0DA
:103120003FFC012002F017F800200CF0EDFCD24823
:10313000C168012292051143C160C1685200114368
:10314000C160CE4908690226B0430861C84C002519
:10315000A561CB482574606107F063FD6561667405
:1031600070BDF8B504000E000BF3B9FF00903006F7
:103170000D00000E0DF0F3FC616801278978002333
:103180000A07920FFF03022A0ED10E09042E0BD15B
:103190008602B748009AC038006A0021C0888018AB
:1031A0006941801B99410EE0012A11D109090E29BC
:1031B0000ED1009A80021E00101A2B00B341642227
:1031C0001900801871416161206160883843608016
:1031D000F8BDFEB50C00C969C90408D5210020312D
:1031E0004A7A097A55066D0E8E07B60F1BE000224B
:1031F000130069460CC11100E56A0BE0CB005B19B6
:103200001E685B6801931B031B0F9A18491C0E294B
:10321000009602D263789342F0D2009949044D0E91
:1032200000998E07B60F89068F0FE1690A04120C08
:1032300029000DF02DFC012E029003D10E352D0634
:103240002D0E0EE0022E0CD168060A23400F5843C3
:1032500029075F43090F4018390040181F30050641
:103260002D0E606801230288E0690104090C280022
:103270000BF31EFD029940188249096B08186087FC
:10328000FEBDF8B502203DF083F90500FF217E4820
:1032900000222D3118F31CFA06007ED00221C02036
:1032A000317334183081A078F322800880001040F8
:1032B00008300007000F4030A070E0784008400060
:1032C00008431040CF210840BF210840E070F120A2
:1032D0008000291806220D00A01D17F372EC2000B3
:1032E000062229000C3017F3D6EC20000622290014
:1032F000123017F366EC002020801C203518308136
:103300008421280017F3F8EC2F00162060372C6773
:103310007877574818380090007C00284AD05448E5
:103320007838C088A080FFF772FD002808D1FFF729
:103330004DFD002804D1A0887D2149014018A080BE
:103340004B4878388089A87002203DF021F97061DF
:103350004E480079800607D4A878002804D0A868D1
:10336000012189070843A860082015252D02387718
:10337000FFF72CFD0124002804D0012000F018FEE6
:103380003C484460290030000EF02AF80098007C88
:10339000002806D13949086900E011E002221043F3
:1033A0000861334801001C3184614868401C486052
:1033B0000120F8BD2E48C038016A0988A180C1E704
:1033C0002B491C318868401C88600020F8BD2949C1
:1033D00070B500248A69824221D1254D183D287C90
:1033E00006281CD00020886121488069002803D16C
:1033F000FFF747FF04000AE0254801694069814260
:1034000005D0244807220068012139F0AAFB287C56
:10341000002804D0002C03D12C2019F04DFD70BDE4
:103420000128FCD102202874FFF74AFD00281A4821
:1034300006D03C30040003F357FC00220C2105E0C9
:103440001030040003F350FC00220521200003F398
:10345000FDFB200003F3EAFB70BD10B5054CE169EC
:10346000814204D12F2019F027FD0020E06110BD1A
:10347000304D0400C03D040000900090C0A20080C8
:10348000FFFFFF7F40A60080B0190004ECE80004B5
:1034900000A000800C080004B84C0400F8B500241B
:1034A0000600F9480221846141740BF318FEF74DC0
:1034B000E962A862FFF78AFC6968084303D000202C
:1034C00000F076FD6C60002E04D0EF49380412083D
:1034D00001000000CC330000000400008611AE1A89
:1034E0001C310868401C0860EC4C183C207C022809
:1034F00008D1012001F039FEFFF7ECFC032600287B
:1035000001D02674F8BDE86906F3E9FBE34DE44B0E
:103510000822783D0092EA88E24800211C3302F03C
:10352000CDFC2674FFF79CFD002807D00BF3E1FDCE
:103530002A00383251631063E888A880D748683879
:1035400003F3DCFBF8BDD5491C314869401C4861D8
:103550000120ADE7D14910B51C314869401C4861D4
:10356000322019F0B3FC8CE7F8B5CC4C183C207C29
:1035700006282ED0C9488069002818D10BF3B9FD60
:1035800005000E002000210060382839C788808897
:103590000A6B4B6B0021801859410023C019594117
:1035A000401BB14100280DDD00F017FD0AE0BE48C8
:1035B00001694069814205D0BC48072200680121A9
:1035C00039F0D9FA207C002803D0032801D1052046
:1035D0002074F8BDF8B50BF38CFD07000C0038F033
:1035E0007DF9AE4DAE490090287C496A08432BD145
:1035F00028001838007C002600280AD0062808D0A9
:103600002800783831002A00403A536B8088126BCA
:103610000CE007F0A7FA002801D168690BE09F4A87
:10362000C03A106AD3698088926931008018594184
:10363000C01BA1416861002806DD0EF0B7F8002824
:1036400002D0287C401C2874009838F04BF9F8BD53
:10365000F8B50BF34EFD914A403A51631063904820
:10366000806906F33CFB8D4C0226183C207C25002B
:10367000603D00281FD0FFF7D4FB002819D0FFF7CA
:1036800079FC8B4F002801D0667407E0FFF767FCD8
:10369000002801D0032000E001206074EF80FFF7D4
:1036A00024FC7D21C90041437D200001081AA88027
:1036B00001E0002060747A4B08220092AA887D48BD
:1036C0000021183302F0FAFB01202074744C7A4F69
:1036D000E06801280DD138F001F90021E160796935
:1036E000302291437961754A516AB143516238F091
:1036F000F9F86A49A88848613869B0433861FFF72A
:1037000069FFF8BDF8B50BF3F4FC644A403A516325
:1037100010636348806906F3E2FA604C0026183CA7
:10372000207C2500603D002833D0FFF77AFB644FF2
:1037300000287DD0FFF71EFC00282BD002206074EB
:10374000FFF7BDFB002816D0FFF799FB002812D128
:10375000E8887D21090140180004000CB842E88087
:1037600001D9EF8004E07D21C901884200D2E980BF
:10377000E88854492DE0E8887D21C8380004000C11
:10378000C9018842E88000D2E980E9884D482DE0EF
:10379000A880C5E0FFF7E3FB002829D00320607470
:1037A000FFF78DFB002816D0FFF769FB002812D128
:1037B000E8887D21490140180004000CB842E880E7
:1037C00001D9EF8003E04049884200D2E980E888CF
:1037D0003E49081ADCE7E8883B49C8380004000C79
:1037E0008842E88000D2E980E9883848401ACFE76B
:1037F00001206074FFF763FB00281AD0FFF73FFB3E
:10380000002816D1E8883249FF30F5300004000C5A
:103810008842E88000D9E980A8887D21FF38F53802
:103820000004000C49018842A88079D2A98077E081
:1038300012E0E8887D2164380004000C49018842C8
:10384000E88000D2E980A888224964300004000C96
:103850008842A880EAD863E0FFF7C2FA002804D0C3
:103860001D486674E880AF805AE00D48016A00295F
:1038700001D0066205E01949002082008A58002A1A
:1038800001D0012703E0401C0828F6D33700FFF7DA
:10389000E7FB002F009023D00E4823E0304D0400BA
:1038A000C03D04005B33000000A000800C08000451
:1038B000FF7F0000CF320000C0A20080C0A80080BF
:1038C000204E000030750000E02E0000606D00000A
:1038D000D8590000504600004E7000004D38B2B478
:1038E00001000000C837000000040000D5CB7D7641
:1038F000F4FD02C07D204001A880FFF7EAFA00280D
:1039000003D0FFF7C6FA00280AD0FFF7D1FA002843
:1039100001D0002F04D00098002F03D0002803D13D
:10392000F94805E0002801D1F84801E07D20400178
:10393000E880667408220092AA88F548F54B0021B9
:1039400002F0C6FA01202074F24CF34F183CE068F4
:1039500001280DD137F0CCFFE66079693022914320
:103960007961EE4A516A02239943516237F0C4FFEC
:10397000EB49A88848613969022081433961FFF722
:1039800033FEF8BD10B5FFF7AFFA002802D0FFF7FD
:1039900069FE80E5012001F080FBE1491C3100282F
:1039A00005D0C868401CC860FFF7B6FE73E508691B
:1039B000401C0861DA480421183801746BE5FEB533
:1039C000050002203CF0F8FD0090D5484068002832
:1039D0004AD037F08DFFD24C0126183C0190207C54
:1039E000B602002D37D000283BD120006038006897
:1039F000002836D007F0C0F8002832D1FFF7D8F9F8
:103A0000002803D1FFF7F6F900282AD0FFF729FA9A
:103A1000002803D0FFF7EEF9002822D03FF0F2EBA8
:103A2000207C06280AD0BF480178002906D1012150
:103A3000502201700098130006F052F8FFF754FA74
:103A4000002805D0300000F02DFB300000F01DFBF9
:103A5000FFF798FF05E0002803D00025062804D1D1
:103A60002574019837F048FFFEBDAA4F183FF8694A
:103A700006F33FF9B86906F33CF9FFF744FB300061
:103A800000F010FB300000F008FB207C0628E7D097
:103A9000A44801780029E3D0282205700098290065
:103AA000130006F01DF8DBE71CB500200190009024
:103AB000694601A8FFF72EFA99480199C0380268B3
:103AC0008A4203D18288009B9A4226D00160009AE4
:103AD00082809349C3889C399A180A80019B9A1A5C
:103AE0004389D21A4A80C388D218643A8A80C2882D
:103AF0004389D21ACA800289009B0831D2180A80F1
:103B0000019B9A1A4389D21A4A800389D218643ACF
:103B10008A8002894089101AC8801CBD804870B50F
:103B2000406800282ED037F0E3FE040007F024F8A8
:103B3000002824D00020FFF742FF3FF064EBFFF79E
:103B4000B3FF7948C168012252051143C16073492E
:103B50008039886AFF229204104388624D0D280044
:103B600000F0A0FA280000F090FA6D481838007CA8
:103B7000062804D0082200210120FFF761FA200066
:103B800037F0BAFE70BD664870B5406800283AD07C
:103B900037F0AEFE5F4C0600183CA06906F3A9F8AA
:103BA0000025A561A06806F3A4F85B48A5604169FB
:103BB0003022914341615949486A02229043486248
:103BC00056488038816AFF22920491438162440DF5
:103BD000200000F067FA200000F05FFA5048C0387B
:103BE0004561FFF790FA4E481838007C062804D04B
:103BF000002211001000FFF723FA300037F07CFE9E
:103C00000120FFF7DCFE70BD424918398A68824204
:103C10000DD1002088600120C8603F4841693022F2
:103C2000114341613D49486A02221043486270478E
:103C3000F8B507003A484068002858D03848783826
:103C40000068002853D037F053FE354C0126183C4D
:103C50000090354D207C7605002F1CD0002808D11F
:103C600006202074FFF7BBF800283DD0FFF78BFF3C
:103C70003AE0062838D0274F183FF86906F339F89C
:103C8000B86906F336F806202074E868B043E860A7
:103C9000FFF739FA28E0062826D1FFF7A0F8002818
:103CA0000FD1FFF785F8002803D1FFF7A3F800280C
:103CB00007D0FFF7D6F800280FD0FFF79BF80028B1
:103CC0000BD1207C06280FD10020207406F054FF71
:103CD000002809D0FFF722FF06E0E8683043E860DB
:103CE0003FF090EAFFF74EFE009837F0950393E619
:103CF00001000000C43B00000004000021A408C231
:103D000005FEF8BD084910B518394A69824203D149
:103D10000020486100F06AF939E40000D859000039
:103D200010270000CF320000D83D0400C0A2008060
:103D3000C0A80080304D0400103E040000900090A8
:103D400038B5C94C2169814216D100202061C7488D
:103D5000007C032801D004280ED1012000F046F990
:103D6000606905F3D0FFC04B082200926288C0480A
:103D70000021143302F0B6F838BDF8B5BD48446BE5
:103D800000250BF3CAF9B84E00196941716330631D
:103D900006F0FCFE002811D0B448A838406900287D
:103DA0000CD0B06805F3AFFF08220092192233004F
:103DB000B14852010021083302F094F8AB48007C6E
:103DC000002825D0062823D0012822D10BF3A5F9FD
:103DD0000C00A64928390A6B4B6B2100821A9941C5
:103DE0000B00A249A54C603988882900801A9941A6
:103DF00000040014A0420BDAB06905F384FF9A4B6B
:103E0000082200929E4822000021183302F06AF82E
:103E1000F8BD306905F377FF082200923088924B95
:103E2000221A002197481033F0E7F8B5263801250B
:103E30008E4A8D4E117CAD020224030017F3FAE87E
:103E400014A30D0D390B0E7E1113361729300D0DED
:103E5000A8A8AAAAAA0DFFF76BFEF8BDFFF79DFE62
:103E6000F8BD012000E00020FFF7B3FDF8BD864853
:103E7000062904D0C168012252051143C160C168FE
:103E80002143C160280000F017F9280000F007F96D
:103E9000F8BD280000F010F9280000F008F9F8BD7E
:103EA0007248243802F33EFFFFF772FBFFF774FD00
:103EB000F8BD6E4FA83F388A002807D138002C3053
:103EC0003862F8893882FFF7F9FD04E067498439E0
:103ED000401E3962388201207861280000F0DFF846
:103EE0000BF31BF9F961B861B06905F30CFF082207
:103EF0000092386A5C4B428861480021183301F017
:103F0000F1FFF068614D01280DD137F0FBFC002175
:103F1000F16069693022914369615D4A516AA14348
:103F2000516237F0F3FC386A81885048183041619B
:103F30002869A0432861FFF761FBF8BD4B4B18339C
:103F4000587C002813D0401EFF24F53458745C615F
:103F5000FFF754FBB06905F3D6FE434B08220092ED
:103F6000474822000021183301F0BCFFF8BD0129A9
:103F7000FCD13E49147434318869401C88610120A9
:103F8000FFF7AAFAF8BD0429FCD1FFF7CFFBF8BD73
:103F9000012000E00020FFF755FEF8BD10B505F048
:103FA0004BFF324C1834A068002812D0E06800287B
:103FB0000FD006F041FE01280BD129F09AF8022813
:103FC00007D0012060602D2018F094FF2A2018F0FF
:103FD00091FFE8E42B2010B5FFF727FF2E20FFF715
:103FE00024FF2249002018314860DCE403222649DE
:103FF00012050028086901D0104300E090430861D1
:104000007047F8B502203CF0E1FA07000E216A463D
:1040100010F099F8050024D000981E4E046F00207F
:104020002071607120706070FF220621A01D37F0A2
:10403000C0E8F12080003918200006220C3016F369
:10404000DEED02203CF0C2FA686100980821603081
:104050000177310028000DF0E1F9002801D001209E
:10406000F8BD0020F8BD0000C03D0400184D04005C
:10407000C93B000000A60080E13A000034080000BF
:10408000CF320000053C000000900090C0A20080EC
:10409000C0A80080021100000948006A7047084962
:1040A0004A6902434A61CA690243CA617047044AC5
:1040B00051698143516170470149C04308627047AB
:1040C000802200804B490A6802430A608A680243E2
:1040D0008A600120704747490A6882430A608A68FB
:1040E00082438A6001207047424940310868086075
:1040F00070474049C043C860012070477A1FBA0A20
:1041000001000000C03F000000040000727EDBAE32
:104110003D4B80339969DA690901120909091201D5
:10412000002804D00520400701430A2003E00520B1
:104130000007014305200243D961DA617047334823
:10414000016B022291430163016B402291430163A1
:10415000016B04229143016370472C48016B0622D6
:1041600091430163016BC0221143016370472748EB
:10417000016B802291430163016B4622114301636D
:10418000016B3822914318221143016370471F4885
:10419000006B810701D500207047400601D5022041
:1041A00070470120704710B501F039FA002804D09B
:1041B0001749886901221043886110BD10B501F0CC
:1041C0002EFA002804D0124881694908490081610B
:1041D00010BD10B501F023FA002804D00C48806906
:1041E00001210904084010BD10B501F018FA00289B
:1041F00003D007488069C007C00F10BD0348C168DD
:10420000C2051143C16070478022008000210080F8
:10421000C02A008070477047FF484068816B090CD6
:1042200001D000207047816B090504D5816B09041A
:10423000090FFBD100E0806B01207047F649496807
:104240008A69120C120402438A617047F24840687E
:10425000816BC907FCD041680122D20391434160C0
:104260007047ED4949680A6B086348680122D20328
:10427000104348607047E8484068406A7047E64924
:10428000496880314A6A0001120F1207000902438F
:104290004A627047E0484068C06A7047DE49496832
:1042A000CA698243CA617047DB494968CA690243E7
:1042B000CA617047D84949680A6D02430A65704768
:1042C000D54949680A6A02430A627047D249496877
:1042D0000A6A82430A627047CF484068C03001686A
:1042E0004908490001607047CB48406880308188A8
:1042F0004908490081807047C748406880308188FC
:10430000012211438180704770B5C34D68688030C9
:1043100001680122114301600168C04C490205D5C2
:104320000168A14301600A203EF0ACEE686880306D
:1043300001682143016070BDB74840688030016862
:104340004908490001607047B34840688030006800
:10435000C007C00F7047B048406880300168AF4A5E
:10436000914301607047AC48406880300168012289
:104370001206114301607047A74840688030016809
:1043800001221206914301607047A34840688030C3
:10439000C068704770B5050016003EF04CEF9E4CAB
:1043A0006068010080300269056142694361826989
:1043B000F0228261C269C6618A68102002438A6065
:1043C0008A6820239A438A606068416B426B8A4204
:1043D000FCD0FFF7DAFF0028F6D160688168194346
:1043E00081604168012252031143416070BD8A48D7
:1043F00040688030006970478748406881682022A3
:10440000114381607047844840688168202291434D
:1044100081607047804949688031CA8801238340A0
:10442000C8881A43CA8070477B4840688168012267
:10443000D2041143816070477047774840688030EC
:104440000168FF22521C11430160704772484168A5
:10445000092080010818C169012292031143C1613A
:10446000C16952001143C161C16952001143C16168
:10447000704769484168092080010818C169012214
:1044800092031143C161C16952001143C161C16905
:1044900052009143C16170475F48406881681022B3
:1044A0001143816070475C48416809208001081809
:1044B000C169012252041143C161C169D200114393
:1044C000C1617047544905224968D2018918CA69F7
:1044D000382340079A43800E0243CA61C86901220B
:1044E0001043C86170474C4A0023D3561F21C0189F
:1044F0001F2800DA01000806000E70470D2804D8B6
:10450000454900228A56002A00DBECE73299AC7F4D
:1045100001000000BC43000000040000708703B8E5
:104520007047F0B593B0434C2068030960681B01E5
:104530000109A06809010209E068120100090001EF
:10454000C01C12902069491C050960692D010009F1
:104550000001401D1190A069921C00090001801DFE
:104560001090E0692D1D0609206A3601000900013E
:1045700008300F90606AF61D0009000109300E90A6
:10458000A06A000900010A300D90E06A00090001EC
:104590000B300C90206B000900010C300B90606B0D
:1045A0000709A06B3F01000900010D300A90E06B84
:1045B0000D37000900010D308646F020814310318F
:1045C00009911299854340350895119D8243854391
:1045D00050350795109D20328543503506950F9D27
:1045E00094468543503505950E9D0C9A854350356C
:1045F00004950D9D82438543503503950B9D5032A4
:104600008543503501950A9D029281438643874335
:10461000854372468243303150365037503583439C
:1046200050321F2000028343964605E0000100043B
:10463000000040002C2D0004009513252D025B196D
:104640002360099B814383435B1963606346834313
:104650005B194919A360E160089D0B21854349025C
:104660006A182261079D864385436A186261069D28
:10467000874385436918A1610321C9027218E26169
:10468000059D85436A182262049D85436A1862620B
:10469000039D85436A18A262029A82435218E2621D
:1046A000019D85436A1822637A186263009D8543E1
:1046B0006A18A26372468243511800250700E1631D
:1046C000AE00A059C004C00EFFF717FFA159C006E5
:1046D000C00CB9436D1C01432D062D0E102DA151A8
:1046E000EED313B0F0BDF0B588B0FF490A6A1206E8
:1046F000130F4A6A1206120F120113438A6A120636
:10470000120F12021343CA6A1206120F1203134346
:104710000A6B1206120F120413434A6B1206120F91
:10472000120513438A6BC96B1206120F0906120693
:10473000090F134309070B43EC494A68D11DFF31A8
:10474000FA310C690B610C6B0B630924A40112197B
:10475000D468D360E44BDC682406260F04969C687A
:1047600035012406240F03942C431D692D062E0FBA
:10477000350237032C43059700962600A6465C6950
:104780003E432406240F0194240426430694019CEE
:1047900027059C693E432406240F2506DC692E4329
:1047A0002406240F24072643029607965B68BC461E
:1047B0001B061F0F039B1E013B003343049E059FF6
:1047C00036023343009E3B4336041E4367463E4356
:1047D0002E432643072803D0062801D00A2809D1F2
:1047E000906802989060C8680798C860C86ACE62EE
:1047F00008B0F0BD0528FBD19068019E70463603D5
:104800003043069E30436646304328432043906041
:10481000CA68C860C86A06980343604603432B43CE
:104820002343CB62E4E7F0B5AF480168426809076B
:104830001207090F120E11438268036B1207120D43
:104840001143C2681207120C114302691207120BBE
:10485000114342691207120A1143826912071209B1
:104860001143C2699446120711439646026A14071F
:10487000426A240F1207120E1443826A1207120DA5
:104880001443C26A1207120C14431A07120F1504BC
:104890002C43456B26002D072D0A2E43856BC06BDC
:1048A0002D072D092E430007064390484568E81D53
:1048B000FF30FA30476841608768866016053443E8
:1048C000120614431A07144309229201AA18136806
:1048D00011605368546062461207120F13011343AC
:1048E00014022343140323431404234314052343D2
:1048F0001206134372461343426A4162816A83621D
:10490000F0BDF0B5784908684A69C004C50E48682A
:10491000D204C004C00E400105438868EECEB63212
:1049200001000000B847000000040000235DD0D45F
:10493000D20EC004C00E80020543C8685206C004EF
:10494000C00EC00305430869CB69C004C00E04054E
:10495000254315438A69DB04D204DB0ED20E5B01CA
:104960001A430B6AAC46DB04DB0E9B021A434B6A0C
:104970004D6BDB04DB0EDB031A438B6AED04DB04B7
:10498000DB0E1B051A43CB6AED0EDB04DB0E5B0668
:104990001A430B6B6D01DB04DB0E2B438D6BC96B74
:1049A000ED04ED0EAD022B43C904C90E470106000C
:1049B0003E4387023E43C7033E4326434006064329
:1049C00048010C000443880204434D48CD0340686D
:1049D0002B430100FF302C43FF30801C45696546A6
:1049E000456187698261C769C361436B3300466370
:1049F000866B8363C66BC363080009218901401875
:104A0000016905614169426181698461F0BD10B548
:104A10000400FFF712FF2000FFF76FFEFFF77BFF98
:104A200010BD37494968FF31FF31891C0A6800070A
:104A300012091201000F02430A60704730B50400EA
:104A40002F4D04280CD21120FFF76CFD6968092254
:104A500092018918C9698904C90E884200D20424C8
:104A60006868FF30FF30801C01680F2212029143FA
:104A70002207120D1143016030BD214A10B5536861
:104A80000522D2019A1813691F246406C006A343A5
:104A900080080343136110696311C9069843C9096B
:104AA0000843106110BD164A10B553680522D201A3
:104AB0009A1813691F24E403C006A343000B0343A1
:104AC000136110696311C9069843490C08431061CA
:104AD00010BD0B4A10B552680523DB01D2181369CB
:104AE0001F246401C006A343800D034313611069B2
:104AF000C90640094001C90E084303E02C2D0004FB
:104B000000010004106110BDF84A10B55268052379
:104B1000DB01D21853691F246401C006A343800D32
:104B2000034353615069C90640094001C90E084357
:104B3000506110BD0C2010B5FFF7E9FC04001120F6
:104B4000FFF7E5FC2100FFF7DFFF1220FFF7DFFC96
:104B500004001320FFF7DBFC2100FFF78EFF142079
:104B6000FFF7D5FC04001620FFF7D1FC2100FFF76A
:104B70009AFF1720FFF7CBFC04001920FFF7C7FCB2
:104B80002100FFF7A6FF10BDD84905224968D201D0
:104B900089180A699205D20E824206D30A69D206A2
:104BA000D20E824201D8082070470A691203D20E41
:104BB000824206D30A695204D20E824201D80420EE
:104BC00070470A699200D20E824206D30A69D20166
:104BD000D20E824201D8022070474A699205D20E55
:104BE000824206D34969C906C90E814201D8012013
:104BF000704700207047BD4949688031CA6AFF2369
:104C0000E13300079A43C00D0243CA627047B749B7
:104C100000B549688031CA6AC30652095201DB0EE9
:104C20001A43CA62FFF7B0FF0006000EFFF7E3FF6A
:104C300000BDAE494968C0314A69FF23E13300072E
:104C40009A43C00D02434A617047A84900B54968BC
:104C5000C0314A69C30652095201DB0E1A434A6148
:104C6000FFF792FF0006000EFFF7E3FF00BD9F492C
:104C70004968FF3141314A6BFF23E13300079A4312
:104C8000C00D02434A637047984900B54968FF3137
:104C900041314A6BC30652095201DB0E1A434A6383
:104CA000FFF772FF0006000EFFF7E1FF00BD8F491E
:104CB0004968FF31491C4A69FF23E13300079A43E1
:104CC000C00D02434A617047884900B54968FF3109
:104CD000491C4A69C30652095201DB0E1A434A6154
:104CE000FFF752FF0006000EFFF7E1FF00BD7F490E
:104CF0004968FF31FF31891C0A6A0F235B060007F0
:104D00009A43C00802430A627047784900B549686F
:104D1000FF31FF31891C0A6A1F231B059A43C30612
:104D2000DB091A430A62FFF72FFF000605D3773825
:104D300001000000B44B000000040000D732A56061
:104D4000000EFFF7DEFF00BD70B505000D20FFF778
:104D5000F3FB6B494E68092189017118CA699204F5
:104D6000D20E904201D2012200E0002264480024C9
:104D7000401C035DAB4204D0641C2406240E022CAC
:104D8000F7D3086A182555435D4A000C0004083221
:104D9000535B18430862486A000C0004AA18538841
:104DA00018434862886A9388000C0004184388629C
:104DB000C86AD388000C00041843C862086B1389C2
:104DC000000C000418430863486B5389000C00046E
:104DD00018434863886B9389000C00041843886368
:104DE000C86BD389000C00041843C8630520C001B8
:104DF00030180368168A1B0C1B0433430360436896
:104E0000568A1B0C1B04334343608368968A1B0C31
:104E10001B0433438360C368D28A1B0C1B041343F7
:104E2000C3603023364A634338329A18535B0C6AA6
:104E30001B042404240C23430B62521953884C6A2C
:104E40001B042404240C23434B6293888C6A1B04A8
:104E50002404240C23438B62D388CC6A1B042404CF
:104E6000240C2343CB6213890C6B1B042404240CF5
:104E700023430B6353894C6B1B042404240C2343EE
:104E80004B6393898C6B1B042404240C23438B6396
:104E9000D389CC6B1B042404240C2343CB63118AD9
:104EA000036809041B041B0C19430160518A436801
:104EB00009041B041B0C19434160918A836809048F
:104EC0001B041B0C19438160D18AC26809041204B7
:104ED000120C1143C16070BD09494A68092189015A
:104EE0005118CA691F235B02C0069A43800C024313
:104EF000CA61C869012292049043C86170470000EA
:104F0000000100044E494968C0314A690F239B03E0
:104F100000079A43800B02434A61EFE7484900B516
:104F20004968C0314A691F235B029A43C3069B0C40
:104F30001A434A61FFF732FE0006000EFFF7E2FF58
:104F400000BD3F494A68092189015118CA69FF23F8
:104F5000E13300079A43C00D0243CA61CEE73849E6
:104F600000B54A68092189015118CA69C306520966
:104F70005201DB0E1A43CA61FFF710FE0006000E55
:104F8000FFF7DFFF00BD10B504000D20FFF7D4FAD6
:104F9000FFF7A2FF1620FFF7C4FAFFF7C0FEE006F6
:104FA00014D50120C007C07CC1070FD00007400FF7
:104FB00002282AD0032809D11620FFF7BDFAFFF7EF
:104FC0008BFF1620FFF7ADFAFFF7A9FE1620FFF7BB
:104FD000A8FAFFF7C4FF1620FFF7A3FAFFF79EFF1A
:104FE0001820FFF79EFAFFF71CFE1620FFF799FA2C
:104FF000FFF735FE1620FFF794FAFFF74FFE162055
:10500000FFF78FFAFFF76AFE10BD1120FFF794FA41
:10501000FFF762FFDAE70B4880690007000F6DE7D2
:105020000848816801221207914381608168C205A6
:105030009143816081685210914381605EE7000076
:1050400000010004802A008070B504F0D5F8764D88
:105050000226002818D000F0E0F8002814D004F34D
:1050600099FA724C226A636A801A9941E162A062DD
:10507000E868B043E860A068002802D00020A06281
:10508000E06206F000F870BD05F039FD002803D19C
:1050900005F005FD0028F6D000F0BFF80028F2D09A
:1050A000E868B043E86070BD10B5604CA16981420A
:1050B0000ED1FFF7C9FF60694004400CFFF71FF8ED
:1050C00060694004400CFFF71FF80020A061606198
:1050D00010BD042010B5FFF712F80420FFF714F8F4
:1050E000524CA069002804D004F335FE0020A061D2
:1050F000606110BD4C48C06802210840704738B557
:10510000052840D2494D484C2969803400290BD0EC
:1051100004F340FA6962286202E0052000F092F888
:10512000E06A4000F9D530E001218140E8680143A0
:10513000E960FFF7DFFF002801D10120CD1B6FF2EE
:1051400001000000B04F00000004000084E8760C6D
:1051500038BDE06A400022D400F069F800281CD174
:105160000420FEF7DBFF0420FEF7CBFF2C68FDF7E1
:10517000DCFF002800D06C6868690421084368617E
:105180002F4B082200922F4822000021183300F0F4
:10519000DBFE04F309FA69622862002038BD274863
:1051A000C16802229143C160D1E7052810B501D33F
:1051B000002010BD012181402148C2681143C16017
:1051C000FFF7A2FF002814D000F031F800280BD020
:1051D000FFF789FFFDF7A9FF002805D01A48007CDA
:1051E000042801D105F059FF1449C86802229043F0
:1051F000C860012010BD052810B516D2104C01233F
:10520000E16883400A009943E1600ED1002A0CD086
:1052100000F00DF8002801D0FFF765FF0749C868C6
:1052200002221043C860012010BD002010BD0448B8
:105230008069002800D00120704700000090009095
:10524000C80100041D4F0000184D0400F849086B08
:105250008022904308637047F64910B5096836F01C
:1052600074E88905800A084301D03DF034EF10BD91
:10527000F148016A0F22114301620220ECE7EE4877
:10528000016A0909090101620120E5E7EB4970B5EE
:105290000868082290430860E94A506840084000C6
:1052A000506010690B2108431061E64908009369BA
:1052B000DB0601D4401EFAD29069800601D4491E53
:1052C000FAD236F051FBE0490A680124A406A24351
:1052D0000A60DD4A80321368DC4D2B40136013688E
:1052E000ED432B4313600A6822430A6036F040FB0B
:1052F0000120FFF7B1FFFFF7BBFF20F033FD70BDCA
:10530000D349FF22C432888B1042FCD17047F8B5D4
:10531000D04C6069002806D036F026FBCE48FAF75C
:10532000A1FF00F0AFFC36F01FFB606100210120FF
:1053300020F07EFC002810D0C54EB48801208002E9
:105340000440B088C24D3527A0433F012035B84204
:1053500004D1287D012108432875F8BD022000F002
:1053600042FB0028F9D03C43B480297D0120014351
:105370002975F8BDB74810B5446900214161FF2186
:105380000170B3482030017D4908490001750120B2
:1053900020F070FC200036F0EBFA10BD70B5FEF284
:1053A000C6E9AC4D04002878022813D1A869401C36
:1053B000A861200605D4A8482030FAF753FF00F072
:1053C00061FC802C02D1FEF2B2E970BD2000FEF239
:1053D000B8E970BD6869002805D09F481630FAF713
:1053E00041FF00F04FFC0021012020F021FC0028AB
:1053F000EFD002206C6128700120A86197480068F6
:105400000028E6D1924DAC88012080020440A88893
:105410006B26A043F600B042DBD0022000F0E3FA96
:105420000028D6D03443AC8070BD8A4910B5886955
:10543000401E88610FD14C694861FF20087001202F
:1054400020F018FC802C02D1FEF270E910BD200083
:10545000FEF276E910BD0028FCDAFEF268E97E482B
:105460001730FAF7FFFE00F00DFC10BD70B5794E55
:105470007069002807D036F077FA7748001FFAF7EE
:10548000F1FE00F0FFFB36F06FFA706100210120A1
:1054900020F0CEFB002814D06D4DAC880120800296
:1054A0000440A888A04382280BD02888F0800020E0
:1054B00000F099FA002804D0A888308182200443A3
:1054C000AC8070BD634810B56149028944698A8027
:1054D000C2880A8000214161FF210170012020F073
:1054E000C9FB200036F044FA10BD70B5594D68690B
:1054F000002807D036F038FA5748C01EFAF7B2FE37
:1055000000F0C0FB36F030FA68610021012020F085
:105510008FFB00281BD04E4EB4880120800204402F
:10552000B088A043022812D0FEF759FE002803D00D
:10553000012803D13F2002E01A2000E07F203188BB
:10554000E9803080B088288102200443652DE8E49A
:1055500001000000AC530000000400003B2D53BFCD
:10556000B48070BD404810B53E49028944698A80C4
:10557000C2880A8000214161FF210170012020F0D2
:1055800083FB200036F0FEF910BD30B505000C009D
:10559000FFF7C0FE334B20331D81FFF7BBFE9C801D
:1055A000FFF7B8FE30BD10B50400FFF7B3FE2D4B7A
:1055B00020331C81FFF7AEFE187910BD30B5040012
:1055C0000D00FFF7F0FF284301002000FFF7DDFF8B
:1055D00030BD30B504000D00FFF7E5FFA843010022
:1055E0002000FFF7D2FF30BD1F484178002909D1C4
:1055F00020490968012209024270090F0200243281
:10560000515C817080787047174910B5C8780028C0
:1056100015D10861174840680A008007800F1032D2
:1056200010230124002807D0012803D0022803D02A
:10563000032803D1136001E030201060CC700869AA
:1056400010BD0000400C0090C0B601C080A10080D9
:1056500000A3008040A60080881300000021008085
:10566000FF7FFFEF00080090F80100043700010001
:10567000E407000400200080E54800880006000ED2
:10568000704700B5FFF7F8FF022806D1E0488038E0
:1056900040688007800F012800D0002000BDDD4B4E
:1056A0005968382291431040084358607047D94BDD
:1056B00059680F2292019143104008435860704787
:1056C00010B50C00FFF7F3FF2000FFF7E8FFB7E786
:1056D000D14810B5446900214161FF2101700120CA
:1056E00020F0D2FA200036F04DF9A9E770B5CA4C87
:1056F0006069002806D036F041F9C848FAF7BCFDC9
:1057000000F0CAFA36F03AF960610021012020F079
:1057100099FA002811D0C24DAC88012080020440C3
:10572000A888B526A0433601B04206D0022000F07A
:1057300064F9002801D03443AC8070BDB4480068DF
:10574000B8498874010CB74820380186B6494969C0
:105750008163704710B504000BF09AF9002802D15C
:10576000200020F07DFE6BE770B50500AD480C0011
:1057700020384169A14212D044610021200020F06C
:10578000BDFA0021200020F0C5FA002D07D100212C
:10579000200020F0B9FA0021200020F0C1FA70BDED
:1057A000A0482038016A0020DEE79E482038C16901
:1057B0000020D9E79B48203881690020D4E7994828
:1057C0002038416881610020CEE796482038816802
:1057D00081610020C8E793482038C16881610020BA
:1057E000C2E790482038016981610020BCE7884801
:1057F0008E4A8030016811430160704784498B4AAA
:10580000803108689043086070478948C168890002
:105810008908C160C168032292071143C160810CED
:105820007C488030416183490161834941610521A0
:1058300001617047814800B50068002801D0FFF77A
:10584000E4FF7F480D21C1632D21416300BD7149F3
:1058500080398868CA0C9043886047E76D48803873
:105860008168C20C1143816032E769488038006862
:10587000000701D501207047002070476648C068C6
:10588000704700207047F7B586B004000D0036F071
:1058900075F800900021012020F0D4F900286FD085
:1058A000032160000A008240059020000838400073
:1058B0000E0086400390200010380492020047003A
:1058C0000800B840029020001838430008009840B3
:1058D000012186460800A0409C460B0001905948D3
:1058E0009340584A4030002D37D0082C04D2156818
:1058F000049EB543156012E0102C03D25568B543E1
:1059000055600CE0182C04D2C569029EB543C561F0
:1059100005E0202C03D2056A7646B5430562089D52
:10592000002D14D0102C04D29368019C2343936063
:1059300002E0426A1A43426282680A438260404B34
:10594000C0335868012212061043586044E03C48B6
:10595000C03001680422914346E0082CE0924FC613
:1059600001000000A85700000004000068F780D381
:1059700007D21568059E049FB140BD430D431560D5
:105980001BE0102C07D25568039FB543B9400D4367
:10599000556012E033E0182C06D2C569029EB9406A
:1059A000B5430D43C56108E0202C06D2056A664662
:1059B000B1407746BD430D4305620899002918D0D0
:1059C000102C04D29168019B9943916002E0416AD6
:1059D0009943416281684908490081601D48C0308F
:1059E0004168012212069143416000211B48416039
:1059F00005E01848C030016804221143016001200D
:105A000020F04CF9009835F0C7FF09B0F0BD102127
:105A10000A2803D2054940003431095A054801805B
:105A2000012070478020008000290080F8010004D8
:105A300037000100000800905CC7000400A8008047
:105A400000044010002A0080170000FF1020000012
:105A5000F09001C08022008000020090C0B601C01A
:105A600070B50024FFF717FE002808D0FEF7F8FBFA
:105A7000002803D1FEF7E9FB002800D0012435F00F
:105A800087FF0500002C07D102203DF00BFE002807
:105A900002D01B49012008600021012020F0DCF821
:105AA000280035F079FF002070BDF8B500201549B9
:105AB0001FF058FB124E0024361D0F273F0308E04D
:105AC0002104090C394300201FF04CFB705980471A
:105AD000641CA50070590028F2D10B480C490268DB
:105AE00000920A4A0B480C4B02F3EEF91AF078F8D0
:105AF0000A480168002901D000208847F8BD00004D
:105B0000F09001C05F5F00006807000488DA0004BD
:105B1000781900046C190004803C04C038020004A9
:105B2000FEB50D001600089F0A9A0999002800D1B9
:105B3000FEE70468002C00D1FEE7029201913200DA
:105B400029002000009720F011FDFEBD10B500F3E4
:105B5000AFFF0006000E10BD10B500F33BFF0006BE
:105B6000000E10BD002810B501D000F36FFF10BD6E
:105B700038B514006A4600F3C9FE00982070002072
:105B800038BD10B5040000F31BFE2060002010BDDE
:105B900010B500F3EBFE10BD7CB50D001600079AA2
:105BA0000699002800D1FEE70468002C00D1FEE72A
:105BB0000192009132002900200020F0D0FD002841
:105BC00000D165637CBD10B5416B20F0DFFD10BDD9
:105BD0007CB50C001500069A002800D1FEE700688D
:105BE000002800D1FEE70021019200912A00210047
:105BF00020F0EAFC7CBD10B520F006FD10BD0028A9
:105C000010B500D1FEE70068002800D1FEE720F0C3
:105C100072FD10BD002810B500D1FEE70068002815
:105C200000D1FEE720F081FD10BD10B520F087FD0A
:105C300010BD10B520F08BFD10BD10B504003DF077
:105C400084EA002801D0002010BDFDF284ED6060E0
:105C500000F3B6FD2200002100F314FE0028F3D06B
:105C60006068802802D1FDF276ED01E0FDF27CED66
:105C7000012010BD38B504003DF066EA002801D0CF
:105C8000002038BD00F39CFD21686A4600F3FAFD50
:105C9000002808D16068802802D1FDF25CEDEFE7B2
:105CA000FDF262EDECE7012038BD0000F8B5974940
:105CB000486B0222904348639548017801297ED0C1
:105CC0000121017035F064FE00909248422115F3E5
:105CD00078E801218F4AC90700200B781354491C2A
:105CE000401C0A28F9DB8C4900200B781418491C49
:105CF000401C0B28A372F8DB874890380178517557
:105D0000017991754179D175017A1176417A51768F
:105D1000017B9176407B8049D076803900200B78DA
:105D20001418491C401C0A282377F8DB7A4950399B
:105D30000A7E7848203082710A7FC271497F0172E1
:105D4000754930390A7842724A7882728A78C2720A
:105D50000A7902734A7942738A7982730A7AC27322
:105D60004A7A02748A7A42740A7B8274A03DEBF507
:105D700001000000A45B0000000400009C98F5678F
:105D80004A7BC2748A7B0275CA7B42750A7C827523
:105D90004A7CC2758A7C0276C97C4176634930317F
:105DA0000A7882764A78C2760A7902774A79427707
:105DB0005F4A137C8377927CC2770A7F203002701F
:105DC000497F4170594E082010368446B078EE283D
:105DD00000E041E0FAD16046F070FF20B070002290
:105DE0002FE0B078EE28FCD10C245443514B1959C4
:105DF000F170080A3071080C7071080EB071FF2044
:105E0000B070002903D1B078FE28FCD11BE0474FC9
:105E1000E51869681A37B078EE28FCD1434813308A
:105E20000B780370491C401CB842F9D9414B686893
:105E30001B59C018884210D8287AB070521C12061C
:105E4000120E6245CDD3009835F0B0FD34483A4982
:105E50004163344800210170F8BDFF20B070DAE7DB
:105E6000324810B510308078EE2804D13348FAF764
:105E700017FAFFF725FF10BDF8B5FCF7D2FC304D3F
:105E8000284E274F2C6804E06068002800D0804727
:105E90002468002CF8D1FFF7E3FF7078401C00065F
:105EA000000E7070FAF7FCF9786BFF21491C08436B
:105EB0007863FCF7B5FCE5E7224810B500F394FDE4
:105EC00010BD10B5184C203C6360E260A1602060FA
:105ED0003DF0A2E920613DF0B0E960613DF0BCE930
:105EE000A0613DF0CAE9E0610D48416B0222914397
:105EF0004163FFF7E5FE10BD10B5040035F052FD1B
:105F00000F4B19680A0000E00968002902D0A1427D
:105F1000FAD101E022601C6035F048FD10BD0000A0
:105F20000034008044020004642F000490010080CB
:105F300080000080E8360400F201010070000100DA
:105F4000F4170004A0B9000407E003788B4207D0DF
:105F50004378801CD21A921E1818022AF5DA002003
:105F6000704710B51C009A4200D81400220014F3A8
:105F700096EE200010BD00002A48816A04221143D9
:105F800081627047FFB581B000241D00FDF2ECEB8B
:105F9000009003F301FE244E0027B06800281DD0B6
:105FA00004004069B0603068401C306001D10120BD
:105FB000306001982060029860603068206103982A
:105FC0006761A0600A98207303F3D2FD0100706836
:105FD00003F318FE2100301D03F338FE706800281B
:105FE00006D03169002903D1806803F3E1FDF06038
:105FF000002C07D02069002804D0002D00D0286094
:10600000012403E0002D00D02F6000240098802898
:1060100002D1FDF2AAEB02E00098FDF2B0EB200005
:1060200005B0F0BD00340080707D0400FF48416879
:106030000068814201D10120704700207047FB4871
:1060400010B541680068012292070B0004009343D9
:106050009443A34205D111401040814201D0012058
:1060600010BD002010BDF24900204861F14A506087
:10607000EE4A1060C8607047EC48416801600168F2
:10608000EB4841610021C16070470021032010B539
:106090001FF0ECFDE6480178002901D1806801601D
:1060A00003201FF005FE10BDF8B504000D0016001A
:1060B00035F078FC0700002103201FF0D7FD002CED
:1060C0000ED0002D0CD032002900200014F3E6ED94
:1060D00003201FF0EDFD380035F068FC0020F8BD0E
:1060E000380035F063FCFEE7D14810B580683421F4
:1060F00014F370EE10BDF8B50C0007000026002860
:106100001CD0CB4D2878012818D1012C02D135F0B4
:1061100049FC0600002103201FF0A8FDFEF79FF8B0
:1061200000280DD0FFF79FFF0020287003201FF0EC
:10613000BFFD012C02D1300035F038FC0120F8BD44
:1061400035F030FC8446FFF77AFF002804D0604623
:1061500035F02CFC002013E0E868401CE860B348F0
:1061600000680C210004000C4143B34808180021CA
:1061700005000A000B000EC0604635F0E1C6162788
:1061800001000000A05F000000040000CF42260BC9
:1061900017FC2800002800D1FEE7FA78082A01D869
:1061A000121D00E00C22390014F382EDA44800F027
:1061B00071F9A749C86B01221043C86303201FF07F
:1061C00081FD012C02D1300035F0FAFB0020F8BD32
:1061D0001CB50024E4439F480122032101AB009435
:1061E000FFF248F801980028F5D00128F3D100F01B
:1061F00061F9F0E710B535F0DFFB04000021032062
:106200001FF03EFD9048001D00F044F99049886B56
:10621000CA0D1043886303201FF054FD200035F0A1
:10622000CFFB10BD002810B50AD00078012807D197
:10623000FFF72CFFFFF7DEFF17F0DDFC002010BD9D
:10624000012010BD10B50178042901D0012010BD36
:106250007C494A68521C4A600969002901D0884774
:1062600001E0FFF7C7FF002010BD0EB504216B460B
:106270001970012159700221D97001781971407883
:10628000587170484168491C4160FFF7B3FF012114
:106290006846FFF73AFF00200EBDF0B587B035F035
:1062A0008BFB070081200003FDF766FF6A49012090
:1062B000000588600820FEF741F80820FEF74AF83C
:1062C000644866492830016065490161654941605B
:1062D0005C4C0026266101220A20059202000390F0
:1062E0006148012189026B46049607C3002359487F
:1062F0005E4AA8385EA100F3B9F9002802D0012057
:1063000007B0F0BD53485CA1FEF242FF002103201C
:1063100026701FF0B5FCA0685A4D0068A84207D14E
:10632000FDF7A7FF00280AD0FDF7AEFF002806D032
:10633000FFF7E4FEA0680560FFF79FFE0DE0FFF7A2
:10634000A5FE4148466001206B461874DE7420703B
:10635000002104A8FFF7D9FE267003201FF0B2FC2D
:10636000380035F02DFB0020CAE700290CD00528A5
:106370000AD2042802D13348016103E0354A800083
:1063800028321150002070470120704770B5FDF78A
:1063900070FF2C4C002802D00020207014E035F053
:1063A0000BFB274D060008E0E168002910D02548C6
:1063B000491E1430E16000F06DF860696968884238
:1063C000F2D1300035F0FCFA30492F48C86070BD7A
:1063D000FEE71B4801684068814201D0012000E0CF
:1063E000002019494A6809688A4201D0012100E069
:1063F0000021084301214840704701001548002250
:1064000010B5FEF2C7FF10BD10B504000D480178AD
:10641000012901D00121017020030BD51B491C4823
:10642000C8600820FDF790FF0820FDF787FF0120D6
:10643000FFF7E3FFE00401D5FFF7A8FF10BD000060
:10644000801300C0E8B601C0001300C0881300C06C
:10645000802A008024FA02C0003000807B600000A7
:1064600055600000356000007CF502C0E15F00006F
:106470004963635461736B0049636351466C6167A0
:1064800073000000CDAB0000FFEFFFFF8022008013
:10649000FFFFF7FF026801231104090C9B07491C49
:1064A0001A4011430A009A43082A01D3594019405F
:1064B00001607047F8B535F07FFA144C144E154D55
:1064C00007001BE0FDF7D5FE002803D0124900208D
:1064D000087017E070680C230004000C5843401942
:1064E0000CD00178052905D28A00A258002A01D0D3
:1064F000002902D12168884700E090477068316820
:106500008842DFD1380035F05BFAF8BD4CFA02C0A2
:10651000001300C0081300C0E8B601C070B535F024
:106520004BFA0500FF4803F33BFA040009D02000B2
:106530005421083014F358ECFA4821000C3003F3CE
:1065400059FA280035F03CFA200070BD70B50400FF
:1065500035F032FA0500002C0DD02000542108300F
:1065600014F342ECEF4821000C3003F381FA0100F0
:10657000EC4803F33FFA280035F022FA70BD10B55D
:1065800001F082FB002010BD70477047630521FFBA
:10659000010000009C63000000040000E7D3A3B6E4
:1065A000002803D02030407D0007C00F704700282E
:1065B00007D02030427DF723C9071A40090F0A434C
:1065C00042757047002807D02030827DFB23C90721
:1065D0001A40490F0A4382757047002806D0826826
:1065E000C90752085200C90F0A4382607047002849
:1065F00006D082680223C9079A43890F0A43826042
:106600007047002806D082681023C9079A43C90E34
:106610000A4382607047F8B500250E0017002C0071
:10662000002824D00D2189014218516A002901D087
:106630000D000835D169002901D00C000834330061
:1066400022002900009704F3E9FD002E06D0002D5A
:1066500004D0280048210C3014F3D0EB002F06D0D2
:10666000002C04D0200048210C3014F3C8EBF8BDF6
:1066700070B50400006800280BD0806D002500284C
:1066800003D0FFF76DFF206885652068FFF768FF7E
:10669000256070BDFFB589B01C00A8A605A88ECEE8
:1066A000139D8EC000210A000B000E0001A84EC0F1
:1066B0000F001298204302D101200DB0F0BDE87800
:1066C000A9780002AE1D0843C00700D0129C002C20
:1066D00010D0A07AC0070DD0206D002804D1FFF79C
:1066E00027FF0028206505D0206D542208302100A6
:1066F00014F352EBE878A9780002084380071ED50E
:106700000A98002808D0914A0998126801219047F8
:106710006B46187D401C18750B9905270622200032
:1067200014F3D0EA8A4A0998126801219047894AED
:10673000099812680121904702212D200155E8781F
:10674000A97800020843C00707D0122706212000BD
:1067500014F354EB01212D20015569782A780902A0
:10676000E0791143000909070001090F0843E071AE
:106770000320A07168792979000208433100208143
:10678000223110220D0001A8E77234F04AFD0028E2
:106790000CD1200010222E3005A914F394EA200019
:1067A00010223E3005A914F38EEA0BE020001022DF
:1067B00029002E3006F338FD2000102229003E303B
:1067C00006F332FD3078207320001022B11C1D30FA
:1067D00014F378EA31002000102212310D3014F346
:1067E00072EAA07A01210843A072002065E770B523
:1067F0001B210022490141188A820D21531E890163
:1068000041181D240B63110064010725ED014E00A2
:106810003618361932828E0036187619491C04292A
:106820003362F4DB70BDFFB587B000200C001500AB
:10683000109E1F00002E039067D070783178000200
:106840000843032841D1079801960095407901211A
:10685000022800D00021404A079823008218FFF741
:1068600019FF002C039007D0E07901210007000FE9
:10687000E071E07A0843E072002D07D0E879022148
:106880000007000FE871E87A0843E872002F07D08C
:10689000F87940210007000FF871F87A0843F87280
:1068A0007078317803020B4307990F208001081894
:1068B000069020004030059028004030049014F3EA
:1068C0001EEC050C2525BFD0DE0007983B002A00F2
:1068D0002100009604F3D6FCC3E70799112040017C
:1068E0000918B2790120CB7990408343002DCB71F8
:1068F00004D00499049A497A01435172002C9BD028
:106900000599497A014305984172B8E0F078B17869
:1069100000020843810707980D2292018018002980
:1069200084462EDA002C31D0A07AC0072BD00798ED
:1069300000281AD0604611E000E101C0365C365CE8
:10694000365C365C365C365C365C365C64F800047B
:106950005CF8000458F8000429020000806B00284D
:1069600003D080308188491C818000202086401E11
:10697000E0620798FFF73BFF00206063012020875B
:1069800001E0002C02D0059900200874002D02D0EF
:10699000049800210174002F02D00020ACE19BD3A9
:1069A000010000009867000000040000B40970DADC
:1069B00040373874F078B17800020843C0070FD030
:1069C000002D0DD0A87AC0070AD00798002807D05C
:1069D0006046806B002803D080300189491C01810A
:1069E00007984079022829D1F078B178000208434D
:1069F000800723D5002C21D0A07AC0071ED007988D
:106A000039F002FE0700079839F025FE2037797823
:106A100089060BD5069909696031097CC90705D03B
:106A200080300069002801D0012100E00021079892
:106A300021F0A9FBA07AFD210840A072F078B1787E
:106A400000020843C10724D0002D09D00006810FA1
:106A500004980174F078B17800020843C00718D098
:106A6000069800696030007CC00712D107980021A9
:106A70001BF051FD0DE0002F0BD0F078B178000233
:106A80000843400505D5079840790328EED0012832
:106A9000ECD01AF05BFE002C05D0A07AC00702D023
:106AA00007983CF030EC03980BB0F0BDF3B581B023
:106AB00000260198002866D001980D21890144180C
:106AC000606A002802D1FFF73DFD6062019839F04D
:106AD0009BFD01994979022925D105002030407894
:106AE000C10903D1010701D4800641D52F008037A9
:106AF0003868002804D1FFF725FD0028386042D00F
:106B00003868E061019821F054FB002806D0FFF7B7
:106B100019FD852189000028485134D0FF35FF3503
:106B2000AD1C68691FE003290ED1206A002803D13B
:106B3000FFF708FD206207E0E169002907D008316E
:106B40000830542214F332E9E069002802D1FFF73B
:106B5000F9FCE061019821F02CFB002801D1A06A2A
:106B600002E0FFF7EFFCA062002801D00600083623
:106B7000606A002807D0E069002804D0019821F05D
:106B800018FB002802D00020C043FEBD616AE06906
:106B9000029A083000920200019808313300FFF792
:106BA0004CFEFEBD70B514001D0000290AD001285E
:106BB00009D0022801D0042804D10A0029002000AD
:106BC00014F38AE870BD10222900200014F384E831
:106BD0001035200008222900103014F37EE8290027
:106BE0000831082220001830EAE7F8B5040039F02F
:106BF00032FD200039F008FD210020314B7DF722C5
:106C000013404B75A5680426B5432122A560125C8C
:106C100097070AD50D229201C56FA218D561C06FE2
:106C20005062082003434B7505E0100701D490061D
:106C300001D53543A56020003CF064EB0020F8BD91
:106C400030B4C279032312091201121DC27110253A
:106C500083710581C37A40242343C372CC8C5023B3
:106C60001C54837A0124234383728B8C03870B6A21
:106C70004363002314070386C362240F0B00020042
:106C80000C322900200030BC8CE7F7B58CB0060030
:106C900039F0E1FC0090300039F0B6FC2121095CAC
:106CA00004000A0701D4890667D5B168042211439C
:106CB0000D22B1600D999201B518012910D137212B
:106CC00009014718200080300B900068002803D18C
:106CD000FFF738FC0B9908600B980068E86113E037
:106CE0000E99012912D17721C9004718300021F0EF
:106CF00060FA002804D0FFF725FC8521890008519F
:106D0000852080000059A862050007E06D6A2822EE
:106D10002900343101A814F34AE801AF002D02D153
:106D200001200FB0F0BD0D980835012804D10020D6
:106D30002200E832287013E00E98012805D1FF22C6
:106D40000121280034F0A2EA0DE0112040013018A2
:106D5000407A2870B06803210843B060009A30324E
:106D60000E98002804D039002800FFF769FF04E0DE
:106D70000D983B00290004F377FD30003CF0C2EA97
:106D80000020CEE710B504000200803420680028FF
:106D90000FD0C17B20320907090F01290AD002292F
:106DA00008D0032905D15078C00902D16179474341
:106DB00001000000946B0000000400004066056EB6
:106DC0002000FFF769FC10BD51780A07FBD4890643
:106DD000F9D4FFF7D9FB0020206010BDFFB50020DB
:106DE00091B00E0014001A9F1D00002B0B9004D0D0
:106DF000E8790007000F2030E871002C04D0E0791A
:106E00000007000F2030E071002F04D0F879000750
:106E1000000F2030F8712100F37A0C311091290015
:106E20000C310F912100300040310E300E9114F3DF
:106E30007AE905047E7EFE7E7D000700002C75D079
:106E4000002DFCD0B07A042870D2707B317B000218
:106E500008434007A07A02D50121084301E0400819
:106E60004000A072E079F17A000909070001090FDA
:106E70000843E071787839780002084320810320C4
:106E8000A0710E98B27A417A0120904001430E9889
:106E90000D224172B07AB91C0301181A00190C3086
:106EA0000A90801C13F322EF7878397800020843A7
:106EB0000D28E07A04D108210843E072012003E0A4
:106EC000F7210840E07200200A9948700A98B17AC8
:106ED0000170707B317B00020843000702D50E99D8
:106EE000B07A0872A07AC0071FD01198012180687B
:106EF000022208431043119A9060A87AC20702D078
:106F0000EA79120711D10843A872E8793F220009F3
:106F10000001E8710320A8717878397800020843ED
:106F2000288110990F9813F34CEF06E2DBE10A90E9
:106F300011980F21890140180D9030001830002D54
:106F40000C906ED0707B317B00020843810768D5BE
:106F50004007A87A02D50121084301E0400840001B
:106F6000A872E879F17A000909070001090F0843BE
:106F7000E8710A98417A027A0802104328810320B6
:106F8000A871B17A502041550121E972A87AC00751
:106F900034D011980321806808431199886000203B
:106FA0002886401EE8621198FFF735FC00206863D0
:106FB0000120288711984079022842D1119839F090
:106FC0002DFB0990119839F050FB0999203149782F
:106FD00089060BD50D9909696031097CC90705D06F
:106FE00080300069002801D0012100E000211198C3
:106FF00021F0D3F8A87AFD210840A8720D98006905
:10700000FF302130C07F002801D001200B900A986A
:107010000C9B417A007A09020143F07A0F9AFFF73C
:10702000CBFD002C6BD0707B317B000200E0C2E016
:107030000843C10763D04007A07A06D50121084361
:1070400005E0A87A02210843D7E740084000A07273
:10705000E079F17A000909070001090F0843E0719E
:107060000A98417A027A0802104320810320A07115
:107070000E99B07A0874E07A02210843E072A07A8F
:10708000C0072AD0707B317B00020843800614D5EC
:107090000A9920000A7820300274497841740A99CC
:1070A0000422891C0C3013F322EE208E002804D118
:1070B000E06A002801D1401EE062707B317B000253
:1070C0000843C00603D50020606301202087119883
:1070D000032180680843119988600D980069603029
:1070E000007CC00701D101200B900A980C9B417ACB
:1070F000007A09020143F07A109AFFF75DFD002F34
:107100007ED0707B317B00020843410578D5400773
:10711000B87A02D50121084301E040084000B87266
:10712000F879F17A000909070001090F0843F8719D
:107130000A98417A027A0802104338810320B87114
:10714000B17A5020C155F87A40210843F872B87AD4
:10715000C00724D0707B317B00020843800614D521
:107160000A9938000A7820300274497841740A99E3
:107170000422891C0C3013F3BAED388E002804D198
:10718000F86A002801D1401EF862707B317B000252
:107190000843C00603D500207863012038870A9889
:1071A0003A00417A007A09020143F07A0C9B0C32D2
:1071B000FFF702FDBDE00021099005A8E57B98F5E9
:1071C00001000000906F00000004000013BCD60214
:1071D0000A91FF4F8ECF8EC000210A000B000F00D6
:1071E00001A88EC0707B317B00020843810700D567
:1071F0000A95C00700D00A940A9800287DD00A9802
:10720000807AC00712D00A98006D002807D1FFF7D6
:10721000ADF900E094E00A990028086506D00A98C4
:107220000A99006D5422083013F3D4ED119901240A
:1072300049792000022900D00020717B327B0902AD
:10724000114389071FD5002809D0119810218068A3
:107250006B46084311998860187D401C18750A9880
:107260000521C172DB491198062241180A9813F3CF
:1072700048ED1198119A80680221204308439060DC
:107280000A9820304173707B317B00020843C007AD
:107290000BD00A991220C8720A98062113F3CCED7C
:1072A0000A982030447301200B900A98F17AC07933
:1072B000090700090001090F08430A99C8710A99D2
:1072C000032088710998417C027C08020A991043C6
:1072D00008810999102201A833F0C1FF00280DD1BF
:1072E0000A9810222E3005A913F30AED0A981022ED
:1072F0003E3005A913F304ED0CE035E00A98099936
:1073000010222E3005F3AEFF0A98099910223E3064
:1073100005F3A8FF0A98B17A017309990A98102217
:1073200012311D3013F3ECEC09990A981022223126
:107330000D3013F3E6EC0A980A99807A204388729C
:107340000B98002803D0119800211BF0F8F81AF0D0
:1073500011FA002D05D0A87AC00702D011983BF091
:10736000E6EF002015B0F0BD0120FBE7F7B582B0D5
:10737000002702983E00019739F05AF90299029BC2
:107380000D22497992019C1802292AD1050020304A
:107390004078C10903D1010701D480064AD52F00E6
:1073A00080373868002804D1FFF7E0F800283860FB
:1073B0000ED03F68E7610298083720F00EFF0028E2
:1073C0000AD0FFF7D3F8852189000028485103D15E
:1073D0000020C04305B0F0BDFF35FF35AD1C686926
:1073E00023E003290ED1206A002803D1FFF7BEF85D
:1073F000206207E0E169002907D0083108305422F3
:1074000013F3E8ECE069002804D1FFF7AFF8002897
:10741000E06101D0E7690837029820F0DEFE00281D
:1074200001D1A06A02E0FFF7A1F8A062002801D014
:1074300008300190606A002804D1FFF797F800280F
:10744000606201D0666A0836019A00920499029837
:1074500033003A00FFF7CCFCBCE770B505000C0028
:107460000026081D31F001F9002815D1201D31F04A
:10747000EDF8002810D1F120800029180622201DE7
:1074800033F0EDFE002807D0201D39F04FF905003C
:1074900001D1012070BD0126220031002800FFF734
:1074A00065FF70BDFFB589B004001F00129E002E5D
:1074B00077D0002CFCD02000403008902338079073
:1074C00010380690401E059010300490083003904C
:1074D0003801C01B0019029020003E30FF290190A6
:1074E00004D1E07900090228E2D0E4E00229FCD1CD
:1074F000FF209D303070000A70700A20B0700020AC
:10750000F0700B990622301D13F3FAEBE0790007B7
:10751000000FF072E07A410602D50121890204E0F1
:10752000800701D5012100E002213173090A71733E
:10753000E07903071B0F30001900103013F3FCED46
:107540000504323232323100042F2AD2B772089940
:10755000097AB94208D1717B327B090211430822B2
:1075600011433173090A71730299497B002901D1D2
:10757000052100E00D21B173090AF173F17BB37BA2
:107580000A0202991A430E3113F3BAEBF078B2787B
:107590000102F07B1143B27B000210430818801CEB
:1075A00031E02AE135003035032944D1217BB17225
:1075B0002021070081730020F87330000E300199FC
:1075C0001022009013F39CEB10223000EE42448214
:1075D000010000008C73000000040000AC79F3B1DE
:1075E000203003E03867000029020000079913F3F8
:1075F00092EB06991022280013F38CEB0199009866
:10760000102205F339FEF078B17800020843F97BC7
:10761000BA7B0902114340181230B070000AF070B2
:10762000A07AC00708D0707B317B00020843042198
:1076300008433073000A7073F078B1780002084391
:10764000001D0004000C0DB0F0BD08990A7CB27258
:107650002289B275120AF275228E21001378B37353
:107660005278F27304222C3113F354EB002131755C
:107670007175E07901073000090F1830012911D127
:107680002021B1750021F1750599102213F342EB09
:10769000300004990822283013F33CEB08220399A8
:1076A000280005E02189B175090AF175228905993B
:1076B00013F330EBF078B2780102F07D1143B27D24
:1076C0000002104308180A30A7E7E079351D0007CB
:1076D000000F3071000A7071FF20401C3070000AEA
:1076E00000227070B270F270E07A410602D501207B
:1076F000800204E0800701D5012000E00220A8708C
:10770000000AE870E07901071ED1A81D042F7ED27F
:1077100021892971090A69710899097AB94202D146
:107720000121417000E042700770029922890E31F8
:10773000801C13F3F0EAF178B07809020143891C48
:10774000B170090AF17041E00007000F012813D160
:10775000202028710020687105991022A81D13F3BC
:10776000DAEA280004990822163013F3D4EA082232
:10777000280003991E300AE0022801D0042809D10C
:10778000102028710020687105991022A81D13F39C
:10779000C2EA1BE0032853D120892871000A6871CE
:1077A000207BA8710120E871AF1D07991022B81C39
:1077B00013F3B0EA380006991022123013F3AAEA44
:1077C000380001991022223005F356FDA07AC00737
:1077D00008D0E878A9780002084304210843A8707B
:1077E000000AE870F178B2780802697910432A79C2
:1077F000090211434018801D020AB070001D0504E3
:10780000F270E0792D0C000718D0741900E017E031
:10781000FF2121312170090A61700621A170002128
:10782000E1700B990622201D13F374EAE178A27827
:10783000080210432D1D401905042D0C280002E7F5
:10784000002000E7FFB581B0002501980A9EC079AD
:10785000000718D1042B16D3019F002440370120C4
:10786000797AA04001420AD0230601A8009607C8F1
:107870001B0EFFF721FE3618281805042D0C641C7A
:10788000042CECDB05E001A8009607C8FFF714FE06
:1078900005002800A8E5FFB581B00024050016000A
:1078A00080681F0040051DD5287901281AD00228BC
:1078B00018D1280038F0C6FE002E13D1002811D0B0
:1078C0008030006800280DD0F90745D00B9AF121CF
:1078D000890000926A18029908300023FFF7ECFD36
:1078E000040039E0F049B8076E180D2189016D18C0
:1078F00000280EDA686A00280BD00B9A00920A9BC7
:10790000029908303200FFF79DFF0B990918040017
:107910000B91F80710D0E86900280DD00B9A00925F
:107920000A9B029908303200FFF78CFF0B99091867
:1079300020180404240C0B9178050DD5A86A0028A2
:107940000AD00B9A00920A9B029908303200FFF786
:1079500079FF20180404240C200045E5FFB587B00A
:10796000FF2100261F00089CD04B35003000062C5C
:10797000059607D20200079801970091FFF78BFF49
:1079800006007BE0140071E0C8480490FF200390DB
:10799000002002906078217800020843C11FF93965
:1079A0000FD1039901970091E179A0790B0203436C
:1079B000029A07980021FFF76EFF05003F18301864
:1079C00044E00100FF399D3942D107980690E078E4
:1079D000A17800020843062829D3201DCBC853A054
:1079E000010000008877000000040000FFA320DDF4
:1079F00030F04FFE002814D1201D30F03BFE00284F
:107A00000FD10798F121890041180622201D33F07B
:107A10003AFC002805D0201D38F09CFE069001207D
:107A20000290E178A278080210430A2809D3A07ACC
:107A30000390627B237BA2481102194300D0080007
:107A400004900698002809D0039901970091049B9F
:107A5000029A06980221FFF728FF05007F19701986
:107A60000604360CE078A1780002084305998300EB
:107A7000091D41180904090C18180419143405913A
:107A800008990598884203D219208001864285D33F
:107A900030000BB0F0BD70B5060004680834E07922
:107AA00003071B0F934201D0012070BD000712D1C4
:107AB000042910D2250040350122687A8A4090437B
:107AC00068720801401A00190C300F2113F3F2E913
:107AD000687A002804D13068FEF774FD0020306019
:107AE000002070BDFFB581B0040000201D000A9F7A
:107AF0000090A06800264005002827DA2079012898
:107B000024D0022801D0032820D1200038F0A4FD81
:107B10002179032902D16179022917D1002F15D1CA
:107B2000002813D080300700006800280ED0E90735
:107B300052D0C17B0A070399120F8A4202D00399DF
:107B4000FF2949D1FEF73EFD3E6045E00D21029838
:107B500089016718FF281BD15A48854218D1786AD5
:107B6000002802D0FEF72EFD7E62F869002808D0BA
:107B7000FEF728FDFE61386A002802D0FEF722FDDC
:107B80003E62B86A002827D0FEF71CFDBE6223E0E3
:107B9000786A002808D0A80706D5D9208000039A63
:107BA00002992018FFF777FFF869002808D0E80746
:107BB00006D0D7208000039A02992018FFF76BFFA8
:107BC000B86A002808D0680506D56D20C000039A61
:107BD00002992018FFF75FFF00980FE4F7B586B011
:107BE000002707983E00062864D314005EE0FF20BB
:107BF00004900390002002906078217800020843EE
:107C0000304DC11FF93901D1012643E00100FF3990
:107C10009D393FD106980590E078A178000208438D
:107C200006282BD3201D30F034FD002814D1201D50
:107C300030F020FD00280FD10698F121890041186D
:107C40000622201D33F01FFB002805D0201D38F030
:107C500081FD059001200290E178A278080210438E
:107C60000A280BD3A07A0490E07A0390617B207BF2
:107C70000D0205431248054000D1124D0598002819
:107C800008D0029A0092039A049905982B00FFF7F6
:107C900029FF0643E078A178000208433F1DC1197F
:107CA00083000F0418183F0C0419143407988742F6
:107CB0009DD300E00126300009B0F0BD290200008C
:107CC00003040000FFFF0000002810D00D218901EF
:107CD0004218916B00290AD00B695B1C0B61916BF8
:107CE000CB685B1CCB60916B0A6E521C0A6611213B
:107CF00049014018C17980221143C1717047704712
:107D00000548142110B513F3ACE8044801210170B3
:107D100000218160C16010BD60FA02C000B701C0DF
:107D200070B538F0C0FC040033F082FE0500206C12
:107D300002F37FF800212800216433F07DFE70BD3E
:107D400070B50D00080038F087FC0600280038F0F8
:107D5000AAFC04002C34A1793000227AE8300429EE
:107D600005D86030407C824213D30F2204E060309B
:107D7000807C82420DD31022022901D001290DD12D
:107D800020002030017E012908D1217202210176D4
:107D9000A1790022280000F02CFA70BDFF482918B4
:107DA00028002AF0D5FC0A20A07170BD38B5040067
:107DB00038F079FC020020320168937CE8315D1EC6
:107DC000032D01D8496F03E05B1F032B1CD8896F7B
:107DD000137D002B05D07D23DB00994200D30B00DF
:107DE0001900127A012A04D1ED4A9142BE1085741D
:107DF00001000000847B0000000400000BCC5569EA
:107E000000D30A001100002200927D22D2004A43D2
:107E10000300E94840332100FEF704F938BDF8B506
:107E2000002844D0002942D0050060352A7CEB7B35
:107E300012021A431206120E84187134DD271C2018
:107E400027706070DD480278A2704278E270807816
:107E50002071092060715020405CA0710A8E22813F
:107E6000CA6A20000A3004C0060010220C3112F346
:107E700066EF297CEA7B0902114362783000891899
:107E8000891C0A0AE9732A7410300822511A4C0717
:107E9000640F0CD00770611E401C13F316E8287C99
:107EA000E97B000208430019E873000A2874F8BD52
:107EB000F7B582B01400060038F0FFFB0500300073
:107EC00038F0D4FB07002200300001A9F9F732FE98
:107ED00004002AD0F068606120890721001901732D
:107EE0000198722112F3F0EFF12080003218B048AF
:107EF0003118019810F3EEF82C35687901231A0037
:107F0000062800D000222879000704D4E037387A08
:107F1000000700D40023A8788006C10F019810F351
:107F20009FFB039801990160200005B0F0BDF3B5F7
:107F300087B00A000025079805A9FFF7B9FF0028B8
:107F4000089002D1012009B0F0BD079838F0B5FBC8
:107F50000490079838F08AFB0700049804002C343A
:107F6000200000F0AAFD20690290E06803907320D1
:107F7000C0003A180092A07839008006C00FC203F2
:107F8000E8310598803202AB069102F3DCFE0598D9
:107F9000069B010060310A7CC97B16020E43372123
:107FA00009017A18A11C03F37FF8059802006030DC
:107FB000017CC77B0B023B43991B182902DD183952
:107FC0000D042D0C049980310969002911D00799FD
:107FD0000D26B60189198E6A002E0AD0002D03D015
:107FE0005B1BC3731B0A0374896A10000831FFF717
:107FF00016FF21000598221D283102F382FF059803
:10800000017D4B0738210A5D21005B0F183110F309
:108010009DF801000898F9F742FE002093E7F3B5B8
:1080200089B00A000700002005000390380007A966
:10803000FFF73EFF00280A9002D101200BB0F0BDEF
:10804000380038F03AFB0600380038F00FFB069095
:108050000D20800138180890406A340014302C3408
:108060000290200000F029FD20690490E068029A47
:1080700005900092A07811218006C00FC003C901AD
:1080800042180798211D04AB02F35DFEC037B868A3
:1080900001894018A1780A0708D504220092484BAC
:1080A0000822DD210BF34CFE039009E0890607D579
:1080B000002200920822302100230BF341FE05002C
:1080C000039A07982B00A11C02F3AEFF002838D0BA
:1080D000A078800639D50798069A03006030017CA5
:1080E000C07B0F020743069837210901411800257C
:1080F000E832180002F39EFE079802006030017C0F
:10810000C37B09021943CB1B182B02DD183B1D044E
:108110002D0C80363369002B0BD0002D03D0491B6A
:10812000C173090A01740898816A10000831FFF7C9
:1081300076FE21000798221D283102F3E2FE002876
:1081400003D10A9813F358FB77E70798017D4B0793
:1081500038210A5D21005B0F18310FF3F7FF010092
:108160000A98F9F79CFD002068E77FB506000D002E
:1081700038F0A3FA04002A00300003A9FFF798FEA4
:10818000050002D1012004B070BD0D20800130181F
:10819000466A2C341436200000F08FFC20690190D0
:1081A000E0680290202130000FF370FA012209E00C
:1081B00029020000B80B0000D97A000047F731000F
:1081C0004EF731000398D202211D01AB009602F355
:1081D000BAFD039A203410006030017CC37B080292
:1081E00018435F300104207E9073090C0320D07384
:1081F00008020B0A18431074000A50745EBA334D1B
:1082000001000000807F0000000400005816860571
:108210002800F9F74EFD0020BFE7F7B582B00C004B
:10822000029838F054FA0700029838F029FA6846A4
:10823000FDF767FD386C002802D00298FFF784FD37
:10824000E00702D1641E2406240E3D002035AC74E4
:1082500002991122287A52018E1801280AD18037FA
:108260003878002806D1718A029801220DF023FF88
:10827000002426E0012C04D104990298FFF77FFF27
:108280000EE0032C04D104990298FFF7D2FE07E018
:10829000052C01D0072C1FD104990298FFF751FE3D
:1082A000040002D1A87C401CA874029810F0F8F8D1
:1082B000002804D0718A029800220DF0FCFE002CE8
:1082C00002D1287D401C28750298FFF783FD68467F
:1082D000FDF734FD200032E60498002802D004980F
:1082E00013F394FA6846FDF729FD012027E610B53F
:1082F00013E0200038F0EBF9A1682C30C90407D551
:1083000080790A2804D1002207212000FFF785FF89
:10831000E279A179200018F070F90400E9D110BDCC
:10832000FF4910B50988C1840121818400210162BF
:1083300010210FF3B5F910BD70B5050038F0A0F9A4
:108340004B210400C9004018F12189006A1801007E
:10835000FF31FF304131193002F3F1FE2120005D81
:10836000800611D50F208001281800696030007C3C
:10837000C00709D07720C0002018FFF7D1FF0122E5
:1083800000212800FEF7BDFC002201212800FEF795
:10839000B8FC70BD70B5050038F072F9060033F016
:1083A0005BFB04000F2080013118CA6A002A0ED03E
:1083B000521ECA620BD1886AC8622800FFF7BCFF50
:1083C000200033F04DFB2800FFF791FF70BD200027
:1083D00033F046FB70BDF8B5050038F051F90700E1
:1083E0000400F120F8378000732137233E002A185B
:1083F000C9001B0141366118E01802F3A0FE0D21EF
:1084000089016418E069012809D1A820415D28008C
:1084100033003A0088300FF303F90020E061F8BD23
:10842000F0B50600A9B04569280038F050F90B9066
:10843000280038F025F90A900B980CAA04000D20AA
:1084400080012818476A30892C3486190A982890A8
:108450003000633041781437891C2FF047FD28988D
:108460000122E0308446807A0990289807A9030009
:108470008033D86E08900E9804900692059160465D
:10848000C089189AA11C039202910190986E0090E5
:10849000089B099A210028002AF026FE012804D111
:1084A0001121280000F007FB24E00A9B6179FF33CB
:1084B0003A330120062900D00020020020003900B4
:1084C0002031283004920391220031000290954817
:1084D0001832113100911400291801922A00180055
:1084E000AC323B0002F37DFD210030000FF30CFEA7
:1084F000002802D1012029B0F0BD2800FFF724FC9C
:108500000B980021203001750A0003212800FFF795
:1085100084FEF0E7012805D0022803D0FF38401E72
:1085200001D10620704700207047FFB583B00600D8
:1085300000250D990C980291117801910778049902
:108540003020012900D0DD2030700498002806D0AA
:1085500075490322684612F3FCEBB41C0AE0734928
:108560000322684612F3F4EB70490422B01C12F3A4
:10857000F0EBB41D0120207000206070A41C0322C9
:108580002000694612F3E4EB002F04D0380001F319
:108590000FFB05042D0C2806000E03F37FF9E07095
:1085A0000698241D20700698000C6070A41C0025FD
:1085B00015E06B4618782070587860709878A07035
:1085C000019801F3F5FA07043F0C3806000E03F397
:1085D00065F9E0700198241DB8436D1C0190069860
:1085E0008542E6DB0E9820700E98000C6070A41C8B
:1085F000002514E06B4618782070587860709878E1
:10860000A070029801F3D4FA0104090CA39D168608
:10861000010000007C830000000400000E3FE545DF
:108620000800FFF781FFE0700298241D88436D1C4D
:1086300002900E988542E7DB049800282ED00F9810
:10864000002827D00F98017821704078607010982A
:10865000A41C20701098000A6070A41C002509E07A
:1086600011991022200012F37EEB11981034103073
:108670006D1C119010988542F2DB0F980078C009AC
:108680000CD02E490322200012F36CEB0620E07080
:10869000241D03E0002020706070A41CA01B0004B7
:1086A000000C811E717007B0F0BDF0B587B00400FA
:1086B0008C4696460CAD0FA8E0CD07C8009503ADDB
:1086C0000297019607C5200072466146FFF737FF03
:1086D0000004000CE7E7F0B50E000700002189B0A8
:1086E0001BF075FEFF229132512307A908A809F05B
:1086F00034FE002836D0380037F0CCFF079900222E
:10870000103103000D00E8330392049205921A8998
:10871000D988009302920191B07808358006AC1C8C
:10872000C10F321D20000123FFF7BFFF2078287002
:10873000000A07E0460200042902000047F7310062
:108740004EF7310068706078A870010AE9700799E7
:10875000001D8872000AC872FD48089A391838004E
:1087600009F0D5FE03E4F8B506004769380037F094
:10877000B8FF050004000D2080013818406A2C3530
:108780001430009030892900801918310FF3C6FC8D
:10879000002801D10120F8BD0098012140300026B9
:1087A000818000983200066431003800FEF7B3FA89
:1087B000002804D00121380000F087F9EAE73800EA
:1087C000FFF7CCFA34200655206820304078800628
:1087D0000DD50F208001381800696030007CC0077B
:1087E00005D080342069002801D0012100E000215B
:1087F00038001FF00EFDA878800607D52900380044
:10880000FFF769FF0A20A8710020F8BD00220521AA
:108810003800FFF70CFDF8BDF8B5018946690F185F
:10882000300037F05EFF0400010005002C344431B5
:1088300038000FF373FC002805D11121300000F03F
:1088400044F90120F8BD3000FFF788FA00202035F8
:108850002875A079062803D121003000FFF73BFFDF
:108860000A20A0710020F8BD70B50E00C179050086
:10887000807937F046FF06E0AC4206D1E279A17973
:10888000200017F0C4FE040018E0200037F029FF94
:10889000010020318A7CD207F0D0097A002905D066
:1088A0000129EBD18021095C0029E7D02030817CAF
:1088B00032002000FFF7BBFC012070BD002CDBD193
:1088C000002070BD10B5040037F0E4FE002811D080
:1088D0006179E83002290DD1A16849070AD55021F4
:1088E000095C002906D04089C10703D1800701D463
:1088F000012010BD002010BDF8B50E0033F0B6F811
:10890000002E009027D0300037F0C4FE040022D0A3
:108910001B20400125182878002701281CD0022898
:1089200016D1E820005D400709D53000FFF7CAFFE7
:10893000002804D00F2080012018816AC1620D2018
:10894000800120182F7087623900300000F0B1F8E4
:10895000009833F08FF8F8BD2F70F9E7F1B582B0C9
:10896000029837F097FE0D21890104004518686AC6
:1089700000283CD033F07AF801901B2040012618E3
:1089800030780127002833D001282DD10220AF6292
:108990003070E86A01F36BFADB20002280002318B4
:1089A00000926C4A6C480299FDF750FB019833F035
:1089B00061F80298272129F045FDE820005D400775
:1089C0000CD50298FFF77EFF002807D00F21890100
:1089D00000206118C8620298FFF7B8FCA86A010479
:1089E0000298090C00F065F8019833F043F8FEBDD9
:1089F000DB200022800023180092564A5648029934
:108A0000FDF724FB3770EFE770B5050046693000CD
:108A100037F067FE0400B068C00407D55E46BA337D
:108A20000100000078870000000400005DE53629A1
:108A3000288941194879400703D53000FFF798FF8E
:108A400070BD200009312C3000F05DF80028F7D00F
:108A50002034A07C022803D12800FFF7F5FC70BD6C
:108A6000042803D12800FFF788FE70BD062801D036
:108A70000828FAD12800FFF7D9FE70BD3EB5FF22C5
:108A80000400062101A832F052EC002200922000DE
:108A90000E2301AA01A90BF0CFFC32F0F1FF050073
:108AA000E179A07937F037FE07E020002AF073F96A
:108AB000E279A179200017F0B4FD0400F5D1280077
:108AC00032F0E2FF3EBD13B5040037F0EDFD284B58
:108AD00020001C684C21022301AAA0471CBD70B5D0
:108AE00004000D00FFF744F91E482A002118200059
:108AF00029F056FE70BDC168491CC16002D10169F0
:108B0000491C016170477CB504000D00042201A8D6
:108B100012F332E90422291D684612F32EE9019866
:108B2000FF21090202000A40030612029D180300F9
:108B30000A0213401B0AEB18000E1818236998420A
:108B400018D100980140030609025B18010011408A
:108B5000090A5918000E0818E16888420AD1012054
:108B60007CBD0000290200000087930355860000A9
:108B700088F800040020F3E7FD4900201422424356
:108B800052189268002A01D000207047401C01282A
:108B9000F4DB01207047F0B58C001025AC431501C3
:108BA0002C43F44DF44E2C400125AD0565190027EA
:108BB0008400A6193560F04D403564192360EC4CF3
:108BC0000501583C2C19402627736673E84EC907E7
:108BD000583E73516360E37BC90F5B085B000B4336
:108BE000FD210B40D107890F0B43042119430228B3
:108BF000E37302D31900FB200140E173A773A76060
:108C0000F0BDDE4870B5012301688A09C16992018F
:108C10001A43430499431943C1610260D849416131
:108C2000D8494162C162D8498160D849C160D04DFC
:108C30000024283D1420604300224019402112F3F3
:108C400085FE641C022CF5D3C94D0024142060431A
:108C500000224019402112F379FE641C012CF5D347
:108C600070BD70B5FCF745FEFFF7CBFFC84D002483
:108C7000E000001B0002002143190A002000FFF75A
:108C80008AFF641C2406240E032CF1D370BDF8B5B2
:108C900005000020009032F0F3FEB54E07000024DE
:108CA000283E14206043801912F380FE08E04169D9
:108CB000A94204D1380032F0E7FE0120F8BD006877
:108CC0000028F4D1641C022CEBD3380032F0DCFE17
:108CD0000098F8BDF3B589B00998A74980000890BD
:108CE0004018006A4022C101C90D571A09990406AB
:108CF000CB00A74A240E5B1A14201B0248439A1883
:108D0000250002940229079255D299492839401822
:108D1000069012F34BFE06004AE070690A998842F9
:108D200045D130898019006F04900020039701908D
:108D30002BE01C2161430798049A4118486890422F
:108D40000BD1009636680099069838F09FFE00987F
:108D5000002132F083FE7F1E1AE01C226A4307982E
:108D600080181C2212F372E800210800402D00D068
:108D7000681C05062D0E402C00D0611C01980C06C5
:108D8000401C240E0006000E019003998842D0D3A7
:108D90000399019888420BD100963668009906988D
:108DA00038F074FE0098002132F058FE00E036687A
:108DB000002EB2D14EE00999891E01294AD26C4990
:108DC00040182838059012F3F1FD060040E0706964
:108DD0000A9988423BD130898019603012F30EE93C
:108DE00004900020039701902AE01C21614307981A
:108DF000049A4118486890420AD100963668009952
:108E0000059838F043FE009834F00DFC7F1E1AE000
:108E10001C226A43079880181C2212F318E80021CC
:108E20000800402D00D0681C05062D0EA7241F61E8
:108E300001000000748B000000040000A98A439D1B
:108E4000402C00D0611C01980C06401C240E00062A
:108E5000000E019003998842D1D301990398814271
:108E600000D13668002EBCD11C2302993C00594326
:108E70005C4307982200411811F3F2EF099800F0C3
:108E800095F8424A01200899C007384340328918B2
:108E9000086209983B49079A000158390A50079A15
:108EA000401812190021426001734021C91B41730F
:108EB0000BB0F0BDF1B582B0FCF725FD0024012711
:108EC000BF073248A1000E183568280038433060CB
:108ED000306A4000FCD532F0DDFD0190680704D413
:108EE00020060299000EFFF7FFFEBD433560019892
:108EF00032F0D4FD641C032CE3D3FEBDFFB583B078
:108F0000FCF701FD00262148B1000F183868012147
:108F10008907019008433860386A4000FCD5142066
:108F2000184970432839401812F34AFD04001E48BE
:108F300006990818029017E02089059905192878E4
:108F40004007400F88420ED1286F0299801D0622EB
:108F500032F0CBF9002806D104997C2041550698BF
:108F6000290034F07BFB2468002CE5D10198012115
:108F7000890788433860761C3606360E022EC2D327
:108F800007B0F0BDF0660400FFFF00FE00A10090F6
:108F900000A00090B0D701C00700070F40A00080DC
:108FA00050E8008018E501C0290200008100034854
:108FB00008180168012211430160704700A1009068
:108FC000FF4900200872487260390867C866486720
:108FD000FF31491C8860C860B0398864C8648865FE
:108FE000C8658866C8660867486708644864886713
:108FF000C8678031086048607047FEB5040032F0F1
:1090000049FD00900120102C04D0202C02D0402CCF
:1090100000D00020EA4960390A780E00303EA242B2
:1090200010D1E84F8200921953697D6EAB4209D18D
:109030009268BB6E9A4205D14200921952887B8A8F
:109040009A4264D04200921902925288D20702D00A
:109050007D25ED0000E0012580008619B2686B4691
:109060001004000C120C9880DA807769D449381A01
:1090700068436039002A886010D1102C07D1D2488B
:10908000D249784312F3D2EB6B46D8800EE0CE483B
:10909000CF49784312F3CAEB6B46D880402C05D1F8
:1090A000F9F7FFFF7D23DB00584303E06B46D888C8
:1090B000381A6843C2496039C86070690A00C449F7
:1090C00068431161C3495060091A1162C04949429D
:1090D000401850616006400F0BD002984088010A8A
:1090E00002D0000A684300E0BB485064BB4890646B
:1090F000D064FFF765FFBA4901200860B1481470D9
:1091000071694166B1688166029949884182009817
:1091100032F0C4FCFEBDAA480021017241727047C2
:10912000F3B581B00D00A800A54CA64E603CB17807
:109130000719B8688D4209D172780199914205D119
:10914000F16E884202D1616B00291ED19C4A903A8F
:10915000116A401AC10F081841106163506A8142B8
:1091600000DC0100616300910098032111F370EFAE
:1091700000222264E06300992163A063E270A27080
:10918000B868F066B57001987070FEBD70B50426C1
:109190008C4C944D00280ED0F9F71FFF002803D007
:1091A000F9F7B9FF002805D0E088401CE080E868A6
:1091B000B043E86070BD2089401C2081E8683043DE
:1091C000F7E78048C078012800D0002070477D482C
:1091D00010B5C07801282BD00020FCF7A2F80120A0
:1091E000FFF7D4FF764C603C20784006400F1FD13B
:1091F00000F370FA734A80325164106422005032D6
:10920000D36B926B801A9941A16AE26A401A521A92
:10921000824200DB10006268511A814200DC0800C3
:10922000216C081870492064884200DD0100216427
:1092300010BD402010B5F9F720FC0028636018D657
:1092400001000000708F000000040000FA5090F14F
:1092500007D06048008B000A02D0032014F0C7F941
:1092600010BD67490020086066490880032014F09B
:10927000BEF9032013F010FF10BD564910B5603938
:109280000A6D82420DD1002008650878012801D0BE
:10929000022807D14F48012189020183222013F0BF
:1092A000FBFE10BDFFF79DFF4B490120C87010BDAC
:1092B000484910B560394A6D824219D10020464AAA
:1092C00048650320D07008784006400F10D0414810
:1092D00001218902040060340183A06A002804D1BE
:1092E00002F069FDA062FCF7F1FA222013F0D4FE2F
:1092F00010BD70B5374E603E30784006400F24D127
:109300003548C078022820D1324C0821200070381E
:109310000C2261568256914217DA32F0C5FB0500E5
:1093200008F02AFB00280DD0207A401C20723178EA
:10933000022901D0082905D100F3D6F9254A103AAF
:1093400051631063280032F0B3FB70BD10B5F9F71C
:109350008CFF002806D02C48007C00280AD0062864
:1093600008D005E01C48C078002803D0042801D0AC
:10937000012010BD002010BD70B50D00154C603CE3
:10938000A16D814207D10020A06520784006400FE2
:1093900002D0FFF758FF70BD14F034F90028FAD05E
:1093A0000221280001F051FD0028F4D0FFF7CEFF84
:1093B0000028F0D02078074C6034042826D1FFF72D
:1093C00098FF606A0028E6D00021280011F038FFDD
:1093D00070BD000098670400103E040010270000D4
:1093E00050C30000204E00006EBE0000983A0000FE
:1093F000B80B000044B701C0009000906079FEFFF8
:1094000014070004A0060004184D04000828DFD14A
:1094100008F06EFA002802D0FFF76BFF70BD606A9B
:109420000028FBD0280011F02AFF70BDF94870B564
:109430000024007812F3C6FD0500092012F3C2FDD6
:10944000430018188008854200D20124F1482038D2
:10945000C07F012800D90124200070BDF8B5002785
:10946000EC4AED4CE03AD16D2600803E814275D148
:10947000EA4BD86804218843D8601000C765503093
:10948000C36C826CC16D806D851A306B9941401C34
:109490003063E91725606160A268E368A81A994102
:1094A00003D261682068E160A06022692068636976
:1094B0006168121A8B4103D2616820686161206182
:1094C0002268206A6368616A80185941616220627B
:1094D000326B3B0011F342EACE4FE161E03FA06105
:1094E000786C7D22D2003C00811A0A23C034A94244
:1094F00027DA797892008900C9198C468968891A17
:10950000A94210DA607F002802D0401E60774BE04D
:1095100063777069002847D1B562706A401C706239
:109520000120A06140E06377F169BD4A40186146BF
:10953000786489688918884200DB08007864F062E2
:1095400032E0F1698C46411A8A1AAA422CD9637713
:10955000227F002A03D0521E227722E03BE07A7855
:10956000AF4B9200D2199268D218904205D1B169DE
:109570006246891A4018786400E07964796CFF20AB
:10958000F530814200DD08007864FFF74FFF0028C6
:1095900005D0A448796C814200DD08007864306A07
:1095A0002077786CF06201E0306A207778780028C4
:1095B00003D0022801D0032804D1E06A002801D09A
:1095C00098487864B86D002802D1706B401C7063B5
:1095D000252013F061FDF8BD10B58E4CE03CE06D28
:1095E00000F363FC0020E06510BD8A4970B5E039E6
:1095F0000A6E824220D100260E66C86D00281BD05C
:109600000C005034A26E206FE36E616F851A994191
:1096100000F36AF8A26CE36C801A9941002D08DC13
:10962000FF22F532801AB14103D308F0ABFB0028CA
:1096300003D0272013F030FD70BDFFF7CDFF0021D0
:109640000800FFF70BFF70BD10B5724C59E7D979D0
:10965000010000006C930000000400004595B54235
:10966000E03C606D00F32BFC0020606510BD6E498E
:1096700010B5E0394A6E824217D100204866486D25
:10968000002812D008005030C36F826F803003C8AA
:10969000801A9941002805DC684869490068096812
:1096A000884203D9282013F001FD10BDFFF7D6FF33
:1096B00000210800FFF706FE10BDF7B582B01400C8
:1096C000594EE03E706840187D218002C90012F3B7
:1096D000C2E80700002505F3FCFD317838001029A9
:1096E0000AD17178890089198969002904D00D008F
:1096F000002C03D140190AE0002C08D071684919E8
:10970000A14204D37D21A002C90012F3A4E80022E3
:10971000454B009202004B480299883BFCF7BEFC87
:10972000FFF2ECFF414A803AD167906705B0F0BD87
:1097300070B532F0C3F93C4D0600E03D286D0024C1
:10974000002802D000F3BBFB2C65686D002802D016
:1097500000F3B5FB6C65E96D080002D000F3AFFBC8
:10976000EC65286E002802D000F3A9FB2C66686E19
:10977000002802D000F3A3FB6C66300032F0A2F99F
:1097800070BD70B532F09AF905001DF095FA04002D
:1097900007D02D4800218A008258491CA41A0929A3
:1097A000F9DD280032F08EF903F0F8F8002815D022
:1097B000264801694069814210D1002C0ED1002059
:1097C00033F0D8FA002809D133F0D4FA002805D1B3
:1097D0001F480078002801D1012400E0002408F08F
:1097E00075FC012C01D1012807D11A480068002816
:1097F00003D1194C2078002803D1192013F056FC0E
:1098000070BD012002F0B8F920781449401E207084
:10981000FF20F53010F09EFE70BD0A6882421FD115
:1098200000200860ADE7000018680400903E0400C6
:109830000090009048F4FFFF10270000C8050004C6
:10984000C405000499900000F4FD02C000A000804F
:10985000FC17000418060004B70500042795000053
:1098600070477CB5040005F334FD05000E00684622
:1098700015F0B0FB00980199421BB1410B00E117B4
:10988000121B8B4101DA01207CBD00207CBDF0B5AC
:1098900001250024F948FA4F017885B04806420FA7
:1098A000F648002A40787ED0F44B1E00726CE036F9
:1098B000012846D110292FD1FFF220FF3A00803233
:1098C000D36A926A801A994103910290F9F7E7FBF3
:1098D000002808D0F9F7C3FB002804D1E749BA896A
:1098E0008878904279D3E64803998030436B026BC5
:1098F0000298801A994109D3E1488030C16A806A90
:109900006140084302D0F878012878D1DB4A94708E
:10991000D0688FE0080096E0D84B402910D19C70A9
:10992000D8681900801A3039D862096A884200DC88
:109930000800D449D862884200DA0100D962DC709C
:10994000A8E0002872D1F9F767FB002804D0CB49C2
:10995000FA898878904240D3FFF2D0FEC84A80321C
:10996000D36A926A801A994103910290F9F728FB11
:10997000002845D0C148C24A4168926B406C891AA0
:10998000081ABE493039096A814200DB080001909B
:10999000B07812F321FB0700092012F31DFB874268
:1099A00005D8B74800E078E0018AB448817015F026
:1099B00081FFB34FF96B88420AD30198FFF751FF3B
:1099C000002805D0AD488470C470019956E004E0C9
:1099D000AA493A8A8878904203D2401C8870CD7098
:1099E00058E04A6C8868801AA44AC862303A126A01
:1099F000904200DC1000C8628C70CC704AE012E02B
:109A00009F4803998030C36B826B0298801A9941FA
:109A10000DD39B488030C16A806A6140084306D0FC
:109A2000F878012803D0954881781EE00EE0934A2B
:109A300094709068516C401A9049D0623039096A2C
:109A4000884200DC66E7D062D47023E0022819D196
:109A5000F9F7CCFA002803D1F9F7BDFAC417FC4F87
:109A6000010000006897000000040000164F662EF9
:109A700000280FD086483A8A8178914203D2491C47
:109A80008170C57010E08470C470426C0169891ADD
:109A9000C16209E07E48F6E77D49032804D18C7055
:109AA000CC704869801AC8620A20747010E0784E41
:109AB00001281BD1F9F7FDFA00280BD0F9F7D9FAE4
:109AC000002807D1B0787989884203D2401CF5700C
:109AD000B0703DE0B470F068B062B26B316B5300AF
:109AE0009A188918401AF062F47031E0F9F79EFA7A
:109AF000002802D0F57034642AE0F9F76BFA0028E8
:109B000003D063483038006A00E0B068316C604FC1
:109B1000431AB362303F7268BF6AD21B9A4200DCBC
:109B20001300B362B76B9C46326B7B00DB19D21813
:109B300063469A1A564BF262303B1B6A9A4202DA2B
:109B4000081AF57003E06246101A0818F4703064C1
:109B50004F48C078F4E510B511F0E9F8002801D0BD
:109B6000012010BD11F0F9F8002801D0022010BD2D
:109B70004748C0308069002820D1454830380088E7
:109B8000042813D0102813D14148407801280DD162
:109B9000F9F79AFA002809D001208002FAF765FB4C
:109BA00001204002FAF761FB402010BD102010BDDB
:109BB00011F08DFB002801D0082010BD042010BD3D
:109BC00033483021303810B511F39AE9FF2130487D
:109BD000113111F396E92E481021303801802F49B8
:109BE00041612F4981600021418081802D4AC180DF
:109BF00082612D4AC2602D4A7D23C261DB002C4A5E
:109C0000036202612B4A42625A008262020001240E
:109C100020321473032454731E4AC385F030D1706C
:109C20008161126A02770A2281774277C8224263F1
:109C30008163403041602049016010BD10B501F0E2
:109C40006EF8002805D0F9F7BAF9002801D10120F3
:109C500010BD002010BD19480021C1607047174891
:109C600000218160704710B5FF24CC340470240AB1
:109C70004470062484700024C47001714471110A78
:109C80008271C171190A037241720A2010BD00006D
:109C900038670400103E04003C730000204E0000B2
:109CA0001027102750C30000307510275CC100003A
:109CB0004E70F22B94110000F0550000386804003B
:109CC0003EB504006846FFF7CEFF03007621200072
:109CD0006A4608F0FBFB3EBD38B5FF4C60780128B2
:109CE00003D12078402822D00AE0FB49C031C96A5C
:109CF000002803D0022801D0032801D1002916D161
:109D0000F648006EE064606E00F3E3F8F24B082260
:109D10000092F348E26C64330021FCF7C9F9FFF2CA
:109D2000F7FCED4A5032D1679067803203C238BDEC
:109D3000F8B5FFF2EDFCE84A5032536C126C861A0B
:109D400099410D00F9F746F9002814D1E249487805
:109D5000012802D1087840280DD0E048006EC86480
:109D6000CC6A4000E317C11780196941001B994173
:109D700001D20120F8BD0020F8BD38B5D64C60787E
:109D8000012803D12078402822D00AE0D249C031EE
:109D9000C96A002803D0022801D0032801D1002974
:109DA00016D1CE48C06DA064206E00F392F8CA4B65
:109DB00008220092CB48A26C60330021FCF778F9AE
:109DC000FFF2A6FCC44A50329066D1665167106714
:109DD00038BDF8B5FFF29CFCBF4ABF4C5032D36C83
:109DE000926C861A607899410D00012811D0F9F71C
:109DF000F1F800280DD1B948C06DA064646C400032
:109E0000E317C11780196941001B994101D2012054
:109E1000F8BD0020F8BD38B5AF4C606D00F359F8BF
:109E2000B148C16804221143C16008222300009296
:109E3000AE48E26A54330021FCF73AF9FFF268FCBD
:109E4000220050325164106438BD10B5A24CC034A9
:109E5000E06B002810D0A148406F00F33AF8E06BA7
:109E600000F337F8002120004030E163741F9C00AC
:109E700001000000649B000000040000E220139A2F
:109E80004160A04901600420FBF773FA08E7F8B5C8
:109E9000002036F08BFC0600FF219B4800222D316C
:109EA00011F324FD050056D002202873C0202C1881
:109EB0002881A078F321800880000840083000073E
:109EC000000F4030A070E07801210843F1210840E4
:109ED000102108439F210840E070F12080003118D4
:109EE00006220E00A01D10F37AEF2000062231009A
:109EF0000C3010F3DEEF200006223100123010F398
:109F00006EEF002020801C202E1828818421300034
:109F100011F300E8370017206037346778777B4803
:109F2000A0800920B070002036F040FC68617848BD
:109F30000079800607D4B078002804D0B0680121E9
:109F400089070843B06008201521387709022800E6
:109F500007F054FB0120F8BD6549496F814200D1EB
:109F600095E77047614938B5C031C96B814220D14E
:109F7000684C6068002815D00420FBF788F9664813
:109F800020605B48406FFFF2AEFF0822009220681D
:109F90007D210901564B421A604800217433FCF7B9
:109FA00091F804E00420FBF7E4F95648206000F043
:109FB00001F838BD38B5F9F74EF8002829D0F9F77F
:109FC00013F8002825D1F9F704F8002821D1F9F772
:109FD0006AF900281DD100F01FFF012819D123F0D4
:109FE00078F9022815D04B4C01206168002900D077
:109FF0000020606047484038C06BFFF274FF454B5B
:10A0000008220092464822681B1F0021FCF75AF8DC
:10A0100038BDFFF724FF38BD10B53E4C403C206BE7
:10A02000002809D0FFF25FFF00202063A063C82052
:10A0300060630320FBF79DF932E6F3B5502087B04B
:10A040000390029000F0E8FE01282ED1FFF79CF962
:10A05000002805D108983D2802D008983728F4D167
:10A06000224F089B38005030069098303C00012663
:10A07000C034282B05907BD018DC172B79D008DC56
:10A08000022B05D00A2B75D00B2B74D0122BDCD1F0
:10A090000CE3192B70D0262B6FD0272BD5D1FFF7CF
:10A0A000A2FE002801D0FFF772FE5BE30F4D353BA7
:10A0B000603511F3B0E80DECECEBBDBDBDBDBD08E6
:10A0C000EAE9BDE8BD00FFF7A7FFFFF773FF084807
:10A0D000C0780428E9D0F8F787FF002826D1F8F7E0
:10A0E000FDFF002820D1F8F7A0FF1BE0386704002F
:10A0F000103E04007B9300000B9300000090009042
:10A10000D18F0000F0550000B0190004B0360000F7
:10A11000ECE8000438680400504600003D9C000054
:10A12000499C0000002801D07E7029E0F8F75CFF10
:10A13000002803D0F8F736FF00280AD0F8F75FFFB1
:10A14000002806D1F8F766FF002804D038781028D8
:10A1500001D1022013E0F8F768FF00280ED0F9F7CC
:10A1600002F800280AD03878102807D1032006E02A
:10A170004EE2EBE2E1E20FE245E259E100207870C5
:10A18000FFF766FD00287DD0FB480778FFF7EDFC60
:10A19000FEF75BFFF948C0780028F748007848D1FF
:10A1A0004006400F28D000F04AFEA06A002802D1E5
:10A1B00001F01FFEA062079803F09AF800280BD068
:10A1C0000798112149014018EC49027D0A71407D30
:10A1D0004871079814F0BFFCE84F387800280ED17A
:10A1E000F8F702FF00280AD13E70029B039A0798F5
:10A1F0003100FFF76FFD02E0012000F00AFEDF4FA3
:10A200000120FE7000F069FD012005F08BFDDA48A9
:10A21000417801292AD10078402827D10020FE70FA
:10A22000FBF7A7F8FF20401C2883222012F052FFE2
:10A2300098E2B8421AD04006400F0BD07806400F83
:10A2400014D100F0FCFDA06A00280FD101F0D1FD6F
:10A25000A0620BE07806400F08D0012000F0D9FD85
:10A26000A06A002802D0059801F029FE00272F835C
:10A27000FFF772FA00F026FDFAF7F3FF6AB352E037
:10A2800001000000609F000000040000B1FAC0F669
:10A290003800BE4FF86605E028E0CAE1B9E187E181
:10A2A0004EE20DE2FEF7BEFE38784106490F02D1BC
:10A2B0007978FEF767FF31F01FFC0490FFF705FB8C
:10A2C000002853D0B248C6700020FBF75CF83878FD
:10A2D000012804D0022802D04006400F05D0FF20FC
:10A2E000401C2883222012F0FFFE95E0A84DE8785C
:10A2F000002835D0042833D0FFF738FA00F0ECFC02
:10A30000FAF7B9FF0026FE66079814F061FC28787A
:10A31000002806D028222E70079831001300FFF77E
:10A32000E3FC0020FBF72FF80020FEF761FFA06A96
:10A33000002802D0059801F0CCFDEE70A6610A203D
:10A34000A6776077286A2077002000F0D0FC0020F4
:10A3500005F0F2FC38784006400F01D0FEF79BFF75
:10A360008C48C16804221143C16005E2FFF707FC75
:10A37000402806D00020FAF794FF002801D1FE669D
:10A380000EE1834DE878012805D1FFF2D5F92A00C6
:10A390008032D1629062FFF2CFF97C4A5032D163B1
:10A3A00090630020FEF724FF0220E8707948C1681E
:10A3B00004221143C160079814F0D7FB3878400697
:10A3C000400F1FD0002002F0C7FAA06A002802D078
:10A3D000059801F07EFD787800280AD0022808D080
:10A3E000032806D0012817D13878102801D040283A
:10A3F00012D1FFF724FDFFF7AFFC00280CD0FFF7C8
:10A400007FFC09E008220092BA6A6348069B00219B
:10A41000FBF762FEFFF713FD387808280FD00428F9
:10A420000DD04106490F7CD07978002907D0022948
:10A4300005D0032903D0012973D11028FCD10022B3
:10A4400011009EE031F058FB002604903D00FE66AE
:10A45000FEF7A4FF002893D04D4FF878012805D1CE
:10A46000FFF26AF93A008032D1629062FFF264F939
:10A47000464A5032D16390630020FEF7B9FE0220B5
:10A48000F8704448C16804221143C160079814F071
:10A490006CFB2878414F4006400F1DD0002002F091
:10A4A0005BFAA06A002802D0059801F012FD6878D6
:10A4B000002808D0022806D0032804D001284AD159
:10A4C0002878102847D1FFF7BAFCFFF745FC002891
:10A4D00041D0FFF715FC3EE0A86A3A68C1177B68D7
:10A4E0008018A862AA6B5941296B53009A188918E1
:10A4F000411AE9620822009202002748069B0021C7
:10A50000FBF7EAFDFFF79BFC287804280AD1FEF749
:10A5100018FF606A00281ED00798002110F0B8FECE
:10A5200019E031E0082801D0022819D107F008FA13
:10A53000002802D0FEF705FF0CE02878082801D19A
:10A54000606A02E0022805D1286F002802D007982F
:10A5500010F0BDFE2E672878082810D004280ED0F1
:10A5600029784806400F0FD06878002807D00228C5
:10A5700005D0032803D0012806D1102904D1396859
:10A5800000220798FFF7B7F8049896E038670400B0
:10A59000103E0400009000909B8F0000F00100042A
:10A5A000049831F0ADFA002009B0F0BD6662E3E036
:10A5B000FFF7DCF8FAF75FFE0020F866387801282C
:10A5C00025D0022823D0042801D008280BD100F080
:10A5D00083FBFEF72EFEFF48C67000206062288BCA
:10A5E000000AE4D113E04006400FE0D0288B000AB7
:10A5F0000DD0FBF79DF9A06A002802D101F003FC01
:10A60000A062F448C1780229D1D103219DE02E83B4
:10A61000B2E038784006400FC9D0FEF70AFEED4898
:10A62000C670A9E0FFF798FB0028C0D0FFF768FBD1
:10A63000A2E031F061FA397805004806400F3BD0BE
:10A640007878002807D0022805D0032803D00128F5
:10A6500032D1102930D1FFF26FF8DE4CA26FE36FD8
:10A66000801A7A789941012A01D1246C08E0022AE3
:10A6700001D1A46C04E0032A01D1E46C00E0646C15
:10A6800000260B003100201A994115D2C7B1BBBB7F
:10A69000010000005CA3000000040000996B454B22
:10A6A000797800208900CA199169002900D0080032
:10A6B000796808189168441A08D0A04206D300F0BF
:10A6C00015FB079822000021FFF71FF8280031F042
:10A6D00021FA5BE00020FEF795FDA06A002802D079
:10A6E000059801F000FCFFF74BF800F0FFFAFAF7CD
:10A6F000CCFD0025FD66079814F074FA002005F0E3
:10A7000025FBFFF7CAFAFFF7C4FA0020FAF745FE67
:10A71000B64AD06804210843D0600898352802D092
:10A720000898362802D1B048C1700BE0AE48290025
:10A73000C5700278002A05D02822017007981300FE
:10A74000FFF7DCFA0A20A5776077A748A561006AC1
:10A7500020771BE0A448C178042917D10021C170DB
:10A7600014E00020FAF719FEA048C1680422114342
:10A77000C1605EE7FFF704F800F0B8FAFAF785FD6C
:10A780000020F866FFF789FAFFF783FA012015E742
:10A7900010B5FEF70DFE002806D09548007840065B
:10A7A000400F01D001205BE4002059E410B5040003
:10A7B000FEF7FEFD002813D0FFF7EAFF002811D1B5
:10A7C0008948C07802280DD1894809216030415656
:10A7D000012901DB002C05D007F336F9002801D050
:10A7E00001203DE400203BE410B5FEF7E1FD002828
:10A7F00006D07D490120C978022900D000202FE42D
:10A8000001202DE410B5FEF7D3FD002810D07848C4
:10A8100000784006400F0BD002F0F1F8002807D175
:10A8200073486030008BC11FF93901D0012017E453
:10A83000002015E46E48C06E70476D49012008671E
:10A8400070476B48406F70476949012048677047FF
:10A8500067490020486770476648806870476548C8
:10A860000121816070476348C068704761480121D9
:10A87000C16070475E481038407B704710B50400D7
:10A88000FEF796FD00288ED0002C8CD1FEF25EFFE4
:10A89000574A50325163106310001030417A491CFE
:10A8A000417280E710B5FEF783FD002815D0504CAB
:10A8B0002078012801D0042806D14D486030017A63
:10A8C000491E0172FEF747FD20784006400F04D074
:10A8D000FEF23CFF474A303A03C264E7FFB587B057
:10A8E0000D00FEF765FD00287DD0414F00263C009D
:10A8F00021003878383106910839603401280591F3
:10A9000001D0042831D1FEF221FF0B00F96B069A29
:10A91000050005980190039202917A6B34480092E9
:10A920005030416B006B2A0000F05FFC607A401EE3
:10A93000607231F0EBF82C4D0490E878032869D16F
:10A94000386D002802D0FFF2E2FA3E65387801281F
:10A9500006D1012040022083222012F0CFFB59E0D3
:10A96000FEF771FC0120E87054E0022802D0204973
:10A9700008286BD10A980028B6D002F005F8002804
:10A9800031D107F0CBFB0128AED0FEF2DFFE07008D
:10A9900017480B00C16B069A059801901448039262
:10A9A0000291426B00925030416B006B3A0000F014
:10A9B0001CFC207A401E20720120002D00D00020B7
:10A9C0000D4908700998002801D0002D6FD0002093
:10A9D000099031F09BF8044F0490F87803281DD1BA
:10A9E000034D286D0AE02AE0103E0400009000901C
:10A9F0003867040038680400B3050004002802D05A
:10AA0000FFF285FA2E6528780228A2D0FEF71BFCFB
:10AA10000120F870049831F07DF848E0049831F096
:10AA200079F812F021FE002841D0BB4800680028C8
:10AA30003DD106F08FFF002802D0FEF78CFC36E0F7
:10AA4000002D34D0079810F04CFC30E0B34C400699
:10AA5000400F2CD0486B0290C517FEF277FE2700FE
:10AA6000703F3A6B7B6B801A029A99412B00121A45
:10AA70008B410BD2A07F401C0006000E0A28A07755
:10AA800005D3A749086D401C0865A661A67704F3A5
:10AA900048FC79653865FEF259FEA04AE52B453C35
:10AAA0000100000058A7000000040000CAB196276A
:10AAB000F965B865109B403A13637967503238677F
:10AAC00003C209980BB0F0BD994970B5C039097837
:10AAD00015004906490F1CD0603010F3E0EA807879
:10AAE0000009042815D00C2813D0914C203460782C
:10AAF000002808D0280011F3A1FA0600A07811F36D
:10AB00009DFA864200D2A5706078FF2801D2401CD1
:10AB1000607070BD10B5FEF755FC002805D0844963
:10AB200001206039098B012900D1002045E68048C9
:10AB30007021C0380078084070477D486038008B2D
:10AB4000000A0002704710B530F0EAFF30F0ECFF69
:10AB500033E6FEB5764DC03D6878012833D12878BC
:10AB6000402806D1FEF2FCFD2A005032536C126CD4
:10AB700004E0FEF2F5FD6F4AD36F926F871A687892
:10AB800099418000401980680190C317686C0C00DF
:10AB9000C117019AC0196141121A8B4113D268780A
:10ABA000800040198068C117C01BA14161494A6DEE
:10ABB000521C4A65FF22F532904203DA10008A6D7A
:10ABC000521C8A656864E86DFFF2ABF9584B0822A5
:10ABD000009259486A6C643B0021FBF791FAFEF23F
:10ABE000BFFD534A703A9064D164D165906507F017
:10ABF00005F9FEBD10B54E4CC03C206EFFF291F938
:10AC000000202066D9E510B5494CC03C606EFFF2CB
:10AC100088F900206066D0E545492031087070470A
:10AC20004349C87770474249C8627047434A506BEE
:10AC3000010C3F480904F038C08D014351633F4A7D
:10AC4000C03A116B0904090C0004084310637047F3
:10AC500010B5F8F71EFA002805D0F8F7E3F9002838
:10AC600001D10120A9E50020A7E53148C06B0028EB
:10AC700000D00120704738B501202D4CA16B002970
:10AC800000D00020A063206BFFF24BF9284B082274
:10AC900000922B48626B30330021FBF731FA38BD4C
:10ACA00010B5234C216B81420ED1A06B002804D03B
:10ACB0000320FAF70AFB234803E00320FAF777FBA7
:10ACC00021486063FFF7D7FF77E51948006B00283C
:10ACD00000D00120704710B5F8F703FB00280DD114
:10ACE00000F045F8002809D0F8F791F9002805D1BF
:10ACF000F8F712FA002801D101205EE500205CE59A
:10AD000010B50B4CC03CA06D002803D0FFF209F930
:10AD10000020A06551E50D49064A002803D00868C7
:10AD200010670B4800E0106F0860704718060004B9
:10AD3000F8670400103E04007D910000C090009070
:10AD400049A9000030750000204E0000C0A9008015
:10AD500001000300FF4810B54068002805D0FEF749
:10AD600031FB002801D1012010BD002010BDF948A1
:10AD700010B50078012815D1F8F732F9002803D171
:10AD8000F8F750F900280DD0F8F783F9002803D020
:10AD9000F8F748F9002805D022F0B9FA022801D0C6
:10ADA000012010BD002010BD10B5F8F79AFA002858
:10ADB00008D0F8F72CF9002812D0E748007C0628C4
:10ADC0000ED00BE0FFF7D3FF002809D0F8F71FF9EA
:10ADD000002805D0FEF7F6FA002801D1012010BDA9
:10ADE000002010BD10B5FFF7C2FF002809D0F8F70A
:10ADF0000EF9002805D001F0D1FD002801D0012076
:10AE000010BD002010BD10B5FFF7B1FF002803D022
:10AE100014F027FA002807D012F063FC002803D1B1
:10AE200005F048FC002800D0012010BD10B5FEF749
:10AE3000C9FA002802D0FFF7E1FC10BD012010BDC7
:10AE400010B5FFF77AFE10BDC24840687047C1498F
:10AE500048607047BF4800787047BE490870704727
:10AE600010B5FEF7AFFA002805D0FFF760FE002806
:10AE700001D0002010BD012010BDB649002010B542
:10AE8000486006F00EFE10BD10B5FEF79BFA0028D4
:10AE900002D0FEF76AFA10BD002000F0A1FA10BD42
:10AEA00010B506F061FD002809D100F00A0EA8B81F
:10AEB0000100000054AB0000000400003EDEE393FC
:10AEC00089FA002805D1FFF7C9FC002801D101202B
:10AED00010BD002010BDF3B50C0081B007D0022CCE
:10AEE00005D0032C03D0042C01D0012C03D19E48A3
:10AEF0000078012814D135F096FC002803D016F014
:10AF000043FD00280CD00127994D9A4E23007F065F
:10AF100010F3A8E9050484070E7C990000F092FB69
:10AF200091E001983D21FFF7B0F8002875D005E0C9
:10AF3000032C03D101982621FFF7A7F8FFF73EFF66
:10AF40000124A402002837D08748012141600198DC
:10AF500013F029FE00F03BFB012006F0F0F810F0A2
:10AF600082F900280DD0E86B08210843E86320002F
:10AF7000F9F7BAF92000F9F7AAF9E86BF721884345
:10AF800006E010F0D6F9002803D0E86BFF21084353
:10AF9000E863B0683843B06010F065F9002808D065
:10AFA0000FF0F7FE00284ED100F016FC00284AD121
:10AFB00030E0FFF773FF46E0FEF70EFA002818D1E5
:10AFC00006F0BDF8E86B000A0002E863B068B84319
:10AFD000B0602000F9F783F9FFF732FEFFF757FF63
:10AFE00065480168583081422DD1232012F09AF82B
:10AFF00029E0012006F0A3F8E86B000A0002E863EC
:10B00000B068B843B060FFF71BFED2E7FFF7ACFEB5
:10B01000002818D0FFF73BFF15E015E000F02FFBEC
:10B02000019813F0F3FD01980221FFF72EF8FFF7C6
:10B030002EFF002006F083F8E86B000A0002E863A8
:10B04000B068B843B0600120FEBD0FB40020F0B579
:10B050008BB035F0D3FB039001A8FAF7C0FEF8F7E8
:10B060004AF910AB197E18AB0A911E7F10AB1F78FE
:10B0700019790991D97818AB089119790791197A3A
:10B080000691D97910AB05915C7818AB5D790028F1
:10B0900042D022F046F9022870D0AC4205D0012DF2
:10B0A00001D12A20ABE02B20A9E0002F02D0099883
:10B0B00000281BD0089800280ED1002C0CD107982E
:10B0C000002802D00698002804D00598002801D155
:10B0D000002D01D02D2092E0002F02D009980028E9
:10B0E00004D00898002801D1002C0CD00798002823
:10B0F00002D00698002806D00598002803D1002D1C
:10B1000001D12E207BE00A98B0427AD0012E01D1E5
:10B11000302074E0312072E00398002871D012488A
:10B12000007801286DD122F0FCF81349583102282B
:10B1300004914ED0104804990068884249D1002FEC
:10B1400002D0099800281DD0089800281AD1002C98
:10B1500018D10798002802D00698002810D005982A
:10B1600000280DD1002D0AE048020004184D04000B
:10B17000C0A200800090009040D400040AE00AD0F1
:10B1800024203CE0AC4206D0012C3AD103980221A5
:10B19000FFF7A1FE35E0002F02D00998002804D067
:10B1A0000898002801D1002C0AD00798002802D066
:10B1B0000698002804D00598002801D1002DE5D07C
:10B1C0000A98002802D1002EE0D11AE0002EDDD02E
:10B1D00017E033480078012813D122F0A2F80228A2
:10B1E0000FD030480168049881420AD00A9800289C
:10B1F00002D1002E05D001E0002E02D1032011F073
:10B2000091FF01A8FAF708FE0BB0F0BC08BC04B02F
:10B210001847F8B506AC171A70CC8B411900002FEF
:10B2200001DC0020F8BDA74200D9270028680321CF
:10B230004000C0190FF35CEF3900B842286000DB12
:10B240000100B84200DC0700C81BB04200D9300042
:10B25000099909684900081803210FF34AEF099971
:10B2600008600120F8BD262010B511F05BFF10BD6D
:10B2700010B507F089FB0A4C002803D107F032FF14
:10B28000002801D0002000E00120207000F099F992
:10B2900000F0D8F9FEF7C6FC2078F7F7AAFF10BD3A
:10B2A0004802000440D4000410B530F043FCFF49CC
:10B2B0000A69002A03D030F041FC01208A5286D16D
:10B2C0000100000050AF0000000400006D0430FFDA
:10B2D00010BD01220A6130F03BFC002010BDF94B8B
:10B2E000586B020CF8481204C1680A435A6342685A
:10B2F00009040A43F349C0390A63016864390162E9
:10B30000002181621E2281614262C1617047EC4965
:10B3100010B54A69824215D1002008704861FFF7D4
:10B32000DEFFEA480068002801D0172008E00FF08F
:10B33000A4FF002803D110F006F8002802D0212035
:10B3400011F0FAFE10BD38B5DD4C6069FEF2FDFD6E
:10B35000082223000092DE48A26900211433FAF784
:10B36000E3FE38BD70B530F0EFFB0600D948016947
:10B370004069814201D0012400E00024D04D2878AA
:10B38000697808431BD0300030F0E2FB6878002871
:10B3900013D0002C0CD0686A0722401C6862CE488B
:10B3A0000121006831F01DFD212011F0C5FE04E0EF
:10B3B000A86A401CA8620120A870012070BD06F395
:10B3C00061FB002808D1300030F0C2FBE86A401C65
:10B3D000E862FFF7B8FFF0E72878401C28703000DB
:10B3E00030F0B6FB002070BD10B530F0ADFBB449B5
:10B3F0000A7849690A4303D030F0AAFB012010BD46
:10B4000030F0A6FB002010BD10B5040006F0C0FA15
:10B41000002822D0FFF7E8FF00281ED1FFF7AEFC7E
:10B42000002803D00FF08FFF002802D1002C14D089
:10B4300008E0002C06D1FFF795FF00280DD1FFF79B
:10B4400082FF08E09E490020C870FFF737FF002800
:10B4500003D1FFF744FF06F0DFFA10BD98498A6870
:10B46000824204D10020886008610120CCE7704747
:10B4700038B5934CA068FEF268FD082223000092C4
:10B480009648E26800210833FAF74EFE38BD10B541
:10B490008B4CA068FEF259FD0020A06010BD10B5D5
:10B4A000874C6069FEF251FD0020606110BDFEB561
:10B4B0000A21040001AA08F068FF814F0500002658
:10B4C000002843D0112040012018408A032189031D
:10B4D00008430199096F8880200006F09FF9010058
:10B4E00001987F4A817000927E4A1279920606D4B2
:10B4F000002904D081680122920711438160006F06
:10B500001022C178784C1143C17002E00220F9F793
:10B5100093FF06F007FB002801D1641EF6D2FFF767
:10B5200012FF012078700099280006F099F8002891
:10B530000AD1280010F3E2F930F006FB3E707E706D
:10B5400030F006FB0020FEBD0120FEBD30F0FCFA0D
:10B550003E70F5E770B506000C001500002B38D0E2
:10B560000FF0F1FE002834D001F02CFA002830D181
:10B5700006F0F2FD01282CD00120002C00D0002084
:10B580005A490870FFF77AFC012808D1FFF787FFB6
:10B5900030F0DAFA4A4A0021117030F0D9FA12F08C
:10B5A00081F8002815D049480068002811D106F01C
:10B5B000EFF9002803D00020FFF726FF08E0002C59
:10B5C00007D04B480078002803D130000FF0A7FEC9
:10B5D0000025280070BD4748C16B474A1143C1632D
:10B5E00070477CB5F7F727FD3D4E444D344CE036AF
:10B5F00000280AD0694601A8F7F7B8FD009901981C
:10B60000884204D8606B401C6063009601952E4D03
:10B610000198E968814203D12969009A91421AD0C0
:10B62000E8600099421A2A604B22D20029618918E9
:10B63000334A8218914200D811006960216A401A89
:10B64000A8600FF080FE002803D0A868FF38F53806
:10B65000A860FFF744FE7CBD70B530F075FA0600B7
:10B66000FFF71DFF164C00257D202570C00065707A
:10B670002062FFF7B6FF06F038F9FFF708FF114820
:10B680002561416B420611434163300030F060FA9E
:10B6900070BD10B5FDF7AAFE002837D1FFF7EEFB0D
:10B6A000012833D1FFF7FBFE30F04EFA05494A6B13
:10B6B0004B061A434A63024900220A70024921E0FC
:10B6C00050020004C0900090A82F00043BD9D56719
:10B6D000010000004CB3000000040000D2C1154C72
:10B6E000180600048FAF000000A000800C080004C2
:10B6F000DDB0000002040000ECE800047017000058
:10B70000B3050004B4050004C0A20080000200805C
:10B71000A60E000048F4FFFF8A61CA6130F022FAE9
:10B7200010BDF94AD368181A401A01041000806845
:10B73000090C5368F5490204086B120C000C000454
:10B74000104308637047F0B5040085B0FFF7A0FB15
:10B75000012853D101F040F900284FD10FF097FD97
:10B76000002801D0FFF7A5FE0FF091FD002807D1BA
:10B770000FF0F3FD00282CD04034207EC00628D5E1
:10B78000E14C206A0490A56AFEF208F823682200C2
:10B7900007000E002832590810000093083801AB4A
:10B7A00007C33300E169A0693A00FFF746FD606A0C
:10B7B000002808D0A26A216A8A18049949198A4285
:10B7C00001DA401E04E0A16A206AFFF7AAFF1E20EA
:10B7D000606230F0C3F9CD490400C031486B4A06BD
:10B7E000104348630FF053FD002804D0C8490020DF
:10B7F000087006F01BF9200030F0B4F905B0F0BD78
:10B80000C34800797047F8B50400002035F00AF805
:10B810000500F7F784FD00285CD1002D5AD0A868F8
:10B82000C00457D501F0D8F8002853D1FFF730FBFA
:10B8300001284FD121F089FD02284BD0F7F705FCF4
:10B84000002847D030F08AF900902000B049B14C70
:10B85000AE4EB14F11D001200871002005F083FCDD
:10B86000E06B000A0002E063B068B843B060600DAE
:10B87000F8F749FDFFF7F8F929E0002008710120E9
:10B88000FFF703FB280013F0A2F9FFF7B4FE012035
:10B8900005F069FC0FF0FBFC002807D0E06B0821E5
:10B8A0000843E063E06BF721884306E00FF055FDA5
:10B8B000002803D0E06BFF210843E063B068384301
:10B8C000B0600FF0E4FC002801D1FFF7FBFA00980C
:10B8D00030F048F9F8BD70B505008B4C0026E169E1
:10B8E000A0697140704008430FD0A269E36931003C
:10B8F000A81A994109D28649086B401C0863A269BD
:10B90000E369501BB341E361A06170BD70B50400F1
:10B910000D00FDF243FF7C4AD161906129002000B7
:10B9200035F0C6F8FFF7D7FF70BDF7B582B00D0050
:10B930001600F7F7F4FC00280AD0FFF729FA0028D0
:10B9400011D0002D7ED07C20405D07280BD80DE063
:10B95000286F80780007800F06D1FFF761FA002872
:10B9600002D0FFF78FFDEDE0002DEBD0306900280D
:10B97000E8D0286F80780007800F02280BD101F0F3
:10B980002BF8002807D10FF0E8FC002803D0FFF7C0
:10B99000FFF900280CD1FFF743FA002804D0286FE4
:10B9A00080780007800F03D0F7F7B9FC0028DAD0C1
:10B9B0005A4807685A4800780002074330F0CEF82A
:10B9C0000190574834680078143481005548405835
:10B9D000010604D00006000E001F384301E0FC20E1
:10B9E00038430068A0427ED1F7F799FC002833D095
:10B9F0000020F07560880007000F012831D0316801
:10BA0000606860318A7F801C521E1206120E8A778F
:10BA100075D04178090714D401780A07920F022AD9
:10BA200002D1090908290CD03F49096B01220909F3
:10BA3000D20289180A0161680B8B1B071B0F134385
:10BA40000B8300E076E041780822114341700298B0
:10BA50002100F7F708FD04E030686030817F491E5F
:10BA6000817730686030807F002848D0F07D0028E2
:10BA700045D1FC2038430668380004210843FC22E5
:10BA800039002FF0CAEC3E60254828490078800034
:10BA90000A58521C0A5026490A58121D0A50F7F734
:10BAA0003EFC002804D160680822C1781143C170AF
:10BAB00001202070F7F733FC002804D0F7F749FC89
:10BAC000F7F7C8FE16E01149C031486B4A0610432B
:10BAD0004863FFF7EEFC0E4800210170CAEE472EC6
:10BAE0000100000048B7000000040000811BC620D0
:10BAF000286F80780007800F00E00AE001D1012064
:10BB000000E00020FFF794FC019830F035F80120A8
:10BB10007EE6019830F030F81EE00000A82F000407
:10BB20000090009050020004C0A2008000000002BB
:10BB300000A0008038B701C01CFE02C0C0A6008073
:10BB4000F4FD02C044FE02C027480078002803D05C
:10BB500002983100FFF7E4FE002059E610B504001A
:10BB600037290CD007DC21290DD0352901D0362901
:10BB700008D1012004E0382901D0392902D1002060
:10BB8000FFF74BFE10BD00F031FF002826D10FF06B
:10BB900088FB002812D014494878002807D0C869CB
:10BBA000022804D2401CC861FFF7E1FB10BD002051
:10BBB000C861010020000FF0A7FB10BD0FF0D7FBFC
:10BBC0000028FAD005F0F8FE002803D00020FFF787
:10BBD0002FFC10BD20000FF0B6FB10BD0120F6E7D2
:10BBE000014900204870704750020004002800D02E
:10BBF0000120FC4988607047FA48C06870470028F7
:10BC000000D00120F74908607047F6484068704747
:10BC10000020704710B541690979012903D100213D
:10BC200029F0CBFD10BD05F03CFC10BD0100EE4835
:10BC300010B5C069072231F0E8F8002010BDF7B553
:10BC400084B000242500EA480194E84E4269049932
:10BC5000430619430A434261E64BD96804229143E3
:10BC6000D960E34980310A6907231B041A430A613A
:10BC7000DF4BC0331968082291431960DE4B196805
:10BC800002229143196080690290FDF291FD0F003C
:10BC900000902DE0D6486D1C80690290D74800695D
:10BCA0007F214905084003D001214905411A03D1EC
:10BCB000864201D1641C00E000240600FDF278FDFC
:10BCC000009A0023801ACE4AB941121A8B410FD232
:10BCD000CA480169C448C94A8160FF213331803AAA
:10BCE0001161C6498031C968C1600220019002E03B
:10BCF00006988442CED3FDF25BFD009A801ABA4AC0
:10BD0000B9415166106602990498884304D001989D
:10BD1000002801D101200190B74801680222114397
:10BD20000160B349C0310868082210430860B04878
:10BD3000803001690722120491430161AD49C8684E
:10BD400004221043C86005980560019807B0F0BD53
:10BD5000F8B50700FDF22CFD0C0000901DF0FEF878
:10BD6000A14D0026002804D0A6490888B8430880C1
:10BD700003E0A549380002F304F9FDF219FD009A29
:10BD8000801AA1410B000400686D3100001B99412D
:10BD900000D36C6D6C65F8BDF1B584B0924C206C2D
:10BDA000401C20641DF0DAF8002806D09549049A5A
:10BDB00008881043088005B0F0BDFDF2F9FC029040
:10BDC0008D480D004038C66A9049C162884FB869F5
:10BDD000854901908E481E223431FFF730FF02283A
:10BDE00003D16068401C606004E0012802D1206D2E
:10BDF000401C206580484038C662B869E063FDF2A7
:10BE0000D7FC029AE76C861AA9410D007A1C002023
:10BE1000A06CE16C002348430021801969410EF3B6
:10BE200002EEA064E06C401CE064606C0021801BAA
:10BE3000A94100D3666C6664606BA16B884201D92E
:10BE4000606B00E0A06BA063049A019970481143F5
:10BE5000884301D0FFF77CFF226D616C11202CF02C
:10BE600087F8A8E76B480088002804D06A490120B9
:10BE70000978042900D0002070472020D6E6F8B5C4
:10BE800000242600584D2869002801D12000F8BD63
:10BE90002FF06EFE0090E86A01210B00002800D010
:10BEA0000023002001218140EA6A0F00174202D1DD
:10BEB0000C000A43EA62401C002C01D11F28F1DD6E
:10BEC000002B12D0FEF796FC002807D005F03EFEAE
:10BED000002800D001263000FEF7CDFE002E04D150
:10BEE00003F38BFBFF20FFF757FF00983919323817
:10BEF0000100000044BB0000000400007574B3940E
:10BF00002FF044FECCE7F8B500243C4D286900280A
:10BF100001D12000F8BD2FF035FE0090286B0127DD
:10BF20003B00002800D000230020390081402A6B0C
:10BF30000E00164202D10C000A432A63401C002C5A
:10BF400001D11F28F1DD002B05D003F360FB032096
:10BF50000002FFF72BFF00982FF018FED9E770B50D
:10BF600004002FF00FFE050024480022016900297B
:10BF700001D1226070BD2368C16A9943C162226009
:10BF800007D02B48006881430FD1FF20FFF7EAFE5E
:10BF90000BE01CF0EDFF002807D1FF20FFF7E2FEC9
:10BFA00003F32DFB0120FFF74BFE28002FF0EEFDE1
:10BFB00070BD70B504002FF0E5FD05000F480022AC
:10BFC0000169002901D1226070BD2368016B99438A
:10BFD000016322600CD11CF0CBFF002808D10320A4
:10BFE0000002FFF7BFFE03F30AFB0220FFF728FE63
:10BFF00028002FF0CBFD70BD10B701C088020004EF
:10C000004523010040A200800090009000A700801E
:10C0100080A80080A0860100DE3E0400FFFF000033
:10C02000FF7FFF7FFF030000543C00048D060004E7
:10C03000E83E0400F8B50400466900890519FEF7DA
:10C0400003FF002818D0F7F77EF9002814D1286FD5
:10C0500080780007800F0FD1200036F0FCFF200011
:10C0600005F0C8FC002803D00120FFF7EBF9F8BD6C
:10C07000200037F017F80CE03100200000236A465A
:10C0800033F076FC002802D12000FFF7CDFD002818
:10C09000EDD120000FF350FCF8BD38B5E04C606ADC
:10C0A00030F0C8FEE0690522002130F0B8FEDD481E
:10C0B00005220068002130F0B2FE02E000980FF384
:10C0C0003BFC206A04220023694630F0A4FE0F28BE
:10C0D000F4D1D54800250570D44812210EF36AEF3B
:10C0E000D34865700560002038BD70B50E00A821EA
:10C0F0004143D04800250C18A088E188814201D135
:10C10000012070BD81006118896831602621401CC2
:10C110000FF304ECA1808034206A401E2062306856
:10C120001C3844696179022905D1290013F0B5FE54
:10C1300020000CF0B2F9002070BDF8B504000D002D
:10C1400040791600022815D120000DF017F80128BB
:10C1500010D1300002211C3813F09FFE070001218E
:10C1600020000CF07EFC012F04D1AD49886D401CED
:10C1700088650BE0A8216943AE480C18E5882621A4
:10C18000681C0FF3CCEBA088884201D10120F8BDD8
:10C19000A80020188660E1808034206A401C20625C
:10C1A0000020F8BDA348A82110B50EF304EF9C4968
:10C1B0000020886210BD001F10B50406240E042C58
:10C1C00013D2A82060439B494018A8210EF3F2EE39
:10C1D000934A0120916AA04008431021A1400143E5
:10C1E000FF20401CA0408143916210BDF8B5041FA0
:10C1F000042C24D22FF0C6FC0600894DFF20401CE1
:10C20000A96AA04008420AD003E000981C3831F027
:10C21000F6FA20006946FFF768FF0028F5D0FF21F5
:10C220001231A86AA1408843A862A82060438149CE
:10C230004018A8210EF3BEEE30002FF0A7FCF8BD89
:10C24000F8B5041F042C25D22FF09CFC0600744D79
:10C25000FF20401CA96AA04008420BD004E00098CF
:10C2600000211C382FF07CFC20006946FFF73DFFC1
:10C270000028F4D0FF211231A86AA1408843A862A7
:10C28000A82060436B494018A8210EF394EE3000BB
:10C290002FF07CFCF8BDF8B500242500654EFF2783
:10C2A0007F1CA82060435E4935543800896AA0404D
:10C2B000084202D00120FFF7C3FC641C042CF0DB11
:10C2C000F8BDF1B582B02FF05DFC00905A495B4893
:10C2D00037F0EEE8FFF7DDFD01900298FCF762FE13
:10C2E000574F002426000120250638602D0E0299A4
:10C2F00028001DF052FC029928001DF014853A9C7C
:10C300000100000040BF00000004000026AE60F8FD
:10C31000AFFD641C042C3E60EFDB01A8FFF729FE93
:10C3200000982FF03DFCFEBDF7B582B00025060059
:10C3300015F0F5F8002801D1002050E500216846ED
:10C3400020F0E2FFFF212D31300008F027F8040033
:10C350001DD01C202700C03725182081202138003F
:10C360000EF35CEEB878F321800880000840001DD1
:10C370000007000FB030B8706B462F671878800741
:10C38000800F012801D1052000E00020A8702700BF
:10C3900041D0314801902C6F03992171090A6171D4
:10C3A000002121706170E078062241084900FD20DB
:10C3B00001402A48E1703118A01D0EF36AEDF1200A
:10C3C00080003118200006220C300EF362EDCC20E4
:10C3D00060357E61687704980224022819D004DC55
:10C3E000002807D0012816D104E0032804D0FF2834
:10C3F00011D10820287700E02C770199380005F04A
:10C4000057F9002807D01649086920430861012020
:10C41000E5E40320EEE738000FF398FA8CE71148C3
:10C420000088002805D010480178032901D1042193
:10C4300001707047880200040C080004FC17000417
:10C4400028CB0004F807000488C800041111FFFF7E
:10C45000BBBBBBBBE43D0400021500002902000089
:10C46000C0A20080543C00048D060004FF484078C0
:10C470007047FE4948707047FC490020886070474B
:10C48000FA490020C8607047F7B582B00600F74D42
:10C490001700E86800285FD10398FEF7CDF900285F
:10C4A0005AD0FF21F24800222D310FF379FA04000F
:10C4B00052D001200221E86021736661617B014353
:10C4C000EC486173A061C020208111204001301828
:10C4D000428AE9480092006832000379F120800026
:10C4E0003118AC32200001F3CEFB01901C2025183E
:10C4F0002081842128000EF368ED28003900603087
:10C500000700417701982867300005F0AFF9DB4E4E
:10C51000A870FEF768FC002800D1D94ED9480079F0
:10C52000800607D4A878002804D0A86801218907CC
:10C530000843A860FCF782FF002802D0FEF7E0F96C
:10C5400000E0032038773100200005F0B1F8002822
:10C5500005D120000FF3FAF9002005B0F0BD0398D3
:10C56000FEF7D2F90120F8E7FFB589B007000020F7
:10C5700005900C9800281AD0BC488168002916D074
:10C58000C1490A6949698A420BD041680722491C9E
:10C590004160BE480121006830F04BFC212010F0C2
:10C5A000F3FD0DB0F0BD0120F9F7E0FB01E0FF2441
:10C5B0002D342100380007F0F1FE0500F3D0288962
:10C5C00039794619F12080003C183800AC30062932
:10C5D000089002D10C2006900BE0380034F006FAE7
:10C5E000002801D00C2000E00420069038790628AD
:10C5F0000DD1A748089A3B180192069A02213000F3
:10C60000009401F37DFBF078400840000BE0089AAD
:10C610000192089B069A02213000009401F370FBFE
:10C62000F07801210843F070F078EF2108400A9972
:10C630002C00C907C90E0843F070FF20C01C3071E0
:10C64000000A70710020307070701C202881022058
:10C650002900287330311C340491842120000EF30A
:10C66000B4EC21006031139807917728487701D006
:10C67000782804D1A068012149060843A0602667F4
:10C680000C9800280AD00120C007A060774801213B
:10C690008160687B084368737E48A8610020208021
:10C6A00006980C281FD10B99380034F0ABF94107DC
:10C6B0002078490FC008C000084341072070490F87
:10C6C000380034F0CAFA0101206F028B1207120FF2
:10C6D0000A430283206F017E09090901017620784F
:10C6E0009F21084020700B9A21003800002334F06D
:10C6F000B8F91298002827D1FEF790F8002818D032
:10C70000079908200877002138002AF01BF34134EC
:10C71000010000003CC30000000400002457B8EEF4
:10C7200021F8A0700A99002914D00FF3CDFC06005F
:10C7300009200FF3C9FC864201D90920A070A07816
:10C74000FEF7B0FA06E0079809210177380005F0F6
:10C7500097F823E001200003059021E00021380034
:10C760002AF000F80328A0701AD94B480079C006B7
:10C7700003D53420C05DFE280CD0787902280FD173
:10C780000F2080013818806A0521C90140180078FF
:10C79000000705D50321380004F0DEFFA070D9E7BB
:10C7A0000798407F772803D0782801D0412804D10A
:10C7B0000520A0700120000305903748007980060D
:10C7C00007D4A078002804D0A06801218907084375
:10C7D000A06004990598C86139002800002303AAC5
:10C7E00033F0DAF8012800D1E5E6FEF773FB002804
:10C7F00012D0129800280FD0280036F040FC05997E
:10C80000280005F026F9002802D0FEF783FBD2E6C7
:10C81000280036F05BFC05E00599280004F052FF83
:10C820000028F4D1280018F00DFD28000FF398F827
:10C83000C1E6FFB5FF212D31060085B007F0B8FD38
:10C8400007007ED0174831793418012902D0707959
:10C85000022804D12100300034F0C4F802E0300096
:10C8600034F0CEF86B460390187EF3210840083070
:10C8700018760399002919D00007000FC03018E07E
:10C8800020B701C0B0190004B1C00000C00000040E
:10C890000204000002140000ECE8000400A0008084
:10C8A0000C08000429020000A9C000000007000FC6
:10C8B00040306B46187638893200C519F120800067
:10C8C000AC32311801920091187E049002090007E1
:10C8D000810F2300280001F31DFAFF20C01C2871DE
:10C8E000000A687104986B46A870587EE8707079E9
:10C8F00002280DD1022130000BF085F9E9788A0673
:10C90000D20F1043C007DF22800E11400143E970AF
:10C910001C203C1838813800256708997C30417705
:10C920000E9901770398002835D06B46988B2080AC
:10C930007079032820D1300018F09FFB01003000EF
:10C9400000E03EE034F068F841072078490FC00865
:10C95000C000084341072070490F300034F087F9C8
:10C960000101206F028B1207120F0A430283207805
:10C970009F21084020700EE0A64A50880101401C0B
:10C980005080687E2A7E000210430007000F084393
:10C990002876000A68760021300029F0E3FEA070B6
:10C9A0000898382810D00898312812D03100380063
:10C9B000002302AA32F0F0FF01280AD102980028D1
:10C9C00011D0012009B0F0BD93490869022210433B
:10C9D00008610021380004F075FE012803D03800FA
:10C9E0000EF3BEFFEDE70020ECE702008B4810B528
:10C9F000006804210023F9F70CFA002804D1022072
:10CA0000FFF732F9002010BD012010BD70B5040001
:10CA1000834D28680079A04201D032F018F82868C8
:10CA200004718048446170BD10B533F01CF90028D2
:10CA300001D1012010BD002010BD774970B501253E
:10CA40008031096B490719D5FF2804D1002405F06E
:10CA5000A1F9010001E001000400734B1E1F0AE070
:10CA6000E000C218126880190068824200D00025D8
:10CA7000641C012D08D18C42F2D905E06B48816A13
:10CA8000C06A814200D00025280070BDFF2010B58B
:10CA9000FFF7D3FF002801D005F076F810BD6448F9
:10CAA00070B5007800284BD1624800220068082148
:10CAB000FCF26BFE002843D1FFF7E8FF00283FD0CF
:10CAC0005D48FBF25EFB04005B480821FBF2E8FADC
:10CAD000050059481021FBF2E3FA281884422FD1AF
:10CAE0005648FBF24EFB040054480821FBF2D8FAEA
:10CAF000050052481021FBF2D3FA281884421FD1B6
:10CB00004F48FBF23EFB04004D480821FBF2C8FAF7
:10CB100005004B481021FBF2C3FA28187771AA745C
:10CB20000100000038C7000000040000778D6B8210
:10CB300084420FD14848FBF22EFB040046480821EE
:10CB4000FBF2B8FA050044481021FBF2B3FA2818AA
:10CB5000844201D0002070BD012070BD70B501205D
:10CB600014F08DFF00285ED12F4C364D364E08E074
:10CB70002078401C20700120FFF780F80120F9F791
:10CB800009F928780028F3D1306800220821FCF246
:10CB900006FE0028ECD102E00120F9F7FBF8FFF7D0
:10CBA0007FFF0028F8D02948FBF2F5FA0400274857
:10CBB0000821FBF27FFA050024481021FBF27AFAE3
:10CBC00028188442E8D12248FBF2E5FA0400204804
:10CBD0000821FBF26FFA05001D481021FBF26AFAEA
:10CBE00028188442D8D11B48FBF2D5FA0400194812
:10CBF0000821FBF25FFA050016481021FBF25AFAF1
:10CC000028188442C8D11448FBF2C5FA040012481F
:10CC10000821FBF24FFA05000F481021FBF24AFAF7
:10CC200028188442B8D170BD20B701C0C0A20080CE
:10CC3000A8020004C000000440A6008034A90080BF
:10CC400000A00080FC170004000000046C19000420
:10CC5000B0190004A41A0004401A00040922920129
:10CC6000801889080E2210B50AF317FA800010BD4B
:10CC700070B505000C0016002EF0A2FF0021256003
:10CC8000A171E67108340A0006C42EF09DFF012050
:10CC900070BD10B504000C235843FF494018002113
:10CCA0000A000B000EC0200002F356FE200002F323
:10CCB0005EFE200002F345FE10BDF7B586B01400FD
:10CCC0000600F64A0020009204900798210004AA6A
:10CCD00003AB00F3E4FD6B46187C001F03286AD801
:10CCE0002006000E05900FF323FB0FF332FB050027
:10CCF0007079032806D16B461B7B05992A0030000A
:10CD000018F0D4F92EF05CFF0190E5484769012442
:10CD1000AC402740FFF7DBF82404240C02902000ED
:10CD2000FFF73EF86B46187BB823DB4A5843303296
:10CD300080180021A0300173D7496B46D94A187C6E
:10CD4000383900F361FD6B46197C187B04F399FBBD
:10CD50006B46187CFFF768FA6B46187C059A290029
:10CD60003300FCF761F96B46197B280004F397FA4E
:10CD70006B46187C320029001CF0BBFF6B46187C08
:10CD800029001DF057F8002F02D02000FFF72CF8E3
:10CD900002A8FFF702F901982EF016FF6B46197BE7
:10CDA000079A30001DF0EFFF6B46187BFFF771FF0D
:10CDB000012009B0F0BD0020FBE7F7B584B0050005
:10CDC0001600B64A009200240598310003AA02AB6F
:10CDD000039400F364FDB54FB349380036F086EB99
:10CDE0006B46187B001F032847D8F913380036F02C
:10CDF0007EEB3006000E0FF39BFA0FF3AAFA2EF02B
:10CE0000DFFE0600FFF763F86B460190187AB8233F
:10CE1000A149584330314018A0306B460473A14AF1
:10CE2000187B683900F3F0FC6B46197B187A04F321
:10CE300028FB6B46187BFFF721FA2800FCF7D0F897
:10CE40006B46187A04F3C4FA6B46187B29001CF071
:10CE5000C2FE6B46187B29001DF01EF801A8FFF7E3
:10CE60009CF830002EF0B0FE6B46197A059A280027
:10CE70001DF089FF012007B0F0BD0020FBE7F8B5E9
:10CE80000D00060000242EF09BFE844A07002906B0
:10CE9000090E603230000EF377FF0A280DD27F4A68
:10CEA00000210001603211548018C1602900300057
:10CEB00004F330FC14F03AFD012438002EF084FE17
:10CEC0002000F8BDF0B50400002085B0019008787E
:10CED0000D000007400F16D104F3C1F80700042825
:10CEE00011D0704800F3C3FC0600401C0BD038067C
:10CEF000000E3106090E020004900F00280004F312
:10CF00006BF9002802D1002005B0F0BD607902283D
:10CF10000FD1200033F068FC0521C9014018807A48
:10CF200080070BD55F20005D800707D52DB3C2D1E8
:10CF30000100000034CB00000004000083E21E3634
:10CF40000120019004E0200029F01FFB0028F7D108
:10CF5000019904981DF095F82A00049914322000D4
:10CF60001DF005FF281D0EF3F4E80006000E0FF378
:10CF7000E9F90FF3F8F9029052480068012807D147
:10CF8000B420005B03214902884201D336F0BCEA99
:10CF9000607903280AD1281D0EF3DAE80106049B04
:10CFA000090E3A00200018F08BF801E0022803D1A6
:10CFB0000299300018F035F91F204001201800793F
:10CFC000002806D002200FF3CEF90100300018F03F
:10CFD0001EF93D483D4A416A02984000A430085A73
:10CFE000904201D18031C8690104090C380003F076
:10CFF0004AFF012004F0F3F8300004F3FFFA2B4A53
:10D000000120B100383A5050294A0092049A3B005E
:10D010002900200000F332FB3800FFF7F4F82EF06F
:10D02000D9FD0600FEF75DFF0390281D0EF390E882
:10D0300002060298120E23003900FBF7FFFF281D9D
:10D040000EF386E802060299120E230038001CF047
:10D05000A3FE281D0EF37CE802061D480299231842
:10D06000120E38001CF0A5FF03A8FEF7A0FF300049
:10D070002EF0B4FD012051E7F3B581B006002EF08B
:10D08000A9FD0B4F0024009018206043395C002953
:10D090000BD0C51968780FF355F90FF364F9B04256
:10D0A00003D1E878029903F0EEFE13E074CC00049B
:10D0B0003CCB000440A20080041800046666FFFF19
:10D0C000BBBBBBBBD00600043CC70004FFFF000095
:10D0D00029020000641C2406240E042CD4D30098DA
:10D0E0002EF07CFDFEBDF8B500252D4F18206843BD
:10D0F000395C002924D0C419201D33F0FDFB060043
:10D100001ED061780022300014F094FE6B4619881E
:10D1100000010907090F0143009118780009000177
:10D120001870A078009904F32DF86B461888290030
:10D1300000096081002020736073300000F05DFE04
:10D140006D1C2D062D0E042DD0D3F8BD70B5050035
:10D150000C0002F316FC0C216943124B5A581218AA
:10D160005A50226070BD70B505000C0002F3FEFB42
:10D170000C226A430B4951188A6812188A6022608F
:10D1800070BD70B505000C0002F3E5FB0C226A438C
:10D19000044951184A6812184A60226070BD0000A4
:10D1A0003CCB000474CC000470B50500002433F0BF
:10D1B00025FB0600280013F034FC0F2189012B7990
:10D1C00069180EF3A0E807050F050511110F1100EE
:10D1D0006979022902D1340064340CE000290AD0B4
:10D1E000046808E08C6A06E02EF0F4FCFF48F3F7D0
:10D1F0006FF9F8F77DFE200070BD70B505000024C2
:10D2000013F00FFC2979002908D0012908D003293F
:10D210000CD16979032901D001290FD144680DE0AF
:10D220000F2080012818846A183407E02EF0D2FC01
:10D23000EE48401CF3F74CF9F8F75AFE200070BD99
:10D2400070B50500002413F0ECFB2979002908D003
:10D25000012908D003290CD16979032901D00129BA
:10D260000FD1C4680DE00F2080012818846A25348E
:10D2700007E02EF0AFFCDD48801CF3F729F9F8F742
:10D2800037FE200070BD0179012905D10F218901E8
:10D290004018806A353070475D30704770B50400C3
:10D2A000FFF782FF0500200033F0A8FA6179022918
:10D2B00004D10521C9014018807A0CE006F02AFF4C
:10D2C0000F21890161180128086902D12030807F6F
:10D2D00001E02030007FC006C10F08D020002900E7
:10D2E0005D3000F3FFFE002801D0012070BD00205A
:10D2F00070BD70B504000D0033F080FA6179022929
:10D3000004D10521C9014018807A12E0207906284D
:10D3100002D15F20005D0CE006F0FCFE0F218901C8
:10D3200061180128086902D12030807F01E0203097
:10D33000007F81064006C30FCA0F2000F460D803A7
:10D340000100000030CF000000040000D038CD5AAA
:10D3500029005D3000F3DEFE70BD70B50400407939
:10D36000022802D02079062806D12000FFF726FFE8
:10D37000C0784007C00F70BD2000FFF71FFF0500F9
:10D3800006F0D2FE0F218901020061180969002010
:10D39000012A02D12031897F01E02031097F8907EC
:10D3A000E9D5E9788907E6D0012070BD8168890454
:10D3B0000AD57030817B427B080210438005914979
:10D3C000400F800008587047092000027047010094
:10D3D000603040788A688007800F920409D57031E8
:10D3E0008A7B4B7B110219438905490F884200D87B
:10D3F0000800704780684006C00F704701008968C8
:10D4000000204A0602D5090600D501207047F7B56D
:10D4100084B0002406000F00FFF7D0FE05003000A6
:10D42000FFF7F5FE03903000FFF714FF0200300015
:10D43000FFF733FF0300B0684006C00F0AD003981F
:10D4400000216E4607C61A00069938002B0000F32B
:10D4500078FE0400200007B0F0BD08B50168836ABB
:10D4600001290AD1002202600100674A18000092D7
:10D47000664A674B1C3100F3DBFE08BDF8B50D00B2
:10D48000FF21040017002D3106F0B0FF00282860AE
:10D4900011D0018922004618AC32F1218900009296
:10D4A0003A0061180D2306F0F5FF03202036307096
:10D4B0002968C0200881F8BDF7B5FF2105002D318E
:10D4C000544882B02E18280006F090FF04001BD0AC
:10D4D00020892A00AC32F12127188900009220000F
:10D4E000320069180D2306F0D5FF0420203738706C
:10D4F000C0202081049A0399200001F3F3F9200051
:10D5000007F006F805B0F0BD0020C043FAE7FFB50C
:10D5100087B01C000600002006903F4840680028A5
:10D5200002D03D480BF350FB3B4F089818370028BA
:10D5300030D12079E178000208432BD130790128DD
:10D5400004D07179022901D0062807D16079002220
:10D550008006010F300014F077FC05E0607980064A
:10D56000010F300017F0B6FE050060796B461875A4
:10D57000A0795875244AF120800003922349099A22
:10D5800030180291019000927A89059B29003000A1
:10D5900000F3C0FF30001FF007F905006079C321D8
:10D5A0000840397A23008906090F89000843607111
:10D5B000069A0092099A0899280000F37CFF280037
:10D5C0001FF069F90BB0F0BD7CB504002EF00CFB28
:10D5D0001249050048686B46401C4860E079987025
:10D5E000207AD870A07A617A000208439880E068B7
:10D5F000631C012269461FF0A3FA280010E0000016
:10D6000003000100483704003BD000003CCB00047D
:10D610009CCB00042902000040FD02C030B701C0CD
:10D620002EF0E6FA7CBD7FB504002EF0DDFA050091
:10D63000FE4A210001A801F33FF9002807D001228A
:10D6400000922069621C022101ABFFF760FF2800F5
:10D650002EF0CEFA7FBDF8B50D00012441790229E4
:10D6600015D10F2189014118096801290FD133F023
:10D67000F6F8060028000EF36FFE8521895D009103
:10D68000010000980BF05AF9002800D00024200077
:10D69000F8BDFEB50400401C33F038F9E44F050036
:10D6A0004AD0A8684006C00F46D0207A8006010FF5
:10D6B0002800FFF7D0FF00283ED0207A8006010F17
:10D6C00001916879032801D001280BD1280033F09B
:10D6D000C1F9217A0600C32001403007800E0143C2
:10D6E000217200E00E00D3493200200000F3B4FFA5
:10D6F000411C39D0621C280002A9FFF7BFFE029826
:10D70000002819D000223100280014F09DFB0100F0
:10D710000298220000F378FF207AC3210840019983
:10D720000907890E08432072C048E1790170029808
:10D7300006F0EEFE401C01D1380013E0BE480E2278
:10D7400021000DF3CEEBBC4805611838A64A4256BD
:10D75000010000002CD30000000400006FFDE8E988
:10D760000BF3CCF9B94864220092B94AB74B0121B6
:10D7700018380BF302FA0120411C16D1617B227B81
:10D7800009021143E181E17AA27A0902114321736E
:10D79000090A6173217AA172617AE1720121002282
:10D7A000217262722170A6490A70FEBD7CB5040028
:10D7B000401C33F0B5F8A34E050012D0A86840060F
:10D7C000C00F0ED0621C280001A9FFF761FE01986E
:10D7D000002806D0210000F363FF019806F0A2FEA6
:10D7E0000600701C02D10120207020E0607A217AAE
:10D7F000000208431BD1974A0092974A00212B0050
:10D80000200001F398F8A07A934A8006010F601C6B
:10D810000EF3D8FA0A280AD2E17AA27A0902114351
:10D820008A098E49000141182800FFF73FFA3000AD
:10D830007CBDFEB50400401C33F072F8814E05003B
:10D8400003D0A8684006C00F01D13000FEBD687942
:10D85000032801D001280AD1207A0109280033F0D9
:10D8600003F9217A0907090F000101432172E079C8
:10D870006B461872207A587202980190A07A617AE9
:10D8800007020F43621C28006946FFF701FE00985B
:10D89000002801D1300006E001993A0000F359FD5B
:10D8A000009806F03FFE411C02D101212170FEBD0F
:10D8B0000028FCD165480B2221002C300DF31AEB17
:10D8C00062482C30C56018380BF318F95F486422A1
:10D8D000143003000092624A012118330BF34DF912
:10D8E0000120FEBD70B50B004A780D7811020F22A1
:10D8F000920180180069002429435C30012902D17B
:10D900000422991C02E001000422981C0DF3F2EAA3
:10D91000200070BD10B5FFF7D9FD002800D101200F
:10D9200010BDF7B582B005000E004F6B8C6BFFF792
:10D930004FFCA9684906C90F0BD02979012909D1E3
:10D94000484A2B0000924848049AAC33310000F357
:10D95000EDFEE1E56979032901D00129F9D1002C17
:10D96000F7D0002FF5D001794A07D30F227952075B
:10D97000D20F934204D0FB2319409200114301714E
:10D980000179CA06D30F2279D206D20F934204D06E
:10D99000EF231940120111430171C1780A07D30F17
:10D9A000E2781207D20F934204D0F7231940D20035
:10D9B0001143C170017922798B0792079B0F920F57
:10D9C000934203D089088900114301712800FFF7B1
:10D9D00079FC02000021280029F059F99CE570B576
:10D9E0000400C8798A7905020F20800115432018A8
:10D9F00002698B782032012D02D0022D36D109E048
:10DA00001377CB78537700690A79403002704979EF
:10DA1000417008E09377CB78D37700690A7940307A
:10DA200082704979C170200010F002FF2000FFF7DA
:10DA300049FC02000021200029F029F970BD0000F6
:10DA400030B701C0FFFFFFFF3CCB000458FD02C010
:10DA500007D200003BD000009CCB000488CF00041C
:10DA6000A9D10000404B4C00F0E800041377CB78BC
:10DA7000537702690B79403213704B795370026906
:10DA80008B782032C6E710B5CA798C7913020F2241
:10DA900092018218106923432030022B0AD1837F20
:10DAA0008B70C07FC8701069403082780A71C0786E
:10DAB000487110BD037F8B70407FC8701069403083
:10DAC00002780A714078F3E7F8B505000E000024EB
:10DAD000FE4B310020006A46FFF243FE012808D1C8
:10DAE00021003000FFF7E9F900222100300000F3A7
:10DAF000E8FBF74A31002000FFF262FE012809D15D
:10DB0000220031002800FFF776F9012221003000C1
:10DB100000F3D7FB641C2406240E082CD8D3F8BDD0
:10DB200038B50400FFF754FB0500A068C021884306
:10DB30000022A060E74811001300009200F333FEBA
:10DB4000207901280AD100220F208001201800929C
:10DB5000806A11003530130000F325FEA7045E37FC
:10DB60000100000028D70000000400003C273B858E
:10DB7000DE4A20000092DE4A29005D30002300F3D7
:10DB80001CFEDC4821182000FFF7A8FF002211002E
:10DB9000200029F086F838BD0022010010B5403180
:10DBA00082870A80C2874A8020390A7F20231A434D
:10DBB0000A778A7F44301A4342231A438A7718210E
:10DBC0000DF33EEA10BDF8B50E000189456909184C
:10DBD0000C6F28001AF001FC002807D0E0784006FE
:10DBE00004D52188200020300F1801E027002037BD
:10DBF000380000F342FE002813D0BB4AA31D483270
:10DC000000921C002A003900300000F3F9FD0006E4
:10DC1000000E05D023003200390028001EF0A4FFBA
:10DC2000F8BD380000F333FE0028F9D02879022827
:10DC3000F6D03200390028001EF0ABFFF8BDFFB56A
:10DC400083B01400039832F0F7FD4B21C90040184F
:10DC50000290002001906078217800020843052896
:10DC600064D9401F04060498240E401D00900398B8
:10DC7000C179007912F0B5FB32F005FE092686570E
:10DC80000700007A083780063500800F0B21012835
:10DC90000BD1F21E012A00DDF01E050608002D162C
:10DCA000F11D0B290FDAF01D0DE0032839D10120F9
:10DCB000F21F012A00DDF01F050608002D16F11CD9
:10DCC0000B2900DAF01C060636162AE0009822001E
:10DCD0004921F8F76FFA010028D04A78901C000615
:10DCE000000E84460020521E96460EE00B18DA788D
:10DCF000AA4207DBB24205DC7B78934202D00120C6
:10DD0000019004E0401C0006000E8645EED8009805
:10DD1000081A221A6046101A0406240E60460818D3
:10DD20000090002C02D001980028CFD0029820301B
:10DD3000807C80070BD5049800794007800F02D1C2
:10DD40000198012803D10398002109F067FA04988B
:10DD50000921007908420BD048206B461870012039
:10DD6000587000209870039803226946FFF7B8FBAB
:10DD7000012007B0F0BDFEB50500160048780C0084
:10DD800001270C36002818D001281CD002282FD1DA
:10DD9000A868C0042DD52879002808D1E0780009AA
:10DDA00005D15548002182680B002EF050FC22005E
:10DDB0003100280000F34DFB1BE022003100280059
:10DDC00000F0EAF815E02DF023FF01904848A17813
:10DDD000401E0278914207D10021017023003200D9
:10DDE00028000091FFF7A7FB01982DF015FF00E038
:10DDF00000273800FEBDF8B5002401263D49394F03
:10DE00003603451818206043C119385C0A000A32ED
:10DE100000280BD01088B04208D0091D0622280027
:10DE20002DF021FB002801D10120F8BD641C042C39
:10DE3000E8D30020F8BDFEB504000D0040790228AB
:10DE40000DD120000BF0E0F9002808D0112040018E
:10DE50002018418A0122200008F009FAFEBD18218D
:10DE60006943204802AA0D1868892F000D370190D8
:10DE7000781E00900821200006F0EBFA0600EDD095
:10DE800002980421006F01700021417020300421AC
:10DE900004000DF300E92078042108432070607825
:10DEA00001076878090F000101436170E078A178EB
:10DEB0000002084301990007000F09010843A07000
:10DEC000000AE0700D49300003F02EFC0028C5D098
:10DED0003878401C3870009801210170FEBD0000A8
:10DEE0009CCB00043CCB000424FD02C074FA02C0A9
:10DEF00031B701C029020000B82C00040210000054
:10DF0000F8B505002DF084FE434E070000241820CC
:10DF1000604381190A00305C0C32931E002814D033
:10DF20001078002811D118880122120390420CD0D9
:10DF30003A48091D062228182DF095FA002804D128
:10DF40002106090E2800FFF776FF641C042CDED39F
:10DF500038002DF061FEF8BD10B504005F21095DA9
:10DF60000020C90717D06079022805D1C304EB82CD
:10DF70000100000024DB000000040000C8484E310E
:10DF8000200032F063FC403080780CE006F0EAF8C4
:10DF90000F21890161180128086902D12030807F92
:10DFA00001E02030007FC007C00F10BD7CB5040029
:10DFB0000E00806815004006C00F0FD02EF00EFF37
:10DFC000002807D00F208001201800694030007F12
:10DFD000C00703D100F053FD00280ED0320020000E
:10DFE00001A9FFF769FA0198002805D0290000F37C
:10DFF000D9F9019806F0AAFA7CBD207900280ED143
:10E00000E8788006000F0AD1E8796B461870287A04
:10E0100058700848009A230000212EF022FB2200AD
:10E020002900300000F3DBF97CBD00003CCB00048C
:10E0300029020000B82C000410B5FF4C606B0028CA
:10E0400005D135F08EEA002801D001206063606BB5
:10E0500010BD10B535F088EAF7490020486310BDBF
:10E0600030B50020F54D0D21040003008901691829
:10E0700014E0E868401CE8601000526B8A62002AD5
:10E0800000D1CB620279052A0BD12A69521C2A6180
:10E090008362036003710020002C02D18A6A002A87
:10E0A000E7D130BD10B50A68E44B002A03D11868E7
:10E0B000401C186010BD8A6A824203D05868401C18
:10E0C000586010BDDC480024026A002A0FD08A4242
:10E0D00010D09A68521C9A6004220A71C26A002AFF
:10E0E00001D0516300E08162C1624C6310BD012226
:10E0F00001620A71006A07228462D14840210068E7
:10E100002EF0DDFE10BD10B50A68002A10D0CA4AF4
:10E11000936B83420CD1106A002809D0884207D142
:10E1200000209063C6480722006880212EF0C7FEB9
:10E1300010BDF0B5050085B000F0AEFC002000F089
:10E14000B9FC04007ED0286BBB4F2063786A401C6A
:10E150007862206000F0A8FC01F36FF902900020C3
:10E160000391019020682E0000212036002802D162
:10E170000120786220600023270020372371787BFC
:10E18000EF2108407873307A6071A079717A800845
:10E1900089078000890F0843F321A0710840B17AF4
:10E1A0008907090F0843CF21A0710840F17A890738
:10E1B000890E0843A07169692869594008430DD048
:10E1C0002A6902986B690399121A8B410AD3029A41
:10E1D0002869039B6969801A994102E0A8690028AF
:10E1E00000D0019001A80DC8002180185941E160BC
:10E1F000A060E8692061286A6061686AA061286897
:10E20000E06168682062A8686062787B317B4008C2
:10E2100089074000C90F0843FD2178730840317B0E
:10E220004907C90F49000843FB2178730840317B37
:10E23000C906C90F89000843F72178730840317B6C
:10E24000890600E01DE0C90FC90008437873022069
:10E25000B873307B000701D50620B873317B0120ED
:10E26000C90700D102203873BA7B23000092754899
:10E27000019A28332100F7F7C5FF002806D1206056
:10E2800001E000F011FC002005B0F0BD2068FBE7C4
:10E29000F8B505250E0000F00DFC04006648016A83
:10E2A000A14216D1A06A002803D0FBF2BCFE0020D8
:10E2B000A062002E66610CD000222300009261480B
:10E2C000283332002100F7F79DFF0325002800D1F5
:10E2D00004252800F8BD70B5052500F0EBFB04000F
:10E2E0005548016AA14207D1A06A002804D0FBF278
:10E2F0009AFE00200325A062280070BDF8B50F002B
:10E30000052600F0D7FB4C4C0500216A814215D14F
:10E31000A06B002803D0FBF286FE0020A063002F34
:10E320000CD0454B00220092474838333A00290070
:10E33000F7F768FF0326002800D104263000F8BD57
:10E3400070B5052500F0B6FB3B4C216A814207D130
:10E35000A06B002803D0FBF266FE0020A06303251B
:10E36000280070BD38B50120FDF7BAFC324C2C20D6
:10E37000236AC15C5A6A1868DB699847AAB9745362
:10E380000100000020DF0000000400009B929D5D62
:10E39000206A006B04F02DFB00F088FB2DF04CFC94
:10E3A000216A05000020086000F088FBFFF762FE8C
:10E3B000206228002DF044FC216A002909D02E207B
:10E3C000425C0B000092264A23482833F7F724FFCB
:10E3D00003E0FFF748FE15F087FF032038BDF8B5CE
:10E3E00005002048194F006A002813D0386A046BD2
:10E3F000200014F084FB182D06D1022804D01949FE
:10E4000020310979814204D12A000021200006F040
:10E41000FBF8F8BD072032F033FA4DE0386A006BA4
:10E42000B04204D030001FF0EBFE002840D12C0099
:10E43000162D1FD130001FF0C8FE002833D0707990
:10E44000022830D1386A2030407B0DE06836000465
:10E45000283300047C05000449DC0000ABDC00002C
:10E46000A086010010420004400701D52A241AE0CA
:10E47000282418E0192D03D01A2D01D0182D12D1FF
:10E480000F20800130180069817B002901D02C24E5
:10E4900009E0C07B002801D0292404E0386A006B21
:10E4A000B04200D0182422000021300006F0ACF861
:10E4B0000721300011F052FF0600AFD1F8BDFEB5C4
:10E4C00005250F0000F000FB040073D0A06A0026B1
:10E4D000002802D0FBF2B1FDA662FC4D286AA042E2
:10E4E00073D100F0E3FA2DF0A7FB01902079022808
:10E4F00001D0012810D12034607B102108436073C3
:10E5000000F0DCFAF2480722006840212EF0E1FC1E
:10E5100001982DF095FB53E001982DF091FB2079A7
:10E5200003281ED1267100F0C9FA286A2030072F6F
:10E53000077308D0082F0BD11A20FFF750FF39209E
:10E540000EF072FE42E01920FFF749FF3820F7E78E
:10E55000286A006B1FF082F81820FFF740FF372071
:10E56000EEE704282ED100F0A9FAE369626A206878
:10E570000B219847286A006B04F03BFA00F096FAEA
:10E580002DF05AFB26600700267100F097FAFFF77E
:10E5900071FD286238002DF053FB296A00290BD049
:10E5A0002E20425C0B000092CA4ACB482833F7F772
:10E5B00033FE05E00BE008E0FFF755FD15F094FE93
:10E5C0000320FEBD00F07AFA00E026600325280053
:10E5D000FEBD70B5040004252DF02EFB0600BB48DF
:10E5E000006AA04219D0217920680325042906D1A8
:10E5F00005212171E369626A0B2198470DE0A06A49
:10E60000FBF21BFD012808D1E369626A20680B2137
:10E6100098470021A1622160217130002DF010FB8C
:10E62000280070BD70B50500042400F03FFA2800F2
:10E6300000F04AFA002802D0FFF7CBFF040000F0F8
:10E640003DFA200070BDF8B505000E0000F02EFA6E
:10E65000A24F002438206043C019816900290ED0E0
:10E66000002D03D04521095C890705D4002E06D072
:10E670004521095CC90702D01830FFF7AAFF641CC6
:10E680000F2CE7D300F01AFAF8BD01210020DAE7D9
:10E6900010B51EF0DCFD002801D1012010BD0020C6
:10E6A00010BD38B51EF099FE1620FFF798FE152014
:10E6B000FFF795FE854C206A4179002906D08179C3
:10E6C0000091417900980022FFF7E2FF216A0320C0
:10E6D0000871206A02002030417BCB0608D5EF226A
:10E6E00011404173206A06210068FFF7E8FE1FE031
:10E6F0009069002808D000F3AAFE256AAA68EB6892
:10E70000801A9941A9690860216ACB694A6A086838
:10E7100003219847216A4869002809D08A6A002A9B
:10E7200006D100920B0002006B482833F7F774FD06
:10E73000032038BDF1B582B0694E644D30680028C1
:10E740002BD12C6A27002037787B0107CA0F009253
:10E750004007C30F6179206BA21D15F093FD1EF0D9
:10E760002DFEE369397B626A20689847022829D028
:10E770000298002805D01620FFF731FE01203060F6
:10E7800005E01720FFF72BFE36200EF0FDE3BB5E01
:10E79000010000001CE3000000040000B30318E0C7
:10E7A0004DFD296A02200871306800281BD0286AB4
:10E7B0002030407B400711D5042013F0A6F9002833
:10E7C0000CD111F01CFE040011F026FE844205D08D
:10E7D0004948006A002801D10220FEBD00203060B7
:10E7E00035200EF02BFD0320FEBDF7B586B00400EA
:10E7F0001600002513002F0003AA04A905A830F075
:10E80000E5F9059B002B14D06069002802D130681F
:10E8100001256061039A079901920091220000216D
:10E820001E0004980B00B0470700002D01D0002007
:10E830006061380009B0F0BD70B586B006000025F3
:10E8400003AA04A905A802AB30F0C0F9059C002C6E
:10E8500009D0039A002101920A0000913100049826
:10E860000023A0470500280006B070BD1C482030DA
:10E87000017F491C01771A49096A00290AD00A79DF
:10E88000032A07D1427F521C4277CB694A6A086843
:10E89000092118477047124810B5006A00280BD0AC
:10E8A0002030017B032907D1012101730D48072284
:10E8B000006840212EF017FB10BD70B50420084CF5
:10E8C000236A002B33D02C21C95C18680325012949
:10E8D00018D1FFF7C5FB00281FD0012019E0000068
:10E8E000683600047C050004A086010049DC0000B5
:10E8F000283300040003000410420004206A203082
:10E90000057313E0022913D1FFF7AAFB002804D0F6
:10E910000020FFF719FF0328F0D00120F7F780FA55
:10E9200078480722006840212EF0DDFA032070BDF0
:10E9300003290ED1186B0F218901401800690221AB
:10E9400003F0D6FF206A042120300173FFF7B3FEE5
:10E95000ECE7062901D1062006E0072907D10021AE
:10E960000120FFF77AFE0720FFF710FDDEE70829F8
:10E9700001D10820F8E75A6ADB699847D6E762496F
:10E980000420096A002907D00A79032A04D1CB6937
:10E990004A6A0868052118477047052801D20028EF
:10E9A00001D100207047594AC000801806C906C02E
:10E9B00001207047F3B587B00225079842780378A5
:10E9C00010021843012836D1079F891EBF1C30E072
:10E9D000F8780E1FB97800023C000843B0422ADCE8
:10E9E0006078217800020843FF3864381AD1201D6E
:10E9F0000CF3EAEB401E0090200008300CF3E4EB2F
:10EA00007D23DB005843019020000C300CF3DCEB3D
:10EA10007D23DB0058430290009801A90006000EF8
:10EA2000FFF7BBFFE078A17800020843311A3F1DD1
:10EA3000C7190429CCD2FF2064306B4698810C2082
:10EA4000D881079FBF1C01243048E1000E18601CCC
:10EA50007D2104903068C9000CF3C4EF7D2105903E
:10EA60007068C9000CF3BEEF06901022380003A9AD
:10EA70000CF368EA10371035641C052CE4DB280021
:10EA8000D8E62148006A002800D0012070471E48BF
:10EA9000006A002800D0012070471B48006A002847
:10EAA00000D0006B70471A480068002806D016494D
:10EAB000096A0968814201D101207047002070472E
:10EAC0001148002110B5006BC9432EF010FA10BD9B
:10EAD0000D4810B5006B2EF011FA10BD30B50400D2
:10EAE0000C4D0020010038224A4352199369A34279
:10EAF00001D110001830491C002801D10F29F2D390
:10EB000030BD00007C0500046836000404030004E6
:10EB1000640E00042833000410B5002420290FD00F
:10EB200065290BD108480DF327F8002805D10648C0
:10EB300014300DF321F8002800D00124200010BD6E
:10EB400002488260FAE7000028D000042C03000489
:10EB5000FA48C068012800D00020704710B50400B2
:10EB600003280CD8112017F09CFFCF210840210169
:10EB7000103901430906090E112017F0A8FF10BD36
:10EB800070B504000D001600F6F77AFD2000FFF7BF
:10EB9000E5FF3100280017F09AFF01203F7E813801
:10EBA0000100000018E7000000040000E0D9CB8C51
:10EBB000FFF7DEFFF6F7B5FD70BD70B504000D0080
:10EBC000F6F768FD2000FFF7D3FF280017F073FF6A
:10EBD00004000120FFF7CCFFF6F7A3FD200070BD75
:10EBE0000002FF30313070B500041407000C240F10
:10EBF000CA070FD0491E4910081805042D0C29001A
:10EC00000220FFF7DAFF0007000F210101430A0687
:10EC1000120E0BE04908081805042D0C29000220EB
:10EC2000FFF7CBFF00090001220002432900022068
:10EC3000FFF7B0FF70BD00024018FF301130010433
:10EC4000090C0220A6E70800110010B517F049FFD3
:10EC500010BD080010B517F02EFF10BD70B50C00E8
:10EC60001500080017F027FFA8430100200017F047
:10EC700038FF70BDF8B50120B5498860F6F70AFD88
:10EC800000252C022000FF309F300004000C0721DB
:10EC900017F060FFFF34A0342004000C042117F0AB
:10ECA00059FF2806000E070010222021FFF7D6FF8B
:10ECB00000242606360E002231003800FFF7BBFF85
:10ECC000002231003800FFF78BFF641C142CF0DBAE
:10ECD0006D1C012DD5DBF6F724FD02F042FEF8BDD8
:10ECE000F8B50025F6F7D6FC30272E023000FF30AD
:10ECF000B6300404240C200017F0DDFE3843010078
:10ED0000200017F0EEFE3000FF30BA300004000C97
:10ED1000FF2117F0E6FE3000FF30BB300004000C8E
:10ED2000002117F0DEFE300041300004000C042109
:10ED300017F005FF0024FF22210028001AF0F3FC41
:10ED40000022210028001AF003FD002221002800E3
:10ED5000FFF771FF002221002800FFF741FF641C2C
:10ED60002406240E142CE6D33000FF3017300004A4
:10ED7000000C402117F0E3FE3000FF30A030040407
:10ED8000240C8021200017F0DAFEFF369F36300475
:10ED9000000C022117F0D3FE0421200017F0CFFE53
:10EDA0006D1C2D062D0E012D9FD3F6F7BAFCF8BD74
:10EDB0006749002010B58860FFF792FF02F0DAFD86
:10EDC00010BDF3B581B000250E002C00012701987D
:10EDD00017F071FE3100814304D13800A040284370
:10EDE00005062D0E641C012CF1DB2800FEBD70B55C
:10EDF00005000E0000243100280017F072FE641C8C
:10EE0000012CF8DB70BD70B50C001500080017F080
:10EE100052FE28430100200017F063FE70BD70B55C
:10EE200005000E0000242006000E32002900FFF726
:10EE3000EAFF641C012CF6DB70BD70B505000E0006
:10EE400000242006000E32002900FFF707FF641C93
:10EE5000012CF6DB70BD012804D13E48405C3E49E0
:10EE6000400002E0491E48003C49085A704770B50E
:10EE70000028374B3A4C596018705A70237802D1E9
:10EE8000DF252B4003E0012802D120252B432370EE
:10EE900001F01AF8012070BD2D48406870472C48D9
:10EEA000007870472A484078704702000020002907
:10EEB00000B512D011000120FFF7CDFF2949012232
:10EEC000884209D9274902229631884204D9264925
:10EED0000322884200D90422100000BD23487D216E
:10EEE00010B5006849012CF0ACEB8905800A084395
:10EEF0001F4900E0401E0A68002A01DB0028F9DCF7
:10EF0000002803D112490869401C086110BD002087
:10EF100010B517F0D0FD0E4CA070012017F0CBFDFE
:10EF2000E07010BD08B5F6F7B5FBFFF7F0FF11482C
:10EF300017F0F5FDF6F7F5FB0020694604F024F91B
:10EF4000002819D16B461870587098701BE00000AB
:10EF50003C03000404480400C4EE3100A8EE310074
:10EF6000ECE800043214000044160000C0B601C0F2
:10EF7000002B0080307C01C06B461878012802D13C
:10EF8000FFF778FE03E000210800FFF711FFF6F716
:10EF900081FBF6F7C6FB1AF055FB08BD10B5FFF76D
:10EFA000C1FF01201AF0FEFD012010BDB618B264A9
:10EFB0000100000014EB00000004000014B6BE388D
:10EFC000FF48C0787047FE4880787047704700025D
:10EFD000FF3070B5BC3004040D00240CF6F764FB60
:10EFE0002900200017F087FDF6F7A5FB70BD000291
:10EFF000FF30BC3010B50404240CF6F755FB20009C
:10F0000017F063FD0400F6F796FB200010BDEC48F6
:10F0100010B542680078EB4B002808D151001A0067
:10F020000A32891820391888C98B081821E0110084
:10F030000120FFF71AFFE44C0221595EA04211D9CA
:10F04000E14C0421595E9634A0420BD9DF4C0621D5
:10F05000595EA04206D9DD4C00217D34A04201D882
:10F060000821595EDA48805CD64A40002632105AA0
:10F0700040180004001410BD0002FF3070B5E930E4
:10F0800005040A060C002D0C120E29000320FFF7C0
:10F090008BFD2004020E681C0104090C0320FFF7FD
:10F0A00083FD2002020EA81C0104090C0320FFF7B7
:10F0B0007BFDED1C2904220E090C0320FFF774FDD3
:10F0C00070BDF1B582B0F6F7EFFA0220FFF75AFDF6
:10F0D000002502990024680040180190200246197A
:10F0E0003000FF3091300004000C17F0EEFC870771
:10F0F000FF3671363004BF0F000C17F0E6FC8000BD
:10F10000620001993843641C012C8852E6DB6D1CB7
:10F11000132DDEDB0120FFF735FDF6F70CFBFEBDFE
:10F1200000024018FF3051300104090C022010B5D4
:10F13000FFF74DFD4006400E10BD10B51AF0CAFB9A
:10F1400010BD0002FF3041300004000CCA0710B5AA
:10F1500009D0491E491008180104090C0220FFF7C4
:10F1600036FD000910BD490808180104090C0220E9
:10F17000FFF72DFD0007000F10BD0002FF30801DBE
:10F1800070B505042D0C0024FF2229000220FFF792
:10F190000BFD6D1C641C2D0424062D0C240E022C6A
:10F1A000F2D370BDFF230A3370B5002A00D11B1FB4
:10F1B000CA08D2180002801804044D07240C6D0FF1
:10F1C00021000220FFF703FD0121A94001430A06A7
:10F1D000120E21000220FFF7E7FC70BD10B54C07AE
:10F1E000640FC9080002002A02D0FF310A3101E091
:10F1F000FF31891D40180104090C0220FFF7E7FCCC
:10F2000001210A00A240024200D00021080010BDE6
:10F2100001000120002900D00020704710B5012412
:10F220006420F6F79FF96B487D21006849012CF0B6
:10F2300012EA8905800A0843674900E0401E0A680F
:10F24000002A01DB0028F9DC5D49002805D1486966
:10F25000012200241204801801E04869401C486122
:10F26000200010BD0100012010B5FFF7FEFD564A39
:10F270000021AA3A904217D9534A0121904213D94A
:10F28000514A0221963290420ED9504A0321CD3A7A
:10F29000904209D94D4A0421904205D94B4A052193
:10F2A000C832904200D9891F0804000C1823444931
:10F2B00058433431401817F03CFC10BDF7B58EB000
:10F2C0000E98002800D0012001900F9800250128F9
:10F2D0000BD00F984008012801D1012505E00F98B7
:10F2E00002258008012800D0ED1E019834498000D5
:10F2F0001C310D900858691C74D001990C23304AB8
:10F300005943C4328B18AA000B920C919C582C4B79
:10F31000DC33CB189B580393294BF433C918895815
:10F32000029117F006FC200017F003FC0024F6F70A
:10F33000BBF9E8000A9018206043284926024018CB
:10F340000A990700405801063000FF3031300004B0
:10F35000000C090E099017F0CEFB0A997818406846
:10F3600001063000FF3030300004000C090E089018
:10F3700017F0C1FB022D3AD1FFF7FEFB002836D073
:10F3800017482701C05901060998090E17F0B3FB69
:10F3900013483F18786801063000FF30333000040E
:10F3A000090E000C17F0A7FBB86801060898090EB3
:10F3B00017F0A1FBF868FF360106090E9071E465AD
:10F3C0000100000010EF000000040000476C6D54C5
:10F3D000323612E03C030004A83600043214000068
:10F3E0004416000004480400C0B601C0002B008091
:10F3F000440C00041C540004B1E03004000C17F06D
:10F4000084FB641C2406240E012C9ED3F6F79DF980
:10F410000320FFF7C1FB019801281DD1022D1BD14C
:10F42000A74E0024A00081198978305A17F06DFB8F
:10F43000641C142CF6DBFF20FF21ED3017F065FB78
:10F44000FF20FF21EE3017F060FBFF20FF21EF309F
:10F4500017F05BFBFF213BE00EA807C819F091F8FD
:10F4600006000006000E6B46187007903004000E70
:10F47000587006903002000E98700590300E0024EF
:10F48000D870012704903800A040304205D003997D
:10F49000A00041188978039A04E00299A00041185D
:10F4A0008978029A105A17F030FB641C142CEADB9E
:10F4B000FF200799ED3017F028FBFF200699EE306A
:10F4C00017F023FBFF200599EF3017F01EFB04997E
:10F4D000FF20F03017F019FB03F0E5FA00283BD0CD
:10F4E00078490D98774A08580C99E8328A180B9990
:10F4F0005658754A0C998A180B99575817F023FBE0
:10F500000320FFF749FB019801280DD1022D0BD1F3
:10F510006E4D0024A00041198978285A17F0F5FA99
:10F52000641C142CF6DB17E00EA807C819F029F8A4
:10F53000050000240120A040284204D0A000811929
:10F540008978305A03E0A000C1198978385A17F039
:10F55000DCFA641C142CEDDB0120FFF71DFB11B05D
:10F56000F0BDF7B584B00498002801D0012200E076
:10F5700000220026012909D04808012801D10126CE
:10F5800004E002268808012800D0F61E4D499000AC
:10F5900008310858711C01D1002406E00C215143A8
:10F5A000494A18328918B2008C5817F0CCFA20005A
:10F5B00017F0C9FAF6F782F80024F000039018203B
:10F5C000604343492502471803983858010628002C
:10F5D000FF3031300004000C090E029017F095FA4C
:10F5E00003983818406801062800FF3030300004C6
:10F5F000000C090E019017F088FA022E26D1FFF7B1
:10F60000C5FA002822D033482701C05901060298C4
:10F61000090E17F07AFA2F483F187868010628007B
:10F62000FF3033300004090E000C17F06EFAB86892
:10F6300001060198090E17F068FAF868FF3501060F
:10F6400032352804090E000C17F05FFA641C2406FA
:10F65000240E012CB3D3F6F778F80498012802D1D0
:10F660000698FFF709FE07B0F0BD002810B505D1D8
:10F670001948002900D1194817F065FA10BD10B5D6
:10F68000F6F738F916494000085A4004000C10BD3E
:10F6900070B504000D00FFF7F2FF03002900200001
:10F6A000FFF7EDFB0022190017F073FA70BD0D494A
:10F6B00008680222904308600B49002008607047E8
:10F6C000BC8801C06003000460040004D48F01C042
:10F6D000440C00041C540004E88201C0F88201C0FC
:10F6E00098360400002B0080E407000470B5FE4C3F
:10F6F00060680125ED05284369108843606001209A
:10F70000F5F73AFF60680321890508436060A84364
:10F71000606070BD10B50400F4480068002801D195
:10F7200000240CE00021012016F012FCF049A0009A
:10F73000401800680406240E012016F02BFC20005F
:10F7400010BD70B5040018D00021012016F000FC97
:10F75000E848E74BE849026806E0012A03D1800047
:10F76000A578C0180560241D20888842F5D1A578A9
:10F77000FF2DF2D1012016F00DFC70BDDF480122F3
:10F7800010B5052142700170DD4801681306194368
:10F790000160DC480168114301602CF075FA040037
:10F7A000D948FFF7CEFFD948FFF7B4FFD349891FE7
:10F7B000C87020002CF06CFA012010BD70B52CF040
:10F7C00063FA05000020FFF7A5FFCC4C3B5BE05B34
:10F7D000010000000CF3000000040000F8A948E755
:10F7E000A41F207128002CF05DFA207970BD70B53F
:10F7F0002CF054FA05000120FFF796FFC44CA41F1B
:10F80000607128002CF04EFA607970BD00207047BE
:10F81000BF49891F487070474042022900D9022120
:10F82000BB4A89003E328918BE4A1268012A01D1BA
:10F830008A5601E000228A5601231018B44A921F0A
:10F84000D35602228A56C018824203DB03228A560C
:10F85000824200DD1000000600167047B14910B565
:10F860000A68AB494042891C012A01D18A5601E04D
:10F8700000228A56A64C0223CB56A41C03216156B3
:10F880001018834201DA180002E0814200DD08000E
:10F890009F4B03249B1F1C57121B8A4200DC0A004B
:10F8A000000600169A7010BD99490278891C0A70EA
:10F8B00002794A7082783C310A7082794A704278C3
:10F8C0000A7142794A71C2780A72C07948727047E7
:10F8D0008F4B04219B1CC9431A0019703C3259708C
:10F8E000117051701171517111725172704700286D
:10F8F00001DD002004E06421C943884200DA0800E9
:10F9000040420006001670470020704770B50500A1
:10F910007D480C00006800280AD00021012016F064
:10F9200021FB7849A80040180460012016F03CFB38
:10F9300070BDF7B588B00400002002902CF0AEF93D
:10F94000039000252004000C07900998002824D17A
:10F9500000242806000E069002AA01920094069B3D
:10F960000A9A0799099833F040EE00280FD06848AA
:10F9700029014A300E18A7006B46F05B597AFFF751
:10F98000C5FFF0196B464088197AFFF7BFFF641C6A
:10F990002406240E042CDFD344E00998012841D129
:10F9A00000242806000E059002AA00940192059BEF
:10F9B0000A9A0799099833F018EE00282DD0012CE7
:10F9C0001AD118215248694300265A300F18A0193D
:10F9D000800004906B46385A597AFFF797FF0498D5
:10F9E0006B4638184088197AFFF790FF761C360668
:10F9F000360E052EEBD310E01821454869435A30E6
:10FA00000E18A7006B46F05B597AFFF77FFFF019DD
:10FA10006B464088197AFFF779FF641C2406240E90
:10FA2000022CC1D36D1C012D8FDB03982CF03AF909
:10FA30000BB0F0BDF7B584B005002CF02FF907002E
:10FA400000242804000C039002AA00922306069AC0
:10FA5000039905981B0E33F0CCED00280DD02C4EE9
:10FA6000A500B61D6B46597A705BFFF74FFFA819CA
:10FA70006B46197A4088FFF749FF641C012CE3DBD1
:10FA800038002CF00FF907B0F0BDF7B584B00500D1
:10FA90002CF004F9070000242804000C039002AAAB
:10FAA00000922306069A039905981B0E33F0A4EDE5
:10FAB00000280DD0164EA5000A366B46597A705BA9
:10FAC000FFF724FFA8196B46197A4088FFF71EFF3D
:10FAD000641C012CE3DB38002CF0E4F8D3E73EB5DE
:10FAE0006B460C0019705870009801A903F080FB58
:10FAF000002819D001A8FFF7D7FE3EBD00280080DE
:10FB000028F900040020009024F90004FFFF000001
:10FB10009604000480210080002D00802044040011
:10FB2000CB020000F81700042000FFF7D1FEE4E745
:10FB3000002800B511D1022A05D1092901D8481C95
:10FB400000BD082000BD032A05D1052901D3C81E28
:10FB500000BD022000BD481E00BD022A01D0032ABC
:10FB600045D174293DD011DC8807800F3DD18B1021
:10FB7000093B0BF32CEC142C2C2E2E3A3A30303A55
:10FB80003A3A3A3A3A3A3A323234343A8C292AD02A
:10FB90000EDC802904D005DC782922D07C2924D1F0
:10FBA0007E2000BD842901D088291ED1862000BD79
:10FBB000992904D005DC902915D0952915D19720D5
:10FBC00000BD9D2901D0A1290FD19F2000BD262075
:10FBD00000BD2E2000BD3E2000BD66200A12422A34
:10FBE0000100000008F7000000040000AB739B8BCD
:10FBF00000BD6E2000BD762000BD8E2000BD3620E9
:10FC000000BD900801283BD174291CD011DC880765
:10FC1000800F33D18B10093B0BF3E2EB142A2A2A15
:10FC20002A3030303030303030303030302C2C2CE6
:10FC30002C308C2920D00DDC802904D005DC7829DB
:10FC400001D07C291AD17A2000BD842914D08829BA
:10FC500014D111E0992909D004DC90290CD0952900
:10FC60000CD103E09D2901D0A12907D19B2000BD23
:10FC70002A2000BD6A2000BD8A2000BD3A2000BDB8
:10FC8000080000BD10B50400FFF75CFF002C00D198
:10FC9000401C0006000E10BD417803780A021A438A
:10FCA00001D0012A06D1C17A837A0902194303D00F
:10FCB000012901D001207047FF490A70C27883787A
:10FCC000120612141A434A704279037912021A4337
:10FCD0004A80C279837912021A438A80427A037A6F
:10FCE00012021A43CA80C27A837A12021A430A7233
:10FCF000427B037B120612141A434A72C27B837B37
:10FD000012021A434A81427C037C12021A438A81FE
:10FD1000C27C837C10021843C881012088770020B0
:10FD2000704770B50500E5480C00006800280ED04B
:10FD30000021012016F020F9E149A80040180168CF
:10FD40000906090EA1430160012016F037F970BDC4
:10FD500070B50500D9480C00006800280ED00021BD
:10FD6000012016F009F9D649A800401801680906D3
:10FD7000090E21430160012016F020F970BD38B54D
:10FD80000024CD4D2A69824225D100202B0010335A
:10FD90000129286104D100220092AA69002106E00D
:10FDA000002907D1002200926A6901242100C54878
:10FDB000F6F76EFA2BF07CFF0500002C04D004212E
:10FDC0007020FFF7C5FF03E004217020FFF7A9FFB3
:10FDD00028002BF071FF38BDF8B50400B64DA87FA0
:10FDE000002820D02BF064FF29690600080003D00A
:10FDF000FAF25FF90020286130002BF05DFFEF88F8
:10FE0000002C00D0EF892FF0ADFFF907C90F084390
:10FE10000AD12BF04DFF040004217020FFF781FF71
:10FE200020002BF049FFF8BD2BF042FF0090287F07
:10FE3000FF2803D15F20FFF781FC2877687FFF2828
:10FE400003D16020FFF77AFC687728782900002C1E
:10FE500000D0087A01268E570500002C01D0092613
:10FE60008E578888002C00D088897D23DB0058437A
:10FE700088614888002C00D048897D23DB005843E6
:10FE80000C000028486101D1002506E0012D04D1B5
:10FE900004217020FFF75CFF03E004217020FFF7CE
:10FEA00040FF207F80190106090E5F20FFF738FD13
:10FEB000607F80190106090E6020FFF731FD009870
:10FEC0002BF0FAFE2FF04EFFFF21491C0F40384364
:10FED000A9D0002DA7D0A0690028A4D0764B00227D
:10FEE00000927848626910330121F6F7D1F9F8BD24
:10FEF00070B504002BF0DCFE0500002C04D00421BA
:10FF00007020FFF725FF03E004217020FFF709FFB1
:10FF100028002BF0D1FE70BDF0B506000C006A4839
:10FF20001500816A85B0694A11408162416A684A58
:10FF3000114341622BF0BCFE01901AF03BFC029091
:10FF400080210220FFF704FF0120F5F729FB802123
:10FF50000220FFF7E6FE0120F5F722FB210030002A
:10FF600033F058EB5B48FFF700FC2206120E290025
:10FF7000300003921AF084FA002E17D1022D05D01A
:10FF8000032D03D00E2C01D1534F06E002F044FEA6
:10FF9000012801D1514F00E0514F2BF089FE009014
:10FFA0003800FFF7E2FB00982BF086FE1AF0BAFA51
:10FFB0004C48052C01D00D2C03D1012D01D19A21E3
:10FFC00006E0092C01D00D2C04D1022D02D1BA215A
:10FFD000FFF7A6FC6808012803D143488021FFF7FA
:10FFE000A0FE012D07D14248404901600554A88078
:10FFF0000100000004FB0000000400005F1CEE3F55
:020000021000EC
:10000000416049008160C16001E01AF087F9300069
:10001000FFF7ECFE02981AF0EDFB2A0031002000F9
:10002000FFF747FD2A0031002000FFF717FD2A00E7
:1000300031002000FFF791FC2A0031002000FFF77B
:1000400062FD01982BF042FE2448416A254AD243C2
:1000500011404162F5F750FB220029003000FFF704
:100060009EFAF5F790FB300016F0D7F9F5F744FB50
:10007000300016F041F80700010030001AF06CFA69
:1000800039003000FFF70FFB0221072016F094FD26
:1000900033F0CEEA002F04D01021072016F08CFD9B
:1000A00003E01021072016F07CFD03992A003000A0
:1000B000FFF7F2FD01003000FFF708FB22002900E6
:1000C0003000FFF723F9FFF7D1F81DE0B404000476
:1000D00024F900040020009097F8000000A8008098
:1000E000FCFBFFFFC0000080204404000C4904001A
:1000F00004490400084904005E0200000D040000E9
:100100000101010140B0008033F096EABE4D002F9E
:100110001FD0BE480068002817DB072016F0FDFC42
:100120008009012803D1A869401CA8610AE00228BF
:1001300003D1E869401CE86104E0032802D1286A81
:10014000401C28626869401C68610221072016F083
:1001500028FDF5F718FBAE48026A032189028A439D
:100160000262016A002E01D1020D01E00122920219
:1001700011430162016A0122520211430162A54F3B
:10018000002E01D1A44800E0A44838612878B0428C
:1001900013D030002E7016F06EF8300001F00FFC16
:1001A000300001F022FC012803D12100300001F0D1
:1001B00038FC2100300001F045FC38690821084373
:1001C0003861012005B0F0BD8F49FF2008707047ED
:1001D000F7B580010C00050C8B4A002108325056FF
:1001E000002800DC41420806000E1F261F2800D20E
:1001F00006002BF067FD0700202C05D0402C05D011
:10020000802C05D0002404E0102402E0202400E02B
:1002100030242906090ECD20FFF78CFB290ACE20B9
:10022000FFF788FBD220FFF793FA410902984901B2
:100230003143002802D14020014301E0BF200140AA
:10024000D220FFF777FB210080200143CC20FFF76D
:1002500071FB38002BF03AFDFEBDF3B58FB02BF0EB
:1002600031FD0090D220FFF773FA4021084203D0FD
:100270006B480926019003E0694809300B2601907C
:100280000F9831000AF360EF00252C0003950295CA
:1002900028E0CC20FFF75CFA000900014006400E80
:1002A00020430106090ECC20FFF744FBD120FFF7C5
:1002B0004FFA0004A70004A9C851D020FFF748FA5C
:1002C00004A9C9590002084304A9C851CF20FFF767
:1002D0003FFA04A9C959084304A9C8510399401811
:1002E000641C0390B442D4DB00982BF0EFFC03981D
:1002F00000281AD0002404AF14E0A00038580102EE
:10030000081A03990BF3AAEB0F990006000E085583
:1003100041190D0601992D0E0957414302980818FD
:10032000641C0290B442E8DB09E00F9AFF21701EC2
:100330000D001154019908560302181A02900F98E3
:100340000178FF20401B0A180F990A70019A0021BA
:1003500051564143029808181099002902D010996B
:1003600000120880300011B0F0BD70B504002BF011
:10037000A9FC05002B48002C03D08021FFF7DBFCF3
:1003800002E08021FFF7EEFC28002BF09FFC70BDFF
:10039000F7B582B004000E002BF094FC102C0190F5
:1003A00001D900200EE71F4DFF21113D6019070004
:1003B000FFF7C1FC3106090E3800FFF7D3FC102C03
:1003C00002D11120002403E0A0081230A1074C0F35
:1003D0000321A14009064019090E0500FFF7ABFCF7
:1003E000F005C00FA0400106090E2800FFF7BAFC77
:1003F0000498A0404006010E2800FFF7234AE48736
:100400000100000000FF0000000400000CC63D5386
:10041000B3FC01982BF064FC0120DDE6900400049D
:10042000002B008000280080C0A2008008A80000E7
:1004300008680000583704009305000070B5F84DB7
:100440006969F8484165F84909688165F7480024F9
:100450008461F4F731F91020F4F706F9E80CF4F7A9
:1004600003F92C6070BD10B5EE4C0200616B206B7F
:100470000AF3C6EF7D22D2000AF3C2EFE36AA26A52
:100480000AF384EB10BDF8B57D220700E54CD200DD
:10049000616B206B0AF3B4EF05000E00E16AA06AFD
:1004A0003A000AF3AEEF33002A000AF370EBF8BD0E
:1004B00010B5DC4C0200616B206B0AF3A2EF7D22C9
:1004C000D2040AF39EEFE36AA26A0AF360EB10BD5E
:1004D00010B50400F2F77EFB21002BF0EEE8D44AC1
:1004E00000230AF354EB10BD70B50400CD4D01207C
:1004F0006872D0480168420C11430160F5F722FA96
:10050000CD494000085A64235843A8616043F4F77A
:1005100088F870BD10B50124F4F778F8200010BDFC
:10052000C0480079704770B5F4F785F80600F4F715
:1005300091F8BC4C002526636563A169E5624143DF
:10054000BC48A1620168420C9143016020790028F7
:1005500004D10120FFF7ACFFF4F771F8657270BDAC
:1005600070B5B04C2069FFF77EFF61890BF380EA1C
:10057000E0610500B148A1690BF37AEA0100A842E5
:1005800001D8E06901E00800E1617D21C9000BF3B9
:1005900070EA206270BD0A2010B5FFF7A5FFFFF7D3
:1005A000B9FF040010D0FFF7BEFFFFF7D9FF9D4849
:1005B000016A08000A2907D9FFF796FFF4F726F821
:1005C000FFF7B1FFFFF7CCFF200010BD70B50400AE
:1005D000944D0120687297480168420C11430160F4
:1005E000F5F7B0F994494000085A64214143002CC2
:1005F000A96102D00800604305E0E86948437D2115
:10060000C9000BF336EAF4F70CF870BD85490A6AA5
:10061000824206D84A7A002A03D14979002900D1BA
:10062000D4E77047F3B583B000277E490D006B6BAC
:100630002A6B39000AF3D8EF02900C00E96AA86A25
:10064000049A0AF3DEEE05000E0006220AF3D8EE45
:100650003B0005220AF39AEA0191AA0FB100114367
:100660000090A8003B0005220AF390EA029A2300BA
:10067000121A8B411AD3684607C8801AA14115D3B4
:100680000722310028000AF3BCEE029A801861416B
:10069000644C4A07C0081043636B226BC9080AF315
:1006A00076EAE162A06204986763206305B0F0BD5A
:1006B00070B55C4C6079002811D1F3F7A7FFF3F710
:1006C000BAFF0500F3F7C6FF5A4A01001068530C41
:1006D00098431060A06948432900FFF7A3FF2079E1
:1006E000002804D10120FFF7E3FEF3F7A8FF002064
:1006F000607270BD70B5FF244A4D5A342B68C31A1E
:100700001B1BFF3BFF3B1B1F002B04DC4C49C86A33
:10071000401CC86203E0814201D8824201D200201D
:1007200070BD1800FFF7AFFE06002000FFF7D0FEF7
:1007300004002868FFF7A7FE82192300002130007B
:10074000F4F708F82879002806D12868FFF79BFEFF
:100750000004000CF3F752FF012070BDF8B505004E
:100760006846F5F7B2FB374800990068814201D02E
:10077000F5F790FB344800990068814201D0F5F705
:1007800089FB324C324E2078FF280AD10CF0BDFC98
:10079000002806D0002D04D0306822000D21F5F786
:1007A0008BFB00993068814201D0F5F773FB294833
:1007B00000990068814201D0F5F76CFBF8BD214833
:1007C00038B50068F5F76CFB1F480068F5F768FB63
:1007D0001F4D2868F5F764FB1E480068F5F760FBBD
:1007E0001A4C2178FF2905D028686A46F5F764FB82
:1007F000FF20207038BD70B52BF06EFA104C05004C
:100800006068002805D12FF0C2FB012080E0E9726A
:1008100001000000FC020100000400000E903B7A81
:100820006060002001E0606B401C606328002BF0DA
:1008300061FA70BD00A50080583700048022008056
:1008400040A6008040420F0000210080983604003E
:10085000002D31010C050004A0020004080800046A
:100860004CE9000478050004DC06000410B5FF4CD8
:100870006068002803D02FF0A8FB0020606010BD46
:1008800010B5FAF72DFA04000DF011F8204310BD51
:10089000F74810B50078C00705D0F4F741FFFEF720
:1008A00063FBF4F784FF10BDF8B52BF01FFA0400CA
:1008B0000021012015F07EFBF3F739FEED49086BAE
:1008C000CA0C90430863012015F096FB20002BF022
:1008D00011FA15F0DBFDE54E0025B560E6488168AC
:1008E000AA2211438160E248E44F0078E44CC0073B
:1008F00021D02BF0FBF9009020690B218843206167
:100900002069316908432061A561F3F7DFFEF3F741
:1009100064FFD948C038C760D948C0300168022296
:1009200011430160D7490868082210430860009805
:100930002BF0E0F907E0A561F3F7C8FEF3F74DFFF0
:10094000CD48C038C760FEF20EFFCF48CF49406D9A
:10095000486120691021884320610CF0DBFB0028EE
:1009600000D0022030F026F804000DD0200010F056
:1009700080FE002801D0042100E005210F20800125
:100980002018006902F004F82BF0B0F90400FFF71A
:100990006DFF20002BF0AEF9FFF71BFFF9F207FC0B
:1009A000F8BDB74810B501690B2291430161016997
:1009B000AE4AD2681143016100218161F4F7B0FEB3
:1009C000FEF7D2FAF4F7F3FEAD48C0300168022218
:1009D00011430160AB48016808221143016010BD5A
:1009E000FFB583B004000027A94D0CF093FB00284D
:1009F00000D002202FF0DEFF060002D0B068C00455
:100A0000C00FFFF7B5FE2BF071F900220290A1484C
:100A1000009200680822012101AB2CF0A8FA01988D
:100A200000281BD19C48002200684A21F8F24DFFA3
:100A3000002802D00C98002810D09349974B086EDC
:100A4000496E3F221840520500231140594058403A
:100A5000084303D1F5F757FE00280AD18A488F4C86
:100A6000026E416E3F2322405B05194002664166DB
:100A700020E0002C2AD0FEF244FD00900498226869
:100A800063680F00101A00218B41009A19003B0087
:100A9000121A8B410AD2009A20686168801AB94103
:100AA000069A0599FFF730FE002806D16F48C16904
:100AB000491CC161FFF7F8FE11E1734862682168C3
:100AC00080304261016100F09EF907006D4A1068B4
:100AD0000821884310606A4AC032106802218843A6
:100AE000106067480169614A042319401161016976
:100AF00099430161016903221143016146E05B48AA
:100B0000816A491C6D1E81623DD10100486A401C0A
:100B100048620CF009FB002813D0594881698169AB
:100B200001690B2291430161564A11680823194358
:100B3000116001694D4A126911430161F9F237FBF5
:100B4000CDE04F4DA8698006800F012803D14748AA
:100B50004169491C4161FFF724FF0FF03FFB494900
:100B600008680822904308604549C031086802229D
:100B7000904308602869042188432861286903217B
:100B800008432861424D0120F4F728FD3C48806964
:100B90008006800F0328B2D101F051FA002804D159
:100BA0003249086A401C086295E0002C08D000F029
:100BB0002AF9069907008842F2D805988742EFD3B0
:100BC00032484169304A5165022141613448F3F7A6
:100BD0006DFCFEF2D0FD28488168090A0902816097
:100BE000274908691022104308612048007802282C
:100BF00001D1022500E04025002C02D000F003F9CD
:100C00000700002F01D001200543002E04D00F2043
:100C100080013018006900E0002001210352F44AED
:100C200001000000F8060100000400005D4AE8161B
:100C300001F0B8FEF4F780FFE807C00F01D0F3F72A
:100C400047FD1D4F422005403AD068060AD51020C6
:100C5000F3F718FD1020F3F727FD0420F3F7CEFD7E
:100C6000F3F7DEFDA8072BD53D003800F3F70AFDAA
:100C70002800F3F71FFD0C20F3F7C0FD1EE0000075
:100C80000C050004ECE800040021008040230080F3
:100C9000EFFFFFFF40A6008000A30080583700044C
:100CA00000A5008088130000E0BD01C00000000422
:100CB000180004001000100000100000F3F7B0FD51
:100CC0000320F3F79BFD5D4E0125B560002C16D087
:100CD00000F0A3F80699884202D8059988420ED2FE
:100CE000306A0121090440183062FFF7E7FDFFF781
:100CF000D9FD02982BF008F8002007B0F0BD15F0E0
:100D0000DDFBFFF7C7FD4E4900280D6000D001E074
:100D10004C48056002982AF0F7FF2AF0F1FF040022
:100D20000021012015F050F9F3F715FC4649086B36
:100D300038430863012015F069F920002AF0E4FF28
:100D4000F5F2F6FE4149884216D0414C606B022113
:100D5000884360633F48EFF751FCE2173E4800923A
:100D600000680822012101AB2CF00BF931200003AF
:100D7000EFF744FC394860630120BEE710B50CF082
:100D8000DDF9002803D02D488068002801D0FFF746
:100D900095FD10BDF8B5334A314811680826B143B6
:100DA0001160314B19680222914319602E4CC03CEE
:100DB0002169224D04273940E9602169B943216145
:100DC00021690B2211432161401E1BD1FFF7F3FD66
:100DD0000FF00EFA20693840E8602069B8432061BE
:100DE00020490868B04308601F4A10680221884300
:100DF0001060A0698006800F012802D1A869401CFC
:100E0000A8611748A1698906890F0329D8D1F8BDBF
:100E1000012070471548407A704710B5F3F7DBFCA6
:100E20000400F3F7A6FC201A05D50449086B401C02
:100E30000863002010BDFFF72AFB10BD0C0500045D
:100E4000600700046407000400210080A0B90004CA
:100E50000034008010100300E0BD01C0F201010069
:100E60008813000000A3008000A70080583700040A
:100E7000F8B50024FF484069FF4E8505AD0DB54229
:100E800003D001243000FBF74FF8FC4B00211F007A
:100E9000383788001A58126838580260491C0929E6
:100EA000F7D9002C03D03000A843FBF719F8F44B16
:100EB00000201C1FC100CA18126809190A60401CD2
:100EC0000828F7D30020F8BD13000A00803010B5C1
:100ED000C16D806DFEF28AFE10BD7CB514008030BD
:100EE000069A009301920A00C16D806D2300FEF204
:100EF00094FE7CBD38B51400049A00922200FEF2E4
:100F0000A3FE38BDDF4B10B5186259629862D962F2
:100F1000186359639863D963DA4B4033186059609A
:100F20009860D960186159619861D9611A62FEF2BE
:100F30003BF9D34900208C314860CE49C039486321
:100F400010BD70B50500D0480C004188A1421CD0EE
:100F5000448028002FF0F8FC10F077FE002814D110
:100F6000C549002C12D0022D01D11F2600E00F260A
:100F70000D00002431002000FEF285FA2900200037
:100F8000FEF28BFA641C032CF4DD70BD0F203F22AF
:100F9000FFF7B8FF70BD010000200E2908D2B54848
:100FA0004030072901D889000818006B0004000CA4
:100FB00070470E2806D2AF4A4032072803D8800077
:100FC00080180163704711637047F0B5002087B047
:100FD00010F0F5FD002804D1012010F0F0FD0028EC
:100FE00001D0012100E000210220059110F0E7FD71
:100FF0000490032010F0E3FDA84900914C140599DA
:10100000A24AA34BA34EA44F2500002903930292AA
:1010100001D015001C00049901431FD0022032F0BA
:101020002EEB002801D035403C400320EB081B0686
:1010300001000000F40A010000040000A9259DA29F
:1010400032F026EB002803D00298039905400C40AB
:10105000012032F01EEB002805D0009802990540CF
:1010600003980D4004400498002801D035403C40CE
:101070009048C562046307B0F0BD70B50600FFF28A
:101080009DF98D4C250C002E08D08349002040315D
:101090000862FFF7A4FFE068284316E011F0ADFBFB
:1010A000002810D003210020FEF21DFB7648C0303E
:1010B00001680122D2069143016001680E224908AD
:1010C000490011430160E068A843E06070BD6E49CB
:1010D00001235B04C0395A000028886904D01843F2
:1010E00088618869904303E0104388618869984368
:1010F000886170476948006B7047684910B5040003
:10110000FC31FFF247FD6D4A200011001031FFF263
:101110008EFD10BD614810B5A030FFF2A9FC6749F3
:10112000543908000930FFF2D1FC10BD5B4810B5FE
:101130007830FFF250FC5949604834317438FFF27E
:1011400077FC10BD5E49082010B508705D490A2083
:1011500008705D49012008705C49102008705C49E6
:101160001E20087019F002F919F0FAF8FFF7DEFFF7
:10117000FFF7D0FF4948006B0006000EFFF7BDFFE8
:1011800010BD10B5FFF7DEFF002019F0BFF810BD4D
:10119000F8B522206B461870322058703F4CFF2063
:1011A00098702161A0690E001500002804D101206B
:1011B000A061F4F741FA02E001200FF003F83000DB
:1011C000FFF29CF800285ED0FFF75CFE41482E4AF3
:1011D000406A010080310B7E403213624B7E5362C5
:1011E0003D4B06789E624088D862C8690104090CAC
:1011F000002083009B181963401C0728F9DD01209B
:10120000FEF2BDFEFDF2FDFF6846FEF216F8214932
:101210003439886A05221206904388622548C03016
:10122000016889088900016022491E20886228001F
:1012300001F0ADF8FFF2E4F814493F220F20FFF768
:101240006BFE144925488C310860FFF293FF00F3D0
:1012500053FAFFF796FFFEF290F8FFF249FAFAF719
:10126000F7F80021012019F042FA6069FFF72FFF1B
:101270001B4801680B220904090C520489180160FB
:101280001848016830E049E040A20080FF030000F8
:101290001018000434A9008080A0008038B701C075
:1012A000EBEFEBFFE8EEEAFFFAFEFAFFF8ECEAFFFD
:1012B000FFFFFEFF40A4008000A8008098B901C095
:1012C000E0F80004E1F80004E2F80004E3F80004A8
:1012D000E4F800043CC7000400A6008001000300FD
:1012E00000AE008000210080420C91430160F3F7C2
:1012F00081FAFF4908680122D20610430860FD49BF
:1013000008690A0D10430861FB4819F07BF9F94898
:101310008030016B0322114301630120F8BDF0B559
:1013200004210C05F54ECD058A00921913681F049F
:101330003F0C2300002800D12B003B431360491CC5
:101340000729F1D9F0BDEA490420C03910B5086079
:101350000620F4F757F9EA480068C06B01F017F867
:1013600010BDF8B5002406008500E6484059002865
:101370007DD0F2F7B0F83106090E3702002800914F
:1013800036D0E14900980026FCF2FCFADF4901283A
:101390001CD14A69D84B0A3A13E0DA48A100283038
:1013A0004059401819680006000E38430143086888
:1013B0003A21415E8E19B24202DC002C57D01EE069
:1013C000641CD0484059A042E7D818E0CD48CA4A2A
:1013D00028304059126801240006000E38430243A9
:1013E00010683A22825E48690A3882423FDA06E093
:1013F000C4484159C64AD468A14200D24459C148A0
:101400004159091B4151C348BF4946590098FCF254
:10141000B9FA012820D100201AE0BA49B64B283188
:101420004A591B681106090E3943194309680423F8
:10143000498C121D5B1A9B079B0F59182CFC4CC240
:1014400001000000F00E010000040000FAFF4ECE83
:10145000B14B091D28335A51D205D20D09030A4355
:101460003260401CA042E2D309E00AE0AA49A2008F
:101470002831485980184851C005C00D30600120FE
:10148000F8BD0020F8BD10B50C00A0301100C37DE0
:10149000827D20000C30FEF2BEFC10BD70B506004F
:1014A0008966086F0C000D000188821D143430001D
:1014B0002DF03AFE0200296F2000FEF2C6FC2888BB
:1014C0002084F9F793FD60688078000905280CD125
:1014D000E069012149060843E0610A2128002170E2
:1014E00009210C30FEF288FC04E0220029003000C3
:1014F000FFF7C9FFE16901221203A8789143E16176
:1015000005F3B1FB2565E06270BD0100CA007D49AD
:1015100000207031511809687A4B7433D218126860
:10152000D206D20E01E0091D401C0B1DDB06DB0EAE
:101530009342F8D17047F7B582B001250E0017002D
:101540002AF0F2FB0190C020C45D380011F04FFB7F
:10155000022811D07549097981420DD015235B010C
:1015600072495843203942182C32E0008018030099
:10157000FF33B933181F06E06249E00074314318A5
:10158000624A091F40180C2E1AD101681B680E1DF3
:10159000F606DB06F60EDB0E9E4201D1002514E0B6
:1015A000029B12680326B6023243CE06F60E640191
:1015B000264332431360091D8906890E016004E049
:1015C0005B48EFF72FF8F4F73DFD01982AF0B0FBE8
:1015D000280005B0F0BDF8B5050000896F69441911
:1015E000206F00281ED0002F07D12AF09DFB504805
:1015F000401CEFF717F8F4F725FD260014362100FC
:101600003800FFF74BFF280031F0F7FD6034217FF1
:101610003A003000FFF78FFF002804D1280031F096
:1016200013FE0020F8BD0120F8BDF8B50500012724
:1016300000896E694419280031F0DFFD7C20015DCE
:10164000200032001430FFF776FF002803D1280075
:1016500031F0FAFD00273800F8BDF8B50500008923
:101660006E694419002E00D1FEE7206F2700143761
:10167000002834D021003000FFF710FF786881780F
:101680000909092902D101227C210A55317902294F
:1016900014D1807800090D2810D1206F20300178F6
:1016A00003290BD14178002908D1C0788006000FAA
:1016B0000AF3F2FE0AF301FF7C210855280031F0FD
:1016C0009CFD210030002DF04BFC002806D12800A5
:1016D00031F0BAFD0120F4F711FCEFE70120F8BD6D
:1016E000F8B50C0007008966086F0D001434002857
:1016F0007ED060606120C05D0A49C006400F400096
:10170000483117E0C0A80080C0A2008000A000807F
:10171000C0AE0080D8BD01C0F4FD02C03CCC0004C6
:10172000304D040038B701C04818000430420004AE
:1017300007000100095A21812988218420002030D6
:10174000417AAB78C9095B06C9015B0E1943417246
:10175000E261E9886184A888002806D060880004D6
:1017600003D4210028002DF014FE60682E0080783C
:101770000C360107890F012910D100090A2807D169
:10178000F9F716FC002801D0022104E0002102E054
:10179000082803D103213000FEF22EFB6068807818
:1017A0000107890F02290CD100090C2801D0042857
:1017B00007D1F9F7FBF8002803D002213000FEF230
:1017C0001BFBF9F7CBFB002815D009F0ACFE002875
:1017D00003D1F1F78AFE00280DD02200290038003D
:1017E000FFF751FE21787E2041550021300000E0B6
:1017F00025E0FEF201FBF9F7B1FB002807D009F064
:101800002CFE002803D0210028002DF0C2FD22006C
:1018100029003800FFF737FE2200290038002DF09C
:10182000C8FC298AA181698AE181F1F75EFE00285E
:1018300003D021003800F1F7FCFE01202565F8BD3A
:10184000F8B504000F000089666905191843024BBA
:1018500001000000EC12010000040000453A6B7D1D
:10186000002E06D12AF06AFAFF48EEF7E5FEF4F7FB
:10187000F3FB286F002824D02AF060FA00902000A3
:1018800031F0C5FC3A0029003000FFF733FF0EE0CD
:10189000200031F0E3FC00982AF054FA0120F4F71C
:1018A00037FB2AF04BFA0090200031F0B0FC290001
:1018B00030002DF05FFB0028EAD000982AF042FAB1
:1018C0000120F8BD7FB5040015000200E332511E6F
:1018D000E13001AE07C62200E032200000922A006B
:1018E000D830FEF2E4FA7FBD38B50400E034E27887
:1018F00000920A008030C16DA378806DFEF21DFE5B
:1019000038BD0200803210B5D36D926D0800FEF232
:1019100064F910BDD54A10B5126904231A40D44B9E
:101920005A64D44AFEF282FB10BDD048016989088E
:10193000890001610169CE4A526C1143016170470F
:10194000CA4880698006800F032801D101207047B2
:1019500000207047002801D10820704710207047F0
:10196000C249203108757047C34A8000821810B5FB
:1019700013688806800E0102040421430006014317
:10198000BE4803400B43136010BDBB4A8000801863
:1019900002688906890E0B0409060B43B8490A4000
:1019A0001A4302607047B44B10B5403B196880067B
:1019B000800E02020404224300060243AF480140A5
:1019C0001143196010BDAC4B403B19688006800E76
:1019D000020400060243AA480140114319607047FF
:1019E00010B50524200017F036FF01002000FEF29C
:1019F000C9F8200017F032FFFF2801D0FFF7D3FF0E
:101A0000200017F033FFFF2801D0FFF7DCFF10BDE7
:101A1000E03010B582780100C078824208D20A789E
:101A20004878824204D21BF080FD022801D10520B3
:101A300010BD002010BD10B501F0A6F910BD9148F1
:101A400010B58168090A0902816014F020FD10BDFB
:101A50008C4810B58168AA221143816014F018FDEA
:101A600010BD08B5694601F0FDFB002804D16B46A6
:101A700018705870987003E06B461878002804D1ED
:101A8000002031F01EEE012002E0012802D10020EA
:101A900026F021FB6B46187808BD0EB56B46187012
:101AA0005970009801A901F0B4FB002805D001A8E5
:101AB00031F00AEE012031F004EE0EBD1CB56B468C
:101AC00018705970009801A901F0B8FB002803D0E4
:101AD00001A831F0FEED012031F0FEED1CBD70B526
:101AE0002AF02CF9684C002125000B00283526002F
:101AF00050368A00A350491CAB500929B350F8DD79
:101B00002AF020F970BDF3B581B007002AF016F96C
:101B100000902DF04DF801003800FEF2D9FA5B4933
:101B20000A6880180860524802994030FEF2DDFAD7
:101B300002988400564800590068534D29592E00D8
:101B40005036002907D152493831095909682A000D
:101B50002832315111513159029A3B00FEF2E8FD11
:101B6000002804D100982AF0EDF80020FEBD30597D
:101B7000001D30512859401C285100982AF0E2F8E5
:101B80000120FEBD10B52AF0D9F83F4A00218B0094
:101B9000D358002B03D02AF0D5F8012010BD491CE2
:101BA0000929F4DD2AF0CEF8002010BD70B50189B6
:101BB0000C18216F250040691435002901D100203F
:101BC00070BD2100FFF774FC68688078000909285F
:101BD00001D1012101E06034217F2800FFF793FF4C
:101BE00070BD70B502891418226F25004069143544
:101BF000002A01D1002070BD0A002100FFF77AFD04
:101C00006034217F2800FFF77EFF70BDF8B5002506
